:100000000C94D7400C9406410C9406410C94064184
:100010000C9406410C9406410C9406410C94064144
:100020000C9406410C9406410C9406410C94064134
:100030000C9406410C94586B0C9406410C940641A8
:100040000C9406410C9406410C9406410C94064114
:100050000C9406410C9406410C9406410C94064104
:100060000C9406410C9469E20C9406410C9495E2C0
:100070000C9406410C94B6AB0C9406410C940641CA
:100080000C9406410C9406410C9406410C940641D4
:100090000C9406410C9406410C9406410C940641C4
:1000A0000C9406410C9406410C9406410C940641B4
:1000B0000C9406410C9406410C9406410C94F8688B
:1000C0000C9406410C9406410C9406410C94064194
:1000D0000C9406410C9406410C9406410C94064184
:1000E0000C9406415862FC62A0628662AD62646351
:1000F00064638662F6626463FF62046319631E636D
:10010000B762C062CE628662F16264636D62B2629F
:10011000236338634263646364634663507265704B
:100120006172696E6720666F7220736C6565703AE4
:1001300049276D20636F6D706C6574696E6720610F
:100140006E792020717565756564206D6F766573B5
:100150002E004368616E67696E672046696C616D49
:10016000656E743A202049276D20636F6D706C6551
:1001700074696E6720616E7920207175657565649C
:10018000206D6F7665732E00494E56414C494420D0
:10019000544F4F4C3A2020202020202049207265C7
:1001A000636569766564206120636F6D6D616E645F
:1001B000666F7220546F6F6C2023322C206275742E
:1001C000204920206F6E6C792068617665206F6E03
:1001D0006520546F6F6C2E2000494E56414C4944A7
:1001E00020434F4D4D414E443A202020204920725B
:1001F00065636569766564206120636F6D6D616E0E
:1002000064666F7220612068656174656420706C3B
:100210006174652C20627574204920646F6E2774A8
:100220002068617665206F6E6500492073617720D4
:100230006120676C6974636820696E206D7953442E
:1002400020636172642E2049662074686973206996
:100250007320746865206669727374206572726FAA
:10026000722C2074727974686973206D6F64656C88
:1002700020616761696E2E20202000492074696D1D
:100280006564206F7574207768696C652020206133
:100290007474656D7074696E6720746F2068656131
:1002A0007420206D792065787472756465722E00F3
:1002B000492074696D6564206F7574207768696C76
:1002C00065202020617474656D7074696E67207498
:1002D0006F206865617420206D7920706C61746690
:1002E0006F726D2E00507265706172696E67206664
:1002F0006F7220736C6565703A49276D20636F6F6C
:100300006C696E67206D792020202020206865614F
:100310007465727320616E6420676F696E67207404
:100320006F6D79207761697420706F736974696F7C
:100330006E2E004368616E67696E672046696C6166
:100340006D656E743A202049276D20676F696E676E
:1003500020746F206D792077616974706F73697490
:10036000696F6E2E0052657374617274696E6720D6
:10037000746865204275696C640054686520526534
:10038000706C6963617430720049276D2043616E3F
:1003900063656C6C696E672E2020202020506C6590
:1003A00061736520576169742E002000486561748F
:1003B0006572732073687574646F776E20202020D7
:1003C00064756520746F20696E6163746976697401
:1003D00079202020004578747275646572204F760C
:1003E000657268656174212020536F66747761724D
:1003F000652054656D70204C696D6974205265618B
:10040000636865642120506C65617365202020203D
:100410002053687574646F776E206F722052657315
:10042000746172740048656174696E672046616921
:100430006C75726521202020204D792065787472BA
:10044000756465727320617265206E6F7468656192
:1004500074696E672070726F7065726C792E2020DF
:1004600020436865636B206D7920636F6E6E6563F2
:1004700074696F6E730048656174696E67204661C8
:10048000696C75726521202020204D792065787473
:1004900072756465727320617265202020206C6F14
:1004A00073696E672074656D7065726174757265CD
:1004B0002E20436865636B206D7920636F6E6E65D7
:1004C0006374696F6E73004865617465722045726C
:1004D000726F72212020202020202049276D207259
:1004E000656164696E67206F7574206F6620207285
:1004F000616E67652074656D706572617475726593
:10050000732E20436865636B206D7920636F6E6E78
:10051000656374696F6E7300486561746572204528
:1005200072726F7221202020202020204D792074AB
:10053000656D706572617475726520726561647352
:10054000617265206661696C696E672120506C6517
:1005500061736520436865636B206D7920636F6EFE
:100560006E656374696F6E730093026900000069C1
:1005700000EE016900000069002601B801000000DA
:1005800000270555000000550020065500000055C5
:10059000002D085500000055004D0A55000000557B
:1005A00000400CAB000000AB002D095500000055C9
:1005B000002D085500000055004D0AAB0000005505
:1005C0000000000001C00D5500000055002D085628
:1005D0000100000000C00D20015311BC005B12B1EE
:1005E0000100000000C00DC80000001400C00DC8CC
:1005F0000000001400910E9001000014005A1090A9
:100600000100001400C00D200300000000C805C850
:100610000000001400C805C80000001400C805C888
:100620000000001400DD04B004000014007505C8CB
:1006300000000014007505C800000014007505C80E
:1006400000000014009704B00400000000A9085541
:100650000000005500B807550000005500B909AB6F
:10066000000000AB007D06550000005500C8055590
:100670000000005500B807AB000000AB00C80555EE
:100680000000005500DD04550000005500C8055568
:100690000000005500B8075500000055007D0656C3
:1006A00001000000002D085500000055003F0355D3
:1006B0000000005500B9095500000055003F0355E2
:1006C0000000005500FA0C5500000055003F03558E
:1006D0000000005500B9095500000055003F0355C2
:1006E00000000055002D095500000055003F03553E
:1006F0000000005500EA0A5500000055003F035570
:100700000000005500B909AB000000000053442070
:10071000436172642052656D6F766564007A7A7AFF
:10072000797979797878787878777777777676764F
:100730007675757575757474747474737373737278
:1007400072727272717171717170707070706F6F9E
:100750006F6F6F6E6E6E6E6E6D6D6D6D6D6D6C6CC0
:100760006C6C6C6B6B6B6B6B6A6A6A6A6A6A6969E0
:1007700069696969686868686867676767676766FD
:100780006666666666656565656565646464646419
:100790006464636363636363626262626262626130
:1007A0006161616161606060606060605F5F5F5F48
:1007B0005F5F5F5E5E5E5E5E5E5E5D5D5D5D5D5D5C
:1007C0005D5C5C5C5C5C5C5C5C5B5B5B5B5B5B5B6F
:1007D0005A5A5A5A5A5A5A5A595959595959595981
:1007E0005858585858585858575757575757575791
:1007F00056565656565656565555555555555555A1
:1008000055545454545454545454535353535353AD
:1008100053535352525252525252525251515151B9
:1008200051515151515150505050505050505050C2
:100830004F4F4F4F4F4F4F4F4F4F4E4E4E4E4E4ECE
:100840004E4E4E4E4D4D4D4D4D4D4D4D4D4D4C4CD6
:100850004C4C4C4C4C4C4C4C4C4B4B4B4B4B4B4BDF
:100860004B4B4B4B4A4A4A4A4A4A4A4A4A4A4A4AE4
:1008700049494949494949494949494948484848EC
:1008800048484848484848484747474747474747F0
:1008900047474747464646464646464646464646F4
:1008A00046454545454545454545454545454444F9
:1008B00044444444444444444444444343434343FD
:1008C00043434343434343434342424242424242FF
:1008D0004242424242424242414141414141414100
:1008E0004141414141414040404040404040404002
:1008F0004040404040403F3F3F3F3F3F3F3F3F3F02
:100900003F3F3F3F3F3F3E3E3E3E3E3E3E3E3E3E01
:100910003E3E3E3E3E3E3D3D3D3D3D3D3D3D3D3D01
:100920003D3D3D3D3D3D3D3C3C3C3C3C3C3C3C3C00
:100930003C3C3C3C3C3C3C3C3B3B3B3B3B3B3B3BFF
:100940003B3B3B3B3B3B3B3B3B3B3A3A3A3A3A3AFD
:100950003A3A3A3A3A3A3A3A3A3A3A3A39393939FB
:1009600039393939393939393939393939393939F7
:1009700038383838383838383838383838383838F7
:1009800038383838373737373737373737373737F3
:1009900037373737373737373636363636363636EF
:1009A00036363636363636363636363636363535E9
:1009B00035353535353535353535353535353535E7
:1009C00035353535343434343434343434343434E3
:1009D00034343434343434343434343333333333DC
:1009E00033333333333333333333333333333333D7
:1009F00033333332323232323232323232323232D4
:100A000032323232323232323232323231313131CA
:100A100031313131313131313131313131313131C6
:100A200031313131313130303030303030303030C0
:100A300030303030303030303030303030303030B6
:100A4000302F2F2F2F2F2F2F2F2F2F2F2F2F2F2FB5
:100A50002F2F2F2F2F2F2F2F2F2F2F2F2F2F2E2EA8
:100A60002E2E2E2E2E2E2E2E2E2E2E2E2E2E2E2EA6
:100A70002E2E2E2E2E2E2E2E2E2E2E2D2D2D2D2D9B
:100A80002D2D2D2D2D2D2D2D2D2D2D2D2D2D2D2D96
:100A90002D2D2D2D2D2D2D2D2D2D2C2C2C2C2C2C8C
:100AA0002C2C2C2C2C2C2C2C2C2C2C2C2C2C2C2C86
:100AB0002C2C2C2C2C2C2C2C2C2C2B2B2B2B2B2B7C
:100AC0002B2B2B2B2B2B2B2B2B2B2B2B2B2B2B2B76
:100AD0002B2B2B2B2B2B2B2B2B2B2B2B2A2A2A2A6A
:100AE0002A2A2A2A2A2A2A2A2A2A2A2A2A2A2A2A66
:100AF0002A2A2A2A2A2A2A2A2A2A2A2A2A2A2A2A56
:100B00002929292929292929292929292929292955
:100B10002929292929292929292929292929292945
:100B20002929292929282828282828282828282840
:100B30002828282828282828282828282828282835
:100B40002828282828282828282828282727272729
:100B50002727272727272727272727272727272725
:100B60002727272727272727272727272727272715
:100B70002727272727262626262626262626262610
:100B80002626262626262626262626262626262605
:100B900026262626262626262626262626262626F5
:100BA00025252525252525252525252525252525F5
:100BB00025252525252525252525252525252525E5
:100BC00025252525252525252525252525252424D7
:100BD00024242424242424242424242424242424D5
:100BE00024242424242424242424242424242424C5
:100BF00024242424242424242424242424242323B7
:100C000023232323232323232323232323232323B4
:100C100023232323232323232323232323232323A4
:100C20002323232323232323232323232323232394
:100C30002322222222222222222222222222222293
:100C40002222222222222222222222222222222284
:100C50002222222222222222222222222222222274
:100C6000222222222222222121212121212121216D
:100C70002121212121212121212121212121212164
:100C80002121212121212121212121212121212154
:100C90002121212121212121212121212121212144
:100CA0002120202020202020202020202020202043
:100CB0002020202020202020202020202020202034
:100CC0002020202020202020202020202020202024
:100CD00020202020202020202020202020201F1F16
:100CE0001F1F1F1F1F1F1F1F1F1F1F1F1F1F1F1F14
:100CF0001F1F1F1F1F1F1F1F1F1F1F1F1F1F1F1F04
:100D00001F1F1F1F1F1F1F1F1F1F1F1F1F1F1F1FF3
:100D10001F1F1F1F1F1F1F1F1F1F1F1F1F1E000022
:100D200000000000000000000000000000000000C3
:100D300000000000000000000000000000000000B3
:100D400000000000000000000000000000000000A3
:100D50000000000000000000000000000000127A07
:100D60005F76E4729B6F826C9369CC662964A8619C
:100D7000465F025DD85AC758CE56EB541D53615199
:100D8000B84F204E984C1F4BB44957480647C145B1
:100D90008844594335421B410940013F013E093D0A
:100DA000193C303B4D3A72399D38CE3705374136C4
:100DB0008335CA3415346633BB3215327231D430C0
:100DC0003A30A32F102F812EF52D6C2DE62C642C9C
:100DD000E42B672BED2A762A012A8E291E29B128B9
:100DE0004528DC2775271027AD264C26ED258F25B5
:100DF0003425DA2482242B24D62383233123E122B1
:100E000092224422F821AD2163211B21D3208D2081
:100E100048200520C21F811F401F011FC21E851EC2
:100E2000481E0C1ED21D981D5F1D271DEF1CB91CEE
:100E3000831C4E1C1A1CE71BB41B821B511B201B5E
:100E4000F11AC11A931A651A371A0B1ADF19B31956
:100E500088195E1934190A19E118B91891186A1815
:100E600043181D18F717D217AD17881764174017C6
:100E70001D17FA16D816B616941673165216321691
:100E80001216F215D315B4159515771558153B158F
:100E90001D150015E414C714AB148F1474145814E2
:100EA0003D1423140814EE13D413BB13A113881399
:100EB0006F1356133E1326130E13F612DF12C812C9
:100EC000B1129A1283126D12571241122B1216127E
:100ED0000012EB11D611C111AD11991184117011CD
:100EE0005C114911351122110F11FC10E910D610B7
:100EF000C410B2109F108D107B106A10581047104C
:100F00003510241013100210F20FE10FD10FC00F93
:100F1000B00FA00F900F800F710F610F520F420F93
:100F2000330F240F150F060FF70EE90EDA0ECC0E55
:100F3000BE0EAF0EA10E930E850E780E6A0E5C0EDD
:100F40004F0E420E340E270E1A0E0D0E000EF30D2C
:100F5000E70DDA0DCE0DC10DB50DA90D9C0D900D4F
:100F6000840D780D6C0D610D550D490D3E0D320D42
:100F7000270D1C0D100D050DFA0CEF0CE40CD90C0F
:100F8000CF0CC40CB90CAF0CA40C9A0C8F0C850CB4
:100F90007B0C710C670C5D0C530C490C3F0C350C31
:100FA0002B0C220C180C0E0C050CFB0BF20BE90B96
:100FB000E00BD60BCD0BC40BBB0BB20BA90BA00BDC
:100FC000970B8F0B860B7D0B750B6C0B630B5B0B01
:100FD000530B4A0B420B3A0B310B290B210B190B0C
:100FE000110B090B010BF90AF10AE90AE20ADA0A04
:100FF000D20ACA0AC30ABB0AB40AAC0AA50A9D0AE5
:10100000960A8F0A870A800A790A720A6B0A640AAA
:101010005D0A560A4F0A480A410A3A0A330A2C0A5C
:10102000250A1F0A180A110A0B0A040AFE09F70901
:10103000F109EA09E409DD09D709D109CA09C40996
:10104000BE09B809B109AB09A5099F099909930916
:101050008D09870981097B0975096F096A09640986
:101060005E09580953094D09470942093C093609E7
:1010700031092B09260920091B09160910090B093A
:1010800005090009FB08F608F008EB08E608E10886
:10109000DC08D608D108CC08C708C208BD08B808C3
:1010A000B308AE08A908A408A0089B0896089108F0
:1010B0008C08870883087E087908750870086B0813
:1010C000670862085D085908540850084B0847082B
:1010D00042083E083908350830082C08280823083B
:1010E0001F081B08160812080E080A080508010840
:1010F000FD07F907F507F107EC07E807E407E00744
:10110000DC07D807D407D007CC07C807C407C00737
:10111000BC07B807B407B107AD07A907A507A10722
:101120009D079A07960792078E078B078707830705
:101130007F077C077807740771076D076A076607E2
:1011400062075F075B075807540751074D074A07B7
:10115000460743073F073C073807350732072E0786
:101160002B072807240721071D071A07170714074D
:1011700010070D070A07070703070007FD06FA0611
:10118000F706F306F006ED06EA06E706E406E106D2
:10119000DD06DA06D706D406D106CE06CB06C8068B
:1011A000C506C206BF06BC06B906B606B306B0063B
:1011B000AD06AA06A806A506A2069F069C069906E5
:1011C0009606940691068E068B068806850683068B
:1011D00080067D067A067806750672066F066D062D
:1011E0006A066706650662065F065D065A065706CA
:1011F0005506520650064D064A0648064506430661
:1012000040063D063B0638063606330631062E06F6
:101210002C0629062706240622061F061D061B0685
:1012200018061606130611060E060C060A06070611
:10123000050602060006FE05FB05F905F705F4059F
:10124000F205F005ED05EB05E905E705E405E20526
:10125000E005DE05DB05D905D705D505D205D005A6
:10126000CE05CC05C905C705C505C305C105BF0524
:10127000BC05BA05B805B605B405B205B005AD059F
:10128000AB05A905A705A505A305A1059F059D0516
:101290009B05990597059505930591058E058C0588
:1012A0008A05880586058405820580057E057C05FE
:1012B0007B05790577057505730571056F056D0566
:1012C0006B056905670565056305610560055E05D4
:1012D0005C055A05580556055405520551054F053C
:1012E0004D054B05490547054605440542054005A2
:1012F0003E053C053B053905370535053405320506
:1013000030052E052D052B05290527052605240565
:10131000220520051F051D051B05190518051605C5
:101320001405130511050F050E050C050A05090521
:1013300007050505040502050005FF04FD04FC047E
:10134000FA04F804F704F504F304F204F004EF04DB
:10135000ED04EB04EA04E804E704E504E404E20431
:10136000E004DF04DD04DC04DA04D904D704D60485
:10137000D404D304D104D004CE04CD04CB04C904D6
:10138000C804C604C504C404C204C104BF04BE0426
:10139000BC04BB04B904B804B604B504B304B20475
:1013A000B004AF04AE04AC04AB04A904A804A604C2
:1013B000A504A404A204A1049F049E049D049B040C
:1013C0009A04980497049604940493049204900455
:1013D0008F048E048C048B0489048804870485049C
:1013E00084048304810480047F047D047C047B04E2
:1013F0007904780477047604740473047204700426
:101400006F046E046D046B046A0469046704660467
:10141000650464046204610460045F045D045C04A8
:101420005B045A04580457045604550453045204E8
:10143000510450044F044D044C044B044A04480426
:1014400047044604450444044304410440043F0463
:101450003E043D043B043A0439043804370436049E
:10146000340433043204310430042F042E042C04D9
:101470002B042A0429042804270426042404230412
:101480002204210420041F041E041D041C041A0449
:101490001904180417041604150414041304120480
:1014A000110410040E040D040C040B040A040904B6
:1014B00008040704060405040404030402040104E8
:1014C0000004FE03FD03FC03FB03FA03F903F80326
:1014D000F703F603F503F403F303F203F103F00358
:1014E000EF03EE03ED03EC03EB03EA03E903E80388
:1014F000E703E603E503E403E303E203E103E003B8
:10150000DF03DE03DD03DC03DB03DA03D903D803E7
:10151000D703D603D503D403D303D203D203D10315
:10152000D003CF03CE03CD03CC03CB03CA03C9033F
:10153000C803C703C603C503C403C303C203C2036E
:10154000C103C003BF03BE03BD03BC03BB03BA0397
:10155000B903B803B703B703B603B503B403B303C2
:10156000B203B103B003AF03AF03AE03AD03AC03EB
:10157000AB03AA03A903A803A703A703A603A50314
:10158000A403A303A203A103A103A0039F039E033B
:101590009D039C039B039B039A0399039803970362
:1015A0009603950395039403930392039103900389
:1015B00090038F038E038D038C038B038B038A03AD
:1015C00089038803870387038603850384038303D2
:1015D00082038203810380037F037E037E037D03F6
:1015E0007C037B037A037A03790378037703770319
:1015F000760375037403730373037203710370033B
:1016000070036F036E036D036C036C036B036A035B
:10161000690369036803670366036603650364037C
:101620006303630362036103600360035F035E039C
:101630005D035D035C035B035A035A0359035803BC
:1016400057035703560355035503540353035203DB
:101650005203510350034F034F034E034D034D03F9
:101660004C034B034A034A03490348034803470317
:101670004603460345034403430343034203410334
:10168000410340033F033F033E033D033D033C034F
:101690003B033A033A03390338033803370336036D
:1016A0003603350334033403330332033203310387
:1016B000300330032F032E032E032D032C032C03A2
:1016C0002B032A032A0329032803280327032603BD
:1016D00026032503250324032303230322032103D5
:1016E000210320031F031F031E031D031D031C03EF
:1016F0001C031B031A031A03190318031803170307
:10170000170316031503150314031303130312031E
:1017100012031103100310030F030E030E030D0336
:101720000D030C030B030B030A030A03090308034D
:101730000803070307030603050305030403040363
:10174000030302030203010301030003FF02FF027C
:10175000FE02FE02FD02FD02FC02FB02FB02FA0297
:10176000FA02F902F802F802F702F702F602F602AC
:10177000F502F402F402F302F302F202F202F102C1
:10178000F002F002EF02EF02EE02EE02ED02ED02D5
:10179000EC02EB02EB02EA02EA02E902E902E802E9
:1017A000E702E702E602E602E502E502E402E402FD
:1017B000E302E302E202E102E102E002E002DF0210
:1017C000DF02DE02DE02DD02DD02DC02DC02DB0221
:1017D000DA02DA02D902D902D802D802D702D70235
:1017E000D602D602D502D502D402D402D302D30245
:1017F000D202D202D102D002D002CF02CF02CE0258
:10180000CE02CD02CD02CC02CC02CB02CB02CA0268
:10181000CA02C902C902C802C802C702C702C60278
:10182000C602C502C502C402C402C302C302C20288
:10183000C202C102C102C002C002BF02BF02BE0298
:10184000BE02BD02BD02BC02BC02BB02BB02BA02A8
:10185000BA02B902B902B802B802B702B702B602B8
:10186000B602B502B502B502B402B402B302B302C5
:10187000B202B202B102B102B002B002AF02AF02D4
:10188000AE02AE02AD02AD02AC02AC02AC02AB02E3
:10189000AB02AA02AA02A902A902A802A802A702F0
:1018A000A702A602A602A602A502A502A402A402FD
:1018B000A302A302A202A202A102A102A002A0020C
:1018C000A0029F029F029E029E029D029D029C0218
:1018D0009C029C029B029B029A029A029902990224
:1018E0009802980298029702970296029602950231
:1018F000950295029402940293029302920292023C
:10190000910291029102900290028F028F028E0248
:101910008E028E028D028D028C028C028B028B0253
:101920008B028A028A02890289028902880288025D
:101930008702870286028602860285028502840269
:101940008402840283028302820282028102810273
:101950008102800280027F027F027F027E027E027D
:101960007D027D027D027C027C027B027B027B0287
:101970007A027A0279027902790278027802770291
:10198000770277027602760275027502750274029A
:1019900074027302730273027202720271027102A4
:1019A0007102700270026F026F026F026E026E02AD
:1019B0006E026D026D026C026C026C026B026B02B5
:1019C0006A026A026A0269026902690268026802BE
:1019D00067026702670266026602650265026502C7
:1019E00064026402640263026302630262026202CE
:1019F0006102610261026002600260025F025F02D6
:101A00005E025E025E025D025D025D025C025C02DD
:101A10005C025B025B025A025A025A0259025902E4
:101A200059025802580258025702570256025602EB
:101A300056025502550255025402540254025302F2
:101A400053025302520252025102510251025002F9
:101A5000500250024F024F024F024E024E024E02FF
:101A60004D024D024D024C024C024C024B024B0205
:101A70004B024A024A02490249024902480248020C
:101A80004802470247024702460246024602450212
:101A90004502450244024402440243024302430217
:101AA000420242024202410241024102400240021D
:101AB00040023F023F023F023E023E023E023D0222
:101AC0003D023D023C023C023C023B023B023B0227
:101AD0003A023A023A02390239023902390238022C
:101AE000380238023702370237023602360236022F
:101AF0003502350235023402340234023302330235
:101B00003302320232023202310231023102310238
:101B10003002300230022F022F022F022E022E023C
:101B20002E022D022D022D022C022C022C022C0240
:101B30002B022B022B022A022A022A022902290244
:101B40002902280228022802280227022702270247
:101B5000260226022602250225022502250224024B
:101B6000240224022302230223022202220222024E
:101B700022022102210221022002200220021F0251
:101B80001F021F021F021E021E021E021D021D0254
:101B90001D021D021C021C021C021B021B021B0256
:101BA0001B021A021A021A02190219021902180259
:101BB000180218021802170217021702160216025C
:101BC000160216021502150215021402140214025E
:101BD000140213021302130213021202120212025F
:101BE00011021102110211021002100210020F0262
:101BF0000F020F020F020E020E020E020D020D0264
:101C00000D020D020C020C020C020C020B020B0264
:101C10000B020A020A020A020A0209020902090266
:101C20000902080208020802070207020702070267
:101C30000602060206020602050205020502050268
:101C4000040204020402030203020302030202026A
:101C5000020202020202010201020102010200026A
:101C6000000200020002FF01FF01FF01FE01FE0170
:101C7000FE01FE01FD01FD01FD01FD01FC01FC0174
:101C8000FC01FC01FB01FB01FB01FB01FA01FA0174
:101C9000FA01FA01F901F901F901F901F801F80174
:101CA000F801F801F701F701F701F701F601F60174
:101CB000F601F601F501F501F501F501F401F40174
:101CC000F401F401F301F301F301F301F201F20174
:101CD000F201F201F101F101F101F101F001F00174
:101CE000F001F001EF01EF01EF01EF01EE01EE0174
:101CF000EE01EE01ED01ED01ED01ED01EC01EC0174
:101D0000EC01EC01EB01EB01EB01EB01EA01EA0173
:101D1000EA01EA01E901E901E901E901E901E80172
:101D2000E801E801E801E701E701E701E701E60171
:101D3000E601E601E601E501E501E501E501E40171
:101D4000E401E401E401E401E301E301E301E3016F
:101D5000E201E201E201E201E101E101E101E1016F
:101D6000E101E001E001E001E001DF01DF01DF016D
:101D7000DF01DE01DE01DE01DE01DE01DD01DD016C
:101D8000DD01DD01DC01DC01DC01DC01DC01DB016A
:101D9000DB01DB01DB01DA01DA01DA01DA01D90169
:101DA000D901D901D901D901D801D801D801D80167
:101DB000D701D701D701D701D701D601D601D60166
:101DC000D601D501D501D501D501D501D401D40164
:101DD000D401D401D401D301D301D301D301D20161
:101DE000D201D201D201D201D101D101D101D1015F
:101DF000D001D001D001D001D001CF01CF01CF015E
:101E0000CF01CF01CE01CE01CE01CE01CD01CD015A
:101E1000CD01CD01CD01CC01CC01CC01CC01CC0157
:101E2000CB01CB01CB01CB01CB01CA01CA01CA0155
:101E3000CA01C901C901C901C901C901C801C80153
:101E4000C801C801C801C701C701C701C701C7014F
:101E5000C601C601C601C601C601C501C501C5014D
:101E6000C501C401C401C401C401C401C301C3014B
:101E7000C301C301C301C201C201C201C201C20147
:101E8000C101C101C101C101C101C001C001C00145
:101E9000C001C001BF01BF01BF01BF01BF01BE0141
:101EA000BE01BE01BE01BE01BD01BD01BD01BD013E
:101EB000BD01BC01BC01BC01BC01BC01BB01BB013B
:101EC000BB01BB01BB01BA01BA01BA01BA01BA0137
:101ED000BA01B901B901B901B901B901B801B80133
:101EE000B801B801B801B701B701B701B701B7012F
:101EF000B601B601B601B601B601B501B501B5012D
:101F0000B501B501B401B401B401B401B401B40127
:101F1000B301B301B301B301B301B201B201B20124
:101F2000B201B201B101B101B101B101B101B1011F
:101F3000B001B001B001B001B001AF01AF01AF011C
:101F4000AF01AF01AE01AE01AE01AE01AE01AE0117
:101F5000AD01AD01AD01AD01AD01AC01AC01AC0114
:101F6000AC01AC01AC01AB01AB01AB01AB01AB010E
:101F7000AA01AA01AA01AA01AA01AA01A901A9010B
:101F8000A901A901A901A801A801A801A801A80106
:101F9000A801A701A701A701A701A701A601A60102
:101FA000A601A601A601A601A501A501A501A501FD
:101FB000A501A501A401A401A401A401A401A301F8
:101FC000A301A301A301A301A301A201A201A201F4
:101FD000A201A201A201A101A101A101A101A101EE
:101FE000A001A001A001A001A001A0019F019F01EB
:101FF0009F019F019F019F019E019E019E019E01E5
:102000009E019E019D019D019D019D019D019D01DE
:102010009C019C019C019C019C019C019B019B01DA
:102020009B019B019B019B019A019A019A019A01D4
:102030009A019A01990199019901990199019801CF
:1020400098019801980198019801970197019701CB
:1020500097019701970197019601960196019601C4
:1020600096019601950195019501950195019501BE
:1020700094019401940194019401940193019301BA
:1020800093019301930193019201920192019201B4
:1020900092019201910191019101910191019101AE
:1020A00090019001900190019001900190018F01A9
:1020B0008F018F018F018F018F018E018E018E01A3
:1020C0008E018E018E018D018D018D018D018D019D
:1020D0008D018D018C018C018C018C018C018C0196
:1020E0008B018B018B018B018B018B018A018A0192
:1020F0008A018A018A018A018A018901890189018B
:102100008901890189018801880188018801880184
:10211000880188018701870187018701870187017D
:102120008601860186018601860186018601850178
:102130008501850185018501850185018401840171
:10214000840184018401840183018301830183016B
:102150008301830183018201820182018201820164
:10216000820182018101810181018101810181015D
:1021700080018001800180018001800180017F0158
:102180007F017F017F017F017F017F017E017E0151
:102190007E017E017E017E017E017D017D017D014A
:1021A0007D017D017D017D017C017C017C017C0143
:1021B0007C017C017C017B017B017B017B017B013C
:1021C0007B017B017A017A017A017A017A017A0135
:1021D0007A0179017901790179017901790179012E
:1021E0007801780178017801780178017801770128
:1021F0007701770177017701770177017601760121
:102200007601760176017601760175017501750119
:102210007501750175017501740174017401740112
:10222000740174017401730173017301730173010B
:102230007301730173017201720172017201720103
:1022400072017201710171017101710171017101FC
:1022500071017001700170017001700170017001F5
:1022600070016F016F016F016F016F016F016F01ED
:102270006E016E016E016E016E016E016E016D01E7
:102280006D016D016D016D016D016D016D016C01DF
:102290006C016C016C016C016C016C016C016B01D7
:1022A0006B016B016B016B016B016B016A016A01D0
:1022B0006A016A016A016A016A016A0169016901C8
:1022C00069016901690169016901680168016801C1
:1022D00068016801680168016801670167016701B9
:1022E00067016701670167016701660166016601B1
:1022F00066016601660166016601650165016501A9
:1023000065016501650165016501640164016401A0
:102310006401640164016401630163016301630199
:102320006301630163016301620162016201620191
:102330006201620162016201610161016101610189
:102340006101610161016101600160016001600181
:1023500060016001600160015F015F015F015F0179
:102360005F015F015F015F015F015E015E015E0170
:102370005E015E015E015E015E015D015D015D0168
:102380005D015D015D015D015D015C015C015C0160
:102390005C015C015C015C015C015B015B015B0158
:1023A0005B015B015B015B015B015B015A015A014F
:1023B0005A015A015A015A015A015A015901590147
:1023C000590159015901590159015901580158013F
:1023D0005801580158015801580158015801570136
:1023E000570157015701570157015701570156012E
:1023F0005601560156015601560156015601560125
:10240000550155015501550155015501550155011C
:102410005401540154015401540154015401540114
:10242000540153015301530153015301530153010B
:102430005301530152015201520152015201520102
:1024400052015201510151015101510151015101FA
:1024500051015101510150015001500150015001F1
:1024600050015001500150014F014F014F014F01E8
:102470004F014F014F014F014F014E014E014E01DF
:102480004E014E014E014E014E014E014D014D01D6
:102490004D014D014D014D014D014D014D014C01CD
:1024A0004C014C014C014C014C014C014C014C01C4
:1024B0004B014B014B014B014B014B014B014B01BC
:1024C0004B014A014A014A014A014A014A014A01B3
:1024D0004A014A01490149014901490149014901AA
:1024E00049014901490149014801480148014801A0
:1024F0004801480148014801480147014701470197
:10250000470147014701470147014701460146018D
:102510004601460146014601460146014601460183
:10252000450145014501450145014501450145017B
:102530004501440144014401440144014401440172
:102540004401440144014301430143014301430168
:10255000430143014301430142014201420142015F
:102560004201420142014201420142014101410155
:10257000410141014101410141014101410141014B
:102580004001400140014001400140014001400143
:1025900040013F013F013F013F013F013F013F013A
:1025A0003F013F013F013E013E013E013E013E0130
:1025B0003E013E013E013E013E013D013D013D0126
:1025C0003D013D013D013D013D013D013D013C011C
:1025D0003C013C013C013C013C013C013C013C0113
:1025E0003C013B013B013B013B013B013B013B010A
:1025F0003B013B013B013A013A013A013A013A0100
:102600003A013A013A013A013A01390139013901F5
:1026100039013901390139013901390139013901EA
:1026200038013801380138013801380138013801E2
:1026300038013801370137013701370137013701D8
:1026400037013701370137013601360136013601CE
:1026500036013601360136013601360136013501C3
:1026600035013501350135013501350135013501BA
:1026700035013401340134013401340134013401B1
:1026800034013401340134013301330133013301A6
:10269000330133013301330133013301320132019C
:1026A0003201320132013201320132013201320192
:1026B0003201310131013101310131013101310189
:1026C000310131013101310130013001300130017E
:1026D0003001300130013001300130012F012F0174
:1026E0002F012F012F012F012F012F012F012F016A
:1026F0002F012E012E012E012E012E012E012E0161
:102700002E012E012E012E012D012D012D012D0155
:102710002D012D012D012D012D012D012D012C014A
:102720002C012C012C012C012C012C012C012C0141
:102730002C012C012B012B012B012B012B012B0137
:102740002B012B012B012B012B012B012A012A012B
:102750002A012A012A012A012A012A012A012A0121
:102760002A01290129012901290129012901290118
:10277000290129012901290128012801280128010D
:102780002801280128012801280128012801280101
:1027900027012701270127012701270127012701F9
:1027A00027012701270126012601260126012601EE
:1027B00026012601260126012601260126012501E2
:1027C00025012501250125012501250125012501D9
:1027D00025012501240124012401240124012401CF
:1027E00024012401240124012401240123012301C3
:1027F00023012301230123012301230123012301B9
:1028000023012301220122012201220122012201AE
:1028100022012201220122012201220121012101A2
:102820002101210121012101210121012101210198
:10283000210121012001200120012001200120018E
:102840002001200120012001200120011F011F0182
:102850001F011F011F011F011F011F011F011F0178
:102860001F011F011E011E011E011E011E011E016E
:102870001E011E011E011E011E011E011D011D0162
:102880001D011D011D011D011D011D011D011D0158
:102890001D011D011C011C011C011C011C011C014E
:1028A0001C011C011C011C011C011C011C011B0141
:1028B0001B011B011B011B011B011B011B011B0138
:1028C0001B011B011B011A011A011A011A011A012D
:1028D0001A011A011A011A011A011A011A011A0120
:1028E0001901190119011901190119011901190118
:1028F000190119011901190119011801180118010B
:1029000018011801180118011801180118011801FF
:1029100018011701170117011701170117011701F6
:1029200017011701170117011701170116011601E9
:1029300016011601160116011601160116011601DF
:1029400016011601160115011501150115011501D4
:1029500015011501150115011501150115011501C7
:1029600014011401140114011401140114011401BF
:1029700014011401140114011401130113011301B2
:1029800013011301130113011301130113011301A7
:10299000130113011201120112011201120112019D
:1029A000120112011201120112011201120112018F
:1029B0001101110111011101110111011101110187
:1029C000110111011101110111011001100110017A
:1029D000100110011001100110011001100110016F
:1029E0001001100110010F010F010F010F010F0164
:1029F0000F010F010F010F010F010F010F010F0157
:102A00000E010E010E010E010E010E010E010E014E
:102A10000E010E010E010E010E010E010D010D0140
:102A20000D010D010D010D010D010D010D010D0136
:102A30000D010D010D010D010C010C010C010C012A
:102A40000C010C010C010C010C010C010C010C011E
:102A50000C010C010B010B010B010B010B010B0114
:102A60000B010B010B010B010B010B010B010B0106
:102A70000A010A010A010A010A010A010A010A01FE
:102A80000A010A010A010A010A010A0109010901F0
:102A900009010901090109010901090109010901E6
:102AA00009010901090109010801080108010801DA
:102AB00008010801080108010801080108010801CE
:102AC00008010801080107010701070107010701C3
:102AD00007010701070107010701070107010701B6
:102AE00007010601060106010601060106010601AD
:102AF000060106010601060106010601060106019E
:102B00000501050105010501050105010501050195
:102B10000501050105010501050105010401040187
:102B2000040104010401040104010401040104017D
:102B30000401040104010401040103010301030170
:102B40000301030103010301030103010301030165
:102B50000301030103010301020102010201020159
:102B6000020102010201020102010201020102014D
:102B70000201020102010101010101010101010142
:102B80000101010101010101010101010101010135
:102B9000010101010001000100010001000100012B
:102BA000000100010001000100010001000100011D
:102BB0000001FF00FF00FF00FF00FF00FF00FF001B
:102BC000FF00FF00FF00FF00FF00FF00FF00FF000D
:102BD000FF00FE00FE00FE00FE00FE00FE00FE0004
:102BE000FE00FE00FE00FE00FE00FE00FE00FE00F5
:102BF000FD00FD00FD00FD00FD00FD00FD00FD00ED
:102C0000FD00FD00FD00FD00FD00FD00FD00FD00DC
:102C1000FC00FC00FC00FC00FC00FC00FC00FC00D4
:102C2000FC00FC00FC00FC00FC00FC00FC00FC00C4
:102C3000FB00FB00FB00FB00FB00FB00FB00FB00BC
:102C4000FB00FB00FB00FB00FB00FB00FB00FB00AC
:102C5000FA00FA00FA00FA00FA00FA00FA00FA00A4
:102C6000FA00FA00FA00FA00FA00FA00FA00FA0094
:102C7000F900F900F900F900F900F900F900F9008C
:102C8000F900F900F900F900F900F900F900F9007C
:102C9000F800F800F800F800F800F800F800F80074
:102CA000F800F800F800F800F800F800F800F80064
:102CB000F700F700F700F700F700F700F700F7005C
:102CC000F700F700F700F700F700F700F700F7004C
:102CD000F600F600F600F600F600F600F600F60044
:102CE000F600F600F600F600F600F600F600F60034
:102CF000F600F500F500F500F500F500F500F5002B
:102D0000F500F500F500F500F500F500F500F5001B
:102D1000F500F400F400F400F400F400F400F40012
:102D2000F400F400F400F400F400F400F400F40003
:102D3000F400F400F300F300F300F300F300F300F9
:102D4000F300F300F300F300F300F300F300F300EB
:102D5000F300F300F300F200F200F200F200F200E0
:102D6000F200F200F200F200F200F200F200F200D3
:102D7000F200F200F200F200F100F100F100F100C7
:102D8000F100F100F100F100F100F100F100F100BB
:102D9000F100F100F100F100F100F100F000F000AD
:102DA000F000F000F000F000F000F000F000F000A3
:102DB000F000F000F000F000F000F000F000EF0094
:102DC000EF00EF00EF00EF00EF00EF00EF00EF008B
:102DD000EF00EF00EF00EF00EF00EF00EF00EF007B
:102DE000EE00EE00EE00EE00EE00EE00EE00EE0073
:102DF000EE00EE00EE00EE00EE00EE00EE00EE0063
:102E0000EE00EE00ED00ED00ED00ED00ED00ED0058
:102E1000ED00ED00ED00ED00ED00ED00ED00ED004A
:102E2000ED00ED00ED00ED00EC00EC00EC00EC003E
:102E3000EC00EC00EC00EC00EC00EC00EC00EC0032
:102E4000EC00EC00EC00EC00EC00EC00EB00EB0024
:102E5000EB00EB00EB00EB00EB00EB00EB00EB001A
:102E6000EB00EB00EB00EB00EB00EB00EB00EB000A
:102E7000EA00EA00EA00EA00EA00EA00EA00EA0002
:102E8000EA00EA00EA00EA00EA00EA00EA00EA00F2
:102E9000EA00EA00E900E900E900E900E900E900E8
:102EA000E900E900E900E900E900E900E900E900DA
:102EB000E900E900E900E900E900E800E800E800CD
:102EC000E800E800E800E800E800E800E800E800C2
:102ED000E800E800E800E800E800E800E800E700B3
:102EE000E700E700E700E700E700E700E700E700AA
:102EF000E700E700E700E700E700E700E700E7009A
:102F0000E700E700E600E600E600E600E600E6008F
:102F1000E600E600E600E600E600E600E600E60081
:102F2000E600E600E600E600E600E500E500E50074
:102F3000E500E500E500E500E500E500E500E50069
:102F4000E500E500E500E500E500E500E500E50059
:102F5000E400E400E400E400E400E400E400E40051
:102F6000E400E400E400E400E400E400E400E40041
:102F7000E400E400E400E300E300E300E300E30036
:102F8000E300E300E300E300E300E300E300E30029
:102F9000E300E300E300E300E300E300E300E2001A
:102FA000E200E200E200E200E200E200E200E20011
:102FB000E200E200E200E200E200E200E200E20001
:102FC000E200E200E100E100E100E100E100E100F7
:102FD000E100E100E100E100E100E100E100E100E9
:102FE000E100E100E100E100E100E100E000E000DB
:102FF000E000E000E000E000E000E000E000E000D1
:10300000E000E000E000E000E000E000E000E000C0
:10301000E000E000DF00DF00DF00DF00DF00DF00B6
:10302000DF00DF00DF00DF00DF00DF00DF00DF00A8
:10303000DF00DF00DF00DF00DF00DF00DE00DE009A
:10304000DE00DE00DE00DE00DE00DE00DE00DE0090
:10305000DE00DE00DE00DE00DE00DE00DE00DE0080
:10306000DE00DE00DD00DD00DD00DD00DD00DD0076
:10307000DD00DD00DD00DD00DD00DD00DD00DD0068
:10308000DD00DD00DD00DD00DD00DD00DD00DC0059
:10309000DC00DC00DC00DC00DC00DC00DC00DC0050
:1030A000DC00DC00DC00DC00DC00DC00DC00DC0040
:1030B000DC00DC00DC00DB00DB00DB00DB00DB0035
:1030C000DB00DB00DB00DB00DB00DB00DB00DB0028
:1030D000DB00DB00DB00DB00DB00DB00DB00DB0018
:1030E000DA00DA00DA00DA00DA00DA00DA00DA0010
:1030F000DA00DA00DA00DA00DA00DA00DA00DA0000
:10310000DA00DA00DA00DA00DA00D900D900D900F2
:10311000D900D900D900D900D900D900D900D900E7
:10312000D900D900D900D900D900D900D900D900D7
:10313000D900D900D800D800D800D800D800D800CD
:10314000D800D800D800D800D800D800D800D800BF
:10315000D800D800D800D800D800D800D800D800AF
:10316000D700D700D700D700D700D700D700D700A7
:10317000D700D700D700D700D700D700D700D70097
:10318000D700D700D700D700D700D700D600D60089
:10319000D600D600D600D600D600D600D600D6007F
:1031A000D600D600D600D600D600D600D600D6006F
:1031B000D600D600D600D500D500D500D500D50064
:1031C000D500D500D500D500D500D500D500D50057
:1031D000D500D500D500D500D500D500D500D50047
:1031E000D500D400D400D400D400D400D400D4003E
:1031F000D400D400D400D400D400D400D400D4002F
:10320000D400D400D400D400D400D400D400D4001E
:10321000D300D300D300D300D300D300D300D30016
:10322000D300D300D300D300D300D300D300D30006
:10323000D300D300D300D300D300D300D200D200F8
:10324000D200D200D200D200D200D200D200D200EE
:10325000D200D200D200D200D200D200D200D200DE
:10326000D200D200D200D200D200D100D100D100D1
:10327000D100D100D100D100D100D100D100D100C6
:10328000D100D100D100D100D100D100D100D100B6
:10329000D100D100D100D100D000D000D000D000AA
:1032A000D000D000D000D000D000D000D000D0009E
:1032B000D000D000D000D000D000D000D000D0008E
:1032C000D000D000D000CF00CF00CF00CF00CF0083
:1032D000CF00CF00CF00CF00CF00CF00CF00CF0076
:1032E000CF00CF00CF00CF00CF00CF00CF00CF0066
:1032F000CF00CF00CE00CE00CE00CE00CE00CE005C
:10330000CE00CE00CE00CE00CE00CE00CE00CE004D
:10331000CE00CE00CE00CE00CE00CE00CE00CE003D
:10332000CE00CE00CD00CD00CD00CD00CD00CD0033
:10333000CD00CD00CD00CD00CD00CD00CD00CD0025
:10334000CD00CD00CD00CD00CD00CD00CD00CD0015
:10335000CD00CC00CC00CC00CC00CC00CC00CC000C
:10336000CC00CC00CC00CC00CC00CC00CC00CC00FD
:10337000CC00CC00CC00CC00CC00CC00CC00CC00ED
:10338000CC00CC00CB00CB00CB00CB00CB00CB00E3
:10339000CB00CB00CB00CB00CB00CB00CB00CB00D5
:1033A000CB00CB00CB00CB00CB00CB00CB00CB00C5
:1033B000CB00CB00CA00CA00CA00CA00CA00CA00BB
:1033C000CA00CA00CA00CA00CA00CA00CA00CA00AD
:1033D000CA00CA00CA00CA00CA00CA00CA00CA009D
:1033E000CA00CA00C900C900C900C900C900C90093
:1033F000C900C900C900C900C900C900C900C90085
:10340000C900C900C900C900C900C900C900C90074
:10341000C900C900C900C800C800C800C800C80069
:10342000C800C800C800C800C800C800C800C8005C
:10343000C800C800C800C800C800C800C800C8004C
:10344000C800C800C800C800C700C700C700C70040
:10345000C700C700C700C700C700C700C700C70034
:10346000C700C700C700C700C700C700C700C70024
:10347000C700C700C700C700C700C600C600C60017
:10348000C600C600C600C600C600C600C600C6000C
:10349000C600C600C600C600C600C600C600C600FC
:1034A000C600C600C600C600C600C600C600C500ED
:1034B000C500C500C500C500C500C500C500C500E4
:1034C000C500C500C500C500C500C500C500C500D4
:1034D000C500C500C500C500C500C500C500C500C4
:1034E000C500C400C400C400C400C400C400C400BB
:1034F000C400C400C400C400C400C400C400C400AC
:10350000C400C400C400C400C400C400C400C4009B
:10351000C400C400C400C300C300C300C300C30090
:10352000C300C300C300C300C300C300C300C30083
:10353000C300C300C300C300C300C300C300C30073
:10354000C300C300C300C300C300C200C200C20066
:10355000C200C200C200C200C200C200C200C2005B
:10356000C200C200C200C200C200C200C200C2004B
:10357000C200C200C200C200C200C200C200C1003C
:10358000C100C100C100C100C100C100C100C10033
:10359000C100C100C100C100C100C100C100C10023
:1035A000C100C100C100C100C100C100C100C10013
:1035B000C100C100C000C000C000C000C000C00009
:1035C000C000C000C000C000C000C000C000C000FB
:1035D000C000C000C000C000C000C000C000C000EB
:1035E000C000C000C000C000C000BF00BF00BF00DE
:1035F000BF00BF00BF00BF00BF00BF00BF00BF00D3
:10360000BF00BF00BF00BF00BF00BF00BF00BF00C2
:10361000BF00BF00BF00BF00BF00BF00BF00BF00B2
:10362000BF00BE00BE00BE00BE00BE00BE00BE00A9
:10363000BE00BE00BE00BE00BE00BE00BE00BE009A
:10364000BE00BE00BE00BE00BE00BE00BE00BE008A
:10365000BE00BE00BE00BE00BE00BD00BD00BD007D
:10366000BD00BD00BD00BD00BD00BD00BD00BD0072
:10367000BD00BD00BD00BD00BD00BD00BD00BD0062
:10368000BD00BD00BD00BD00BD00BD00BD00BD0052
:10369000BD00BC00BC00BC00BC00BC00BC00BC0049
:1036A000BC00BC00BC00BC00BC00BC00BC00BC003A
:1036B000BC00BC00BC00BC00BC00BC00BC00BC002A
:1036C000BC00BC00BC00BC00BC00BB00BB00BB001D
:1036D000BB00BB00BB00BB00BB00BB00BB00BB0012
:1036E000BB00BB00BB00BB00BB00BB00BB00BB0002
:1036F000BB00BB00BB00BB00BB00BB00BB00BB00F2
:10370000BB00BA00BA00BA00BA00BA00BA00BA00E8
:10371000BA00BA00BA00BA00BA00BA00BA00BA00D9
:10372000BA00BA00BA00BA00BA00BA00BA00BA00C9
:10373000BA00BA00BA00BA00BA00BA00B900B900BB
:10374000B900B900B900B900B900B900B900B900B1
:10375000B900B900B900B900B900B900B900B900A1
:10376000B900B900B900B900B900B900B900B90091
:10377000B900B900B900B900B800B800B800B80085
:10378000B800B800B800B800B800B800B800B80079
:10379000B800B800B800B800B800B800B800B80069
:1037A000B800B800B800B800B800B800B800B80059
:1037B000B800B700B700B700B700B700B700B70050
:1037C000B700B700B700B700B700B700B700B70041
:1037D000B700B700B700B700B700B700B700B70031
:1037E000B700B700B700B700B700B700B700B60022
:1037F000B600B600B600B600B600B600B600B60019
:10380000B600B600B600B600B600B600B600B60008
:10381000B600B600B600B600B600B600B600B600F8
:10382000B600B600B600B600B600B500B500B500EB
:10383000B500B500B500B500B500B500B500B500E0
:10384000B500B500B500B500B500B500B500B500D0
:10385000B500B500B500B500B500B500B500B500C0
:10386000B500B500B500B500B400B400B400B400B4
:10387000B400B400B400B400B400B400B400B400A8
:10388000B400B400B400B400B400B400B400B40098
:10389000B400B400B400B400B400B400B400B40088
:1038A000B400B400B400B300B300B300B300B3007D
:1038B000B300B300B300B300B300B300B300B30070
:1038C000B300B300B300B300B300B300B300B30060
:1038D000B300B300B300B300B300B300B300B30050
:1038E000B300B300B200B200B200B200B200B20046
:1038F000B200B200B200B200B200B200B200B20038
:10390000B200B200B200B200B200B200B200B20027
:10391000B200B200B200B200B200B200B200B20017
:10392000B200B100B100B100B100B100B100B1000E
:10393000B100B100B100B100B100B100B100B100FF
:10394000B100B100B100B100B100B100B100B100EF
:10395000B100B100B100B100B100B100B100B100DF
:10396000B100B000B000B000B000B000B000B000D6
:10397000B000B000B000B000B000B000B000B000C7
:10398000B000B000B000B000B000B000B000B000B7
:10399000B000B000B000B000B000B000B000B000A7
:1039A000B000B000AF00AF00AF00AF00AF00AF009D
:1039B000AF00AF00AF00AF00AF00AF00AF00AF008F
:1039C000AF00AF00AF00AF00AF00AF00AF00AF007F
:1039D000AF00AF00AF00AF00AF00AF00AF00AF006F
:1039E000AF00AF00AE00AE00AE00AE00AE00AE0065
:1039F000AE00AE00AE00AE00AE00AE00AE00AE0057
:103A0000AE00AE00AE00AE00AE00AE00AE00AE0046
:103A1000AE00AE00AE00AE00AE00AE00AE00AE0036
:103A2000AE00AE00AE00AD00AD00AD00AD00AD002B
:103A3000AD00AD00AD00AD00AD00AD00AD00AD001E
:103A4000AD00AD00AD00AD00AD00AD00AD00AD000E
:103A5000AD00AD00AD00AD00AD00AD00AD00AD00FE
:103A6000AD00AD00AD00AD00AD00AC00AC00AC00F1
:103A7000AC00AC00AC00AC00AC00AC00AC00AC00E6
:103A8000AC00AC00AC00AC00AC00AC00AC00AC00D6
:103A9000AC00AC00AC00AC00AC00AC00AC00AC00C6
:103AA000AC00AC00AC00AC00AC00AC00AB00AB00B8
:103AB000AB00AB00AB00AB00AB00AB00AB00AB00AE
:103AC000AB00AB00AB00AB00AB00AB00AB00AB009E
:103AD000AB00AB00AB00AB00AB00AB00AB00AB008E
:103AE000AB00AB00AB00AB00AB00AB00AB00AB007E
:103AF000AB00AA00AA00AA00AA00AA00AA00AA0075
:103B0000AA00AA00AA00AA00AA00AA00AA00AA0065
:103B1000AA00AA00AA00AA00AA00AA00AA00AA0055
:103B2000AA00AA00AA00AA00AA00AA00AA00AA0045
:103B3000AA00AA00AA00A900A900A900A900A9003A
:103B4000A900A900A900A900A900A900A900A9002D
:103B5000A900A900A900A900A900A900A900A9001D
:103B6000A900A900A900A900A900A900A900A9000D
:103B7000A900A900A900A900A900A900A800A800FF
:103B8000A800A800A800A800A800A800A800A800F5
:103B9000A800A800A800A800A800A800A800A800E5
:103BA000A800A800A800A800A800A800A800A800D5
:103BB000A800A800A800A800A800A800A800A800C5
:103BC000A800A800A700A700A700A700A700A700BB
:103BD000A700A700A700A700A700A700A700A700AD
:103BE000A700A700A700A700A700A700A700A7009D
:103BF000A700A700A700A700A700A700A700A7008D
:103C0000A700A700A700A700A700A700A600A6007E
:103C1000A600A600A600A600A600A600A600A60074
:103C2000A600A600A600A600A600A600A600A60064
:103C3000A600A600A600A600A600A600A600A60054
:103C4000A600A600A600A600A600A600A600A60044
:103C5000A600A600A500A500A500A500A500A5003A
:103C6000A500A500A500A500A500A500A500A5002C
:103C7000A500A500A500A500A500A500A500A5001C
:103C8000A500A500A500A500A500A500A500A5000C
:103C9000A500A500A500A500A500A500A500A400FD
:103CA000A400A400A400A400A400A400A400A400F4
:103CB000A400A400A400A400A400A400A400A400E4
:103CC000A400A400A400A400A400A400A400A400D4
:103CD000A400A400A400A400A400A400A400A400C4
:103CE000A400A400A400A400A300A300A300A300B8
:103CF000A300A300A300A300A300A300A300A300AC
:103D0000A300A300A300A300A300A300A300A3009B
:103D1000A300A300A300A300A300A300A300A3008B
:103D2000A300A300A300A300A300A300A300A3007B
:103D3000A300A200A200A200A200A200A200A20072
:103D4000A200A200A200A200A200A200A200A20063
:103D5000A200A200A200A200A200A200A200A20053
:103D6000A200A200A200A200A200A200A200A20043
:103D7000A200A200A200A200A200A200A200A10034
:103D8000A100A100A100A100A100A100A100A1002B
:103D9000A100A100A100A100A100A100A100A1001B
:103DA000A100A100A100A100A100A100A100A1000B
:103DB000A100A100A100A100A100A100A100A100FB
:103DC000A100A100A100A100A100A100A000A000ED
:103DD000A000A000A000A000A000A000A000A000E3
:103DE000A000A000A000A000A000A000A000A000D3
:103DF000A000A000A000A000A000A000A000A000C3
:103E0000A000A000A000A000A000A000A000A000B2
:103E1000A000A000A000A000A0009F009F009F00A5
:103E20009F009F009F009F009F009F009F009F009A
:103E30009F009F009F009F009F009F009F009F008A
:103E40009F009F009F009F009F009F009F009F007A
:103E50009F009F009F009F009F009F009F009F006A
:103E60009F009F009F009F009F009E009E009E005D
:103E70009E009E009E009E009E009E009E009E0052
:103E80009E009E009E009E009E009E009E009E0042
:103E90009E009E009E009E009E009E009E009E0032
:103EA0009E009E009E009E009E009E009E009E0022
:103EB0009E009E009E009E009E009D009D009D0015
:103EC0009D009D009D009D009D009D009D009D000A
:103ED0009D009D009D009D009D009D009D009D00FA
:103EE0009D009D009D009D009D009D009D009D00EA
:103EF0009D009D009D009D009D009D009D009D00DA
:103F00009D009D009D009D009D009C009C009C00CC
:103F10009C009C009C009C009C009C009C009C00C1
:103F20009C009C009C009C009C009C009C009C00B1
:103F30009C009C009C009C009C009C009C009C00A1
:103F40009C009C009C009C009C009C009C009C0091
:103F50009C009C009C009C009C009C009B009B0083
:103F60009B009B009B009B009B009B009B009B0079
:103F70009B009B009B009B009B009B009B009B0069
:103F80009B009B009B009B009B009B009B009B0059
:103F90009B009B009B009B009B009B009B009B0049
:103FA0009B009B009B009B009B009B009B009B0039
:103FB0009A009A009A009A009A009A009A009A0031
:103FC0009A009A009A009A009A009A009A009A0021
:103FD0009A009A009A009A009A009A009A009A0011
:103FE0009A009A009A009A009A009A009A009A0001
:103FF0009A009A009A009A009A009A009A009A00F1
:104000009A009A00990099009900990099009900E6
:1040100099009900990099009900990099009900D8
:1040200099009900990099009900990099009900C8
:1040300099009900990099009900990099009900B8
:1040400099009900990099009900990099009900A8
:10405000990099009900990099009800980098009B
:104060009800980098009800980098009800980090
:104070009800980098009800980098009800980080
:104080009800980098009800980098009800980070
:104090009800980098009800980098009800980060
:1040A0009800980098009800980098009800980050
:1040B0009700970097009700970097009700970048
:1040C0009700970097009700970097009700970038
:1040D0009700970097009700970097009700970028
:1040E0009700970097009700970097009700970018
:1040F0009700970097009700970097009700970008
:1041000097009700970097009600960096009600FB
:1041100096009600960096009600960096009600EF
:1041200096009600960096009600960096009600DF
:1041300096009600960096009600960096009600CF
:1041400096009600960096009600960096009600BF
:1041500096009600960096009600960096009600AF
:1041600095009500950095009500950095009500A7
:104170009500950095009500950095009500950097
:104180009500950095009500950095009500950087
:104190009500950095009500950095009500950077
:1041A0009500950095009500950095009500950067
:1041B0009500950095009500950095009400940059
:1041C000940094009400940094009400940094004F
:1041D000940094009400940094009400940094003F
:1041E000940094009400940094009400940094002F
:1041F000940094009400940094009400940094001F
:10420000940094009400940094009400940094000E
:104210009400940094009300930093009300930003
:1042200093009300930093009300930093009300F6
:1042300093009300930093009300930093009300E6
:1042400093009300930093009300930093009300D6
:1042500093009300930093009300930093009300C6
:1042600093009300930093009300930093009300B6
:1042700093009200920092009200920092009200AD
:10428000920092009200920092009200920092009E
:10429000920092009200920092009200920092008E
:1042A000920092009200920092009200920092007E
:1042B000920092009200920092009200920092006E
:1042C000920092009200920092009200920092005E
:1042D0009100910091009100910091009100910056
:1042E0009100910091009100910091009100910046
:1042F0009100910091009100910091009100910036
:104300009100910091009100910091009100910025
:104310009100910091009100910091009100910015
:104320009100910091009100910091009100910005
:1043300090009000900090009000900090009000FD
:1043400090009000900090009000900090009000ED
:1043500090009000900090009000900090009000DD
:1043600090009000900090009000900090009000CD
:1043700090009000900090009000900090009000BD
:1043800090009000900090009000900090009000AD
:104390008F008F008F008F008F008F008F008F00A5
:1043A0008F008F008F008F008F008F008F008F0095
:1043B0008F008F008F008F008F008F008F008F0085
:1043C0008F008F008F008F008F008F008F008F0075
:1043D0008F008F008F008F008F008F008F008F0065
:1043E0008F008F008F008F008F008F008F008F0055
:1043F0008F008E008E008E008E008E008E008E004C
:104400008E008E008E008E008E008E008E008E003C
:104410008E008E008E008E008E008E008E008E002C
:104420008E008E008E008E008E008E008E008E001C
:104430008E008E008E008E008E008E008E008E000C
:104440008E008E008E008E008E008E008E008E00FC
:104450008E008E008E008D008D008D008D008D00F1
:104460008D008D008D008D008D008D008D008D00E4
:104470008D008D008D008D008D008D008D008D00D4
:104480008D008D008D008D008D008D008D008D00C4
:104490008D008D008D008D008D008D008D008D00B4
:1044A0008D008D008D008D008D008D008D008D00A4
:1044B0008D008D008D008D008D008C008C008C0097
:1044C0008C008C008C008C008C008C008C008C008C
:1044D0008C008C008C008C008C008C008C008C007C
:1044E0008C008C008C008C008C008C008C008C006C
:1044F0008C008C008C008C008C008C008C008C005C
:104500008C008C008C008C008C008C008C008C004B
:104510008C008C008C008C008C008C008C008C003B
:104520008B008B008B008B008B008B008B008B0033
:104530008B008B008B008B008B008B008B008B0023
:104540008B008B008B008B008B008B008B008B0013
:104550008B008B008B008B008B008B008B008B0003
:104560008B008B008B008B008B008B008B008B00F3
:104570008B008B008B008B008B008B008B008B00E3
:104580008B008B008B008B008A008A008A008A00D7
:104590008A008A008A008A008A008A008A008A00CB
:1045A0008A008A008A008A008A008A008A008A00BB
:1045B0008A008A008A008A008A008A008A008A00AB
:1045C0008A008A008A008A008A008A008A008A009B
:1045D0008A008A008A008A008A008A008A008A008B
:1045E0008A008A008A008A008A008A008A008A007B
:1045F0008900890089008900890089008900890073
:104600008900890089008900890089008900890062
:104610008900890089008900890089008900890052
:104620008900890089008900890089008900890042
:104630008900890089008900890089008900890032
:104640008900890089008900890089008900890022
:104650008900890089008900890089008800880014
:10466000880088008800880088008800880088000A
:1046700088008800880088008800880088008800FA
:1046800088008800880088008800880088008800EA
:1046900088008800880088008800880088008800DA
:1046A00088008800880088008800880088008800CA
:1046B00088008800880088008800880088008800BA
:1046C00088008800880088008700870087008700AE
:1046D00087008700870087008700870087008700A2
:1046E0008700870087008700870087008700870092
:1046F0008700870087008700870087008700870082
:104700008700870087008700870087008700870071
:104710008700870087008700870087008700870061
:104720008700870087008700870087008700870051
:104730008700870086008600860086008600860047
:104740008600860086008600860086008600860039
:104750008600860086008600860086008600860029
:104760008600860086008600860086008600860019
:104770008600860086008600860086008600860009
:1047800086008600860086008600860086008600F9
:1047900086008600860086008600860086008600E9
:1047A00086008600850085008500850085008500DF
:1047B00085008500850085008500850085008500D1
:1047C00085008500850085008500850085008500C1
:1047D00085008500850085008500850085008500B1
:1047E00085008500850085008500850085008500A1
:1047F0008500850085008500850085008500850091
:104800008500850085008500850085008500850080
:104810008500850085008400840084008400840075
:104820008400840084008400840084008400840068
:104830008400840084008400840084008400840058
:104840008400840084008400840084008400840048
:104850008400840084008400840084008400840038
:104860008400840084008400840084008400840028
:104870008400840084008400840084008400840018
:10488000840084008400840083008300830083000C
:104890008300830083008300830083008300830000
:1048A00083008300830083008300830083008300F0
:1048B00083008300830083008300830083008300E0
:1048C00083008300830083008300830083008300D0
:1048D00083008300830083008300830083008300C0
:1048E00083008300830083008300830083008300B0
:1048F00083008300830083008300830082008200A2
:104900008200820082008200820082008200820097
:104910008200820082008200820082008200820087
:104920008200820082008200820082008200820077
:104930008200820082008200820082008200820067
:104940008200820082008200820082008200820057
:104950008200820082008200820082008200820047
:104960008200820082008200820082008200820037
:10497000820082008100810081008100810081002D
:10498000810081008100810081008100810081001F
:10499000810081008100810081008100810081000F
:1049A00081008100810081008100810081008100FF
:1049B00081008100810081008100810081008100EF
:1049C00081008100810081008100810081008100DF
:1049D00081008100810081008100810081008100CF
:1049E00081008100810081008100810080008000C1
:1049F00080008000800080008000800080008000B7
:104A000080008000800080008000800080008000A6
:104A10008000800080008000800080008000800096
:104A20008000800080008000800080008000800086
:104A30008000800080008000800080008000800076
:104A40008000800080008000800080008000800066
:104A50008000800080008000800080008000800056
:104A60008000800080007F007F007F007F007F004B
:104A70007F007F007F007F007F007F007F007F003E
:104A80007F007F007F007F007F007F007F007F002E
:104A90007F007F007F007F007F007F007F007F001E
:104AA0007F007F007F007F007F007F007F007F000E
:104AB0007F007F007F007F007F007F007F007F00FE
:104AC0007F007F007F007F007F007F007F007F00EE
:104AD0007F007F007F007F007F007F007F007F00DE
:104AE0007F007E007E007E007E007E007E007E00D5
:104AF0007E007E007E007E007E007E007E007E00C6
:104B00007E007E007E007E007E007E007E007E00B5
:104B10007E007E007E007E007E007E007E007E00A5
:104B20007E007E007E007E007E007E007E007E0095
:104B30007E007E007E007E007E007E007E007E0085
:104B40007E007E007E007E007E007E007E007E0075
:104B50007E007E007E007E007E007E007E007E0065
:104B60007D007D007D007D007D007D007D007D005D
:104B70007D007D007D007D007D007D007D007D004D
:104B80007D007D007D007D007D007D007D007D003D
:104B90007D007D007D007D007D007D007D007D002D
:104BA0007D007D007D007D007D007D007D007D001D
:104BB0007D007D007D007D007D007D007D007D000D
:104BC0007D007D007D007D007D007D007D007D00FD
:104BD0007D007D007D007D007D007D007D007D00ED
:104BE0007C007C007C007C007C007C007C007C00E5
:104BF0007C007C007C007C007C007C007C007C00D5
:104C00007C007C007C007C007C007C007C007C00C4
:104C10007C007C007C007C007C007C007C007C00B4
:104C20007C007C007C007C007C007C007C007C00A4
:104C30007C007C007C007C007C007C007C007C0094
:104C40007C007C007C007C007C007C007C007C0084
:104C50007C007C007C007C007C007C007C007C0074
:104C60007C007B007B007B007B007B007B007B006B
:104C70007B007B007B007B007B007B007B007B005C
:104C80007B007B007B007B007B007B007B007B004C
:104C90007B007B007B007B007B007B007B007B003C
:104CA0007B007B007B007B007B007B007B007B002C
:104CB0007B007B007B007B007B007B007B007B001C
:104CC0007B007B007B007B007B007B007B007B000C
:104CD0007B007B007B007B007B007B007B007B00FC
:104CE0007B007B007B007A007A007A007A007A00F1
:104CF0007A007A007A007A007A007A007A007A00E4
:104D00007A007A007A007A007A007A007A007A00D3
:104D10007A007A007A007A007A007A007A009500A8
:104D200000000046696E64207468652034206B6E54
:104D30006F6273206F6E200095010000007468653B
:104D400020626F74746F6D206F6620746865202018
:104D500020009501000000706C6174666F726D2018
:104D6000616E64207469676874656E009507000061
:104D700000666F7572206F722066697665207475A3
:104D8000726E732E00950000000049276D20676F3A
:104D9000696E6720746F206D6F7665202020009506
:104DA000010000007468652065787472756465722E
:104DB00020746F20202020200095010000007661E3
:104DC00072696F757320706F736974696F6E732089
:104DD0002020009507000000666F722061646A75EC
:104DE00073746D656E742E009500000000496E208E
:104DF0006561636820706F736974696F6E2C202021
:104E00002000950100000077652077696C6C206EAA
:104E100065656420746F202020202000950100002B
:104E20000061646A7573742032206B6E6F62732048
:104E300061742020200095070000007468652073CD
:104E4000616D652074696D652E0095000000004E4F
:104E50006F7A7A6C65732061726520617420746862
:104E60006520200095010000007269676874206861
:104E70006569676874207768656E20202000950159
:104E8000000000796F752063616E206A757374206D
:104E9000736C6964652061009507000000736865A4
:104EA0006574206F66207061706572009500000067
:104EB000006265747765656E20746865206E6F7A30
:104EC0007A6C652020009501000000616E642074FA
:104ED000686520706C6174666F726D2E20202000F2
:104EE000950100000047726162206120736865656A
:104EF00074206F662020202020009507000000709D
:104F00006170657220746F206173736973742075AA
:104F1000732E009502000000506C65617365207768
:104F2000616974008403690100001400830488002F
:104F3000000014008C000000000000000030F8FFAA
:104F4000FF00000000000000008E000000000000D4
:104F500000000000000000000000000000005729D1
:104F60000400188304DC05000014008CE537000001
:104F7000941B000000000000000000000000000082
:104F80009502000000506C6561736520776169745B
:104F9000008EE6370000941B0000D00700000000E0
:104FA0000000000000000D450300188E0000000006
:104FB000CAE4FFFFD007000000000000000000006E
:104FC0002A0D3B00188E00000000C9E4FFFF00001E
:104FD000000000000000000000000D4503001895CF
:104FE0000000000041646A7573742074686520666F
:104FF000726F6E742074776F0095010000006B6E05
:105000006F627320756E74696C20706170657220B8
:1050100020200095010000006A75737420736C698C
:10502000646573206265747765656E20009507007E
:1050300000006E6F7A7A6C6520616E6420706C611E
:1050400074666F726D009502000000506C656173AC
:10505000652077616974008E00000000CAE4FFFFDC
:10506000D007000000000000000000000D45030014
:10507000188E000000007A1A0000D007000000001F
:1050800000000000000051812800188E0000000080
:105090007A1A00000000000000000000000000007C
:1050A0000D45030018950000000041646A75737493
:1050B00020746865206261636B2074776F200095AF
:1050C000010000006B6E6F627320756E74696C2056
:1050D00070617065722020200095010000006A75E3
:1050E000737420736C696465732062657477656599
:1050F0006E200095070000006E6F7A7A6C65206163
:105100006E6420706C6174666F726D0095020000B1
:1051100000506C656173652077616974008E0000D2
:1051200000007A1A0000D007000000000000000014
:1051300000000D450300188EC6240000000000008A
:10514000D00700000000000000000000A82F22008F
:10515000188EC624000000000000000000000000BF
:105160000000000000000D4503001895000000003D
:1051700041646A7573742074686520726967687425
:105180002074776F0095010000006B6E6F627320D2
:10519000756E74696C2070617065722020200095B6
:1051A000010000006A75737420736C696465732074
:1051B0006265747765656E200095070000006E6F6C
:1051C0007A7A6C6520616E6420706C6174666F72AF
:1051D0006D009502000000506C6561736520776179
:1051E0006974008EC624000000000000D007000093
:1051F00000000000000000000D450300188E3ADB9F
:10520000FFFF00000000D0070000000000000000C9
:1052100000008B7C3700188E3ADBFFFF0000000097
:105220000000000000000000000000000D45030029
:1052300018950000000041646A75737420746865F5
:10524000206C6566742074776F2000950100000063
:105250006B6E6F627320756E74696C20706170651F
:10526000722020200095010000006A75737420737D
:105270006C69646573206265747765656E2000955E
:10528000070000006E6F7A7A6C6520616E64207092
:105290006C6174666F726D009502000000506C6561
:1052A0006173652077616974008E3ADBFFFF00004F
:1052B0000000D007000000000000000000000D45C5
:1052C0000300188E0000000000000000D00700005E
:1052D000000000000000000045BE1B00188E00000A
:1052E00000000000000000000000000000000000BE
:1052F00000000D4503001895000000004368656339
:105300006B207468617420706170657220202020A9
:105310000095010000006A75737420736C69646500
:1053200073206265747765656E2000950700000044
:105330006E6F7A7A6C6520616E6420706C61746641
:105340006F726D00891F9502000000506C656173DB
:105350006520776169742E2E2E0084036901000098
:10536000140083048800000014008C00000000007A
:1053700000000030F8FFFF00000000000000008E79
:10538000000000000000000000000000000000001D
:105390000000000057290400188304DC05000014F5
:1053A00000901F891F950000000046696E642074FC
:1053B00068652034206B6E6F6273206F6E200095DD
:1053C0000100000074686520626F74746F6D206F57
:1053D0006620746865202020009501000000706C34
:1053E0006174666F726D20616E64207469676874A1
:1053F000656E009507000000666F7572206F722061
:1054000066697665207475726E732E0095000000D3
:105410000049276D20676F696E6720746F206D6F7C
:1054200076652020200095010000007468652065E5
:105430007874727564657220746F202020202000BB
:105440009501000000766172696F757320706F734B
:105450006974696F6E732020200095070000006654
:105460006F722061646A7573746D656E742E009539
:1054700000000000496E206561636820706F7369E9
:1054800074696F6E2C202020009501000000776564
:105490002077696C6C206E65656420746F20202015
:1054A000202000950100000061646A757374203249
:1054B000206B6E6F627320617420202000950700BE
:1054C00000007468652073616D652074696D652ED8
:1054D0000095000000004E6F7A7A6C65732061724F
:1054E000652061742074686520200095010000002B
:1054F0007269676874206865696768742077686591
:105500006E202020009501000000796F75206361F6
:105510006E206A75737420736C69646520610095F0
:10552000070000007368656574206F662070617005
:1055300065720095000000006265747765656E20F5
:10554000746865206E6F7A7A6C6520200095010082
:105550000000616E642074686520706C6174666F11
:10556000726D2E20202000950100000047726162BC
:105570002061207368656574206F662020202020DC
:10558000009507000000706170657220746F2061E3
:1055900073736973742075732E00950200000050B8
:1055A0006C6561736520776169740084036901002B
:1055B00000140083048800000014008C0000000028
:1055C0000000000030F8FFFF0000000000000000B5
:1055D0008E0000000000000000000000000000003D
:1055E000000000000057290400188304DC050000B7
:1055F00014008CE5370000941B0000000000000040
:10560000000000000000009502000000506C656181
:1056100073652077616974008EE5370000941B0084
:1056200000D007000000000000000000000D45034E
:1056300000188E12060000CAE4FFFFD00700000029
:1056400000000000000000DADF3700188E110600AD
:1056500000CAE4FFFF00000000000000000000009E
:10566000000D45030018950000000041646A757341
:1056700074207468652066726F6E742074776F0092
:1056800095010000006B6E6F627320756E74696C1B
:105690002070617065722020200095010000006A72
:1056A00075737420736C69646573206265747765C3
:1056B000656E200095070000006E6F7A7A6C652099
:1056C000616E6420706C6174666F726D009502008B
:1056D0000000506C656173652077616974008E11FC
:1056E000060000C9E4FFFFD0070000000000000032
:1056F0000000000D450300188E110600007A1A0004
:1057000000D00700000000000000000000518128C8
:1057100000188E120600007A1A0000000000000037
:10572000000000000000000D450300189500000077
:105730000041646A75737420746865206261636BEC
:105740002074776F200095010000006B6E6F62730C
:1057500020756E74696C2070617065722020200065
:1057600095010000006A75737420736C6964657339
:10577000206265747765656E200095070000006EF5
:105780006F7A7A6C6520616E6420706C6174666FEC
:10579000726D009502000000506C656173652077A2
:1057A000616974008E110600007B1A0000D00700AA
:1057B0000000000000000000000D450300188E2AC4
:1057C00027000000000000D00700000000000000DB
:1057D000000000CFF91F00188E2A270000000000EB
:1057E000000000000000000000000000000D450364
:1057F0000018950000000041646A75737420746895
:10580000652072696768742074776F0095010000E5
:10581000006B6E6F627320756E74696C20706170BE
:1058200065722020200095010000006A75737420C5
:10583000736C69646573206265747765656E2000BA
:1058400095070000006E6F7A7A6C6520616E6420A7
:10585000706C6174666F726D009502000000506C90
:10586000656173652077616974008E2A27000000E6
:10587000000000D007000000000000000000000D44
:10588000450300188EF8E4FFFF00000000D0070079
:1058900000000000000000000017F03100188EF931
:1058A000E4FFFF0000000000000000000000000016
:1058B0000000000D45030018950000000041646AD7
:1058C00075737420746865206C6566742074776FD6
:1058D000200095010000006B6E6F627320756E747E
:1058E000696C2070617065722020200095010000B5
:1058F000006A75737420736C6964657320626574E3
:105900007765656E200095070000006E6F7A7A6CEF
:105910006520616E6420706C6174666F726D0095B5
:1059200002000000506C6561736520776169740046
:105930008EF9E4FFFF00000000D007000000000027
:1059400000000000000D450300188E110600000045
:10595000000000D007000000000000000000000B65
:10596000F81800188E11060000000000000000006A
:105970000000000000000000000D45030018950025
:10598000000000436865636B207468617420706177
:10599000706572202020200095010000006A757358
:1059A0007420736C69646573206265747765656ED5
:1059B000200095070000006E6F7A7A6C6520616E9A
:1059C0006420706C6174666F726D00891F990000AD
:1059D000000052657047204275696C64009600FFB4
:1059E0008600860088001F026E0088011F026E007C
:1059F000860088000302DC00860188010302DC00C7
:105A0000840369010000140083048800000014006E
:105A10008C000000000000000030F8FFFF000000D4
:105A200000000000008E00000000000000000000E8
:105A30000000000000000000000057290400188347
:105A400004DC0500001400901F8B5ED7FFFFCAE442
:105A5000FFFF60EA0000000000000000000080007E
:105A60000000910014910114910214910314910407
:105A7000148600860087006400FFFF8D006400FF2D
:105A8000FF8601860187016400FFFF8D006400FF2F
:105A9000FF91007F91017F91022891037F91047F04
:105AA00086008E5DD7FFFFCAE4FFFF5000000000B4
:105AB0000000000000000003387500188988880085
:105AC0000A010388000401FF8E00000000000000AE
:105AD0000000000000C0FEFFFF0000000060E316B1
:105AE000001F8E42E6FFFFB7E9FFFF680100005B81
:105AF000FFFFFF000000002ED60B00188E43E6FFCC
:105B0000FFB7E9FFFF68010000E3FFFFFF000000AF
:105B1000001C5800001889888E42E6FFFFB7E9FF95
:105B2000FFF0000000ECFFFFFF000000000032006B
:105B300000188E42E6FFFFB7E9FFFFF0000000E427
:105B4000FFFFFF00000000F22B0000188E8DD7FF32
:105B5000FFB7E9FFFFF00000009BFEFFFF00000021
:105B600000862F3000188E42E6FFFF6EEDFFFFF03B
:105B7000000000300000000000000012720B00184E
:105B80008E42E6FFFF6EEDFFFFF0000000E4FFFF36
:105B9000FF00000000F12B0000188E3ADBFFFF6EC3
:105BA000EDFFFFF00000009BFEFFFF00000000A5DE
:105BB000232400188E42E6FFFF25F1FFFFF00000CE
:105BC00000300000000000000031C80800188E43BB
:105BD000E6FFFF25F1FFFFF0000000E4FFFFFF00FC
:105BE000000000F12B0000188E3ADBFFFF25F1FFCB
:105BF000FFF00000009BFEFFFF00000000A5232433
:105C000000188E42E6FFFFDBF4FFFFF000000031DA
:105C10000000000000000031C80800188E42E6FFB6
:105C2000FFDCF4FFFFF0000000E3FFFFFF000000D7
:105C300000F22B0000188E3ADBFFFFDBF4FFFFF0D1
:105C40000000009BFEFFFF00000000A523240018B9
:105C50008E42E6FFFF93F8FFFFF0000000310000E6
:105C6000000000000031C80800188E42E6FFFF92D5
:105C7000F8FFFFF0000000E3FFFFFF00000000F26C
:105C80002B0000188E3ADBFFFF92F8FFFFF00000B8
:105C9000009BFEFFFF00000000A5232400188E4398
:105CA000E6FFFF4AFCFFFFF00000003100000000AB
:105CB00000000031C80800188E42E6FFFF49FCFFD3
:105CC000FFF0000000E3FFFFFF00000000F22B00E8
:105CD00000188E3ADBFFFF49FCFFFFF00000009B3D
:105CE000FEFFFF00000000A5232400188E42E6FFFF
:105CF000FF00000000F00000003100000000000084
:105D00000031C80800188E42E6FFFF00000000F0D6
:105D1000000000E3FFFFFF00000000F22B0000186E
:105D20008E3ADBFFFF00000000F00000009CFEFF49
:105D3000FF00000000A5232400188E43E6FFFFB7F4
:105D4000030000F0000000300000000000000031FF
:105D5000C80800188E42E6FFFFB7030000F00000FD
:105D600000E3FFFFFF00000000F22B0000188E3A56
:105D7000DBFFFFB6030000F00000009CFEFFFF0009
:105D8000000000A5232400188E42E6FFFF6E0700E6
:105D900000F0000000300000000000000031C808E2
:105DA00000188E42E6FFFF6E070000F0000000E3DF
:105DB000FFFFFF00000000F22B0000188E3ADBFF0F
:105DC000FF6D070000F00000009CFEFFFF000000D8
:105DD00000A5232400188E43E6FFFF250B0000F0EA
:105DE000000000300000000000000031C80800186A
:105DF0008E42E6FFFF240B0000F0000000E3FFFFEF
:105E0000FF00000000F12B0000188E3ADBFFFF2599
:105E10000B0000F00000009CFEFFFF00000000A54A
:105E2000232400188E42E6FFFFDB0E0000F0000086
:105E300000300000000000000031C80800188E4249
:105E4000E6FFFFDB0E0000F0000000E3FFFFFF00B5
:105E5000000000F12B0000188E3ADBFFFFDB0E0084
:105E600000F00000009CFEFFFF00000000A52324BE
:105E700000188E43E6FFFF92120000F00000003091
:105E80000000000000000031C80800188E42E6FF44
:105E9000FF92120000F0000000E3FFFFFF0000008F
:105EA00000F12B0000188E3ADBFFFF92120000F089
:105EB0000000009CFEFFFF00000000A52324001846
:105EC0008E42E6FFFF49160000F00000003000009F
:105ED000000000000031C80800188E42E6FFFF49AC
:105EE000160000F0000000E3FFFFFF00000000F1DB
:105EF0002B0000188E3ADBFFFF49160000F000006F
:105F0000009CFEFFFF00000000A5232400188EC0A7
:105F1000F4FFFFA5F8FFFF6801000030000000005B
:105F200000000018821D00188EBFF4FFFFA5F8FFC7
:105F3000FFF0000000D0FFFFFF00000000AE2500D2
:105F400000188EBFF4FFFFA6F8FFFFF0000000E38B
:105F5000FFFFFF00000000F12B0000188EC0F4FFCF
:105F6000FF5A070000F00000009CFEFFFF00000049
:105F700000862F3000188E76F8FFFFA6F8FFFFF09E
:105F8000000000300000000000000012720B00183A
:105F90008E76F8FFFFA5F8FFFFF0000000E3FFFF9B
:105FA000FF00000000F12B0000188E76F8FFFFAD17
:105FB000030000F00000009CFEFFFF00000000A5B1
:105FC000232400188E2DFCFFFFA5F8FFFFF0000032
:105FD00000300000000000000031C80800188E2DBD
:105FE000FCFFFFA6F8FFFFF0000000E3FFFFFF004B
:105FF000000000F12B0000188E2DFCFFFFAD030008
:1060000000F00000009CFEFFFF00000000A523241C
:1060100000188EE4FFFFFFA5F8FFFFF0000000303E
:106020000000000000000031C80800188EE3FFFFE8
:10603000FFA5F8FFFFF0000000E3FFFFFF000000F6
:1060400000F12B0000188EE4FFFFFFAE030000F00C
:106050000000009CFEFFFF00000000A523240018A4
:106060008E9B030000A5F8FFFFF000000030000049
:10607000000000000031C80800188E9A030000A537
:10608000F8FFFFF0000000E3FFFFFF00000000F159
:106090002B0000188E9B030000AE030000F00000F0
:1060A000009CFEFFFF00000000A5232400188E5175
:1060B000070000A5F8FFFFF000000030000000001E
:1060C00000000031C80800188E52070000A5F8FF34
:1060D000FFF0000000E3FFFFFF00000000F12B00D5
:1060E00000188E51070000AD030000F00000009C76
:1060F000FEFFFF00000000A5232400188E080B00FF
:1061000000A6F8FFFFF000000030000000000000D3
:106110000031C80800188E080B0000A5F8FFFFF03A
:10612000000000E3FFFFFF00000000F12B0000185B
:106130008E080B0000AD030000F00000009CFEFF85
:10614000FF00000000A5232400188EBF0E0000A54C
:10615000F8FFFFF0000000300000000000000031F8
:10616000C80800188EBF0E0000A6F8FFFFF0000060
:1061700000E3FFFFFF00000000F12B0000188EBFBE
:106180000E0000AD030000F00000009CFEFFFF00C9
:10619000000000A5232400188E76120000A5F8FF49
:1061A000FFF0000000300000000000000031C808CF
:1061B00000188E76120000A5F8FFFFF0000000E343
:1061C000FFFFFF00000000F12B0000188E76120088
:1061D00000AE030000F00000009CFEFFFF00000086
:1061E00000A5232400188E2D160000A5F8FFFFF04F
:1061F000000000300000000000000031C808001856
:106200008E2C160000A5F8FFFFF0000000E3FFFF52
:10621000FF00000000F12B0000188E2D160000AECC
:10622000030000F00000009CFEFFFF00000000A53E
:10623000232400188EE3190000A5F8FFFFF00000EA
:1062400000300000000000000031C80800188EE493
:10625000190000A5F8FFFFF0000000E3FFFFFF00BA
:10626000000000F12B0000188EE3190000AE0300BF
:1062700000F00000009CFEFFFF00000000A52324AA
:1062800000188E9A1D0000A5F8FFFFF000000030F6
:106290000000000000000031C80800188E9B1D009F
:1062A00000A5F8FFFFF0000000E3FFFFFF00000083
:1062B00000F12B0000188E9A1D0000AD030000F0C5
:1062C0000000009CFEFFFF00000000A52324001832
:1062D0008E51210000A6F8FFFFF000000030000002
:1062E000000000000031C80800188E51210000A5F0
:1062F000F8FFFFF0000000E3FFFFFF00000000F1E7
:106300002B0000188E51210000AD030000F00000AA
:10631000009CFEFFFF00000000A5232400188E5102
:10632000210000AE030000F000000030000000007B
:10633000000000D99200001889088C51210000AD9E
:10634000030000F0000000000000000000000086D4
:106350000189188E42E6FFFFEFE9FFFF68010000A8
:106360000000000000000000A89A3000188E43E6EC
:10637000FFFFF0E9FFFF6801000000000000E3FFFD
:10638000FFFF1C5800001889908E42E6FFFFEFE9DE
:10639000FFFFF000000000000000EDFFFFFF0032F3
:1063A0000000188E42E6FFFFF0E9FFFFF00000005A
:1063B00000000000E3FFFFFFF22B0000188E4AF1FF
:1063C000FFFFF0E9FFFFF0000000000000009BFE6F
:1063D000FFFFA5232400188E43E6FFFF9DEDFFFF7E
:1063E000F00000000000000031000000EFC50800D0
:1063F000188E42E6FFFF9DEDFFFFF0000000000059
:106400000000E3FFFFFFF12B0000188E4AF1FFFFB1
:106410009DEDFFFFF0000000000000009BFEFFFF6D
:10642000A5232400188E42E6FFFF4AF1FFFFF0008B
:1064300000000000000031000000EFC50800188EC9
:1064400043E6FFFF4AF1FFFFF000000000000000FC
:10645000E3FFFFFFF12B0000188E4AF1FFFF4BF125
:10646000FFFFF0000000000000009CFEFFFFA523DE
:106470002400188E42E6FFFFF8F4FFFFF000000052
:106480000000000030000000EFC50800188E43E651
:10649000FFFFF8F4FFFFF000000000000000E3FF42
:1064A000FFFFF22B0000188E4AF1FFFFF7F4FFFF09
:1064B000F0000000000000009CFEFFFFA523240068
:1064C000188E42E6FFFFA6F8FFFFF0000000000074
:1064D000000030000000EFC50800188E42E6FFFF04
:1064E000A5F8FFFFF000000000000000E3FFFFFF41
:1064F000F22B0000188E4BF1FFFFA5F8FFFFF00014
:106500000000000000009CFEFFFFA5232400188E61
:1065100042E6FFFF53FCFFFFF00000000000000018
:1065200030000000EFC50800188E42E6FFFF52FC65
:10653000FFFFF000000000000000E3FFFFFFF22B70
:106540000000188E4BF1FFFF53FCFFFFF00000002E
:10655000000000009CFEFFFFA5232400188E42E6E9
:10656000FFFF00000000F00000000000000030000D
:106570000000EFC50800188E42E6FFFF0000000093
:10658000F000000000000000E3FFFFFFF22B00001E
:10659000188E4AF1FFFF00000000F000000000002C
:1065A00000009CFEFFFFA5232400188E43E6FFFF9A
:1065B000AD030000F000000000000000300000000B
:1065C000EFC50800188E42E6FFFFAE030000F000A2
:1065D000000000000000E3FFFFFFF22B0000188E18
:1065E0004AF1FFFFAD030000F000000000000000D2
:1065F0009CFEFFFFA5232400188E43E6FFFF5B07E8
:106600000000F00000000000000030000000EFC5B6
:106610000800188E42E6FFFF5B070000F000000054
:1066200000000000E3FFFFFFF22B0000188E4AF18C
:10663000FFFF5A070000F0000000000000009CFE71
:10664000FFFFA5232400188E42E6FFFF090B000080
:10665000F00000000000000030000000EFC508005E
:10666000188E43E6FFFF080B0000F000000000005A
:106670000000E3FFFFFFF12B0000188E4AF1FFFF3F
:10668000080B0000F0000000000000009CFEFFFF6F
:10669000A5232400188E42E6FFFFB50E0000F0008F
:1066A00000000000000030000000EFC50800188E58
:1066B00042E6FFFFB60E0000F00000000000000000
:1066C000E3FFFFFFF12B0000188E4BF1FFFFB60E2A
:1066D0000000F0000000000000009CFEFFFFA5236A
:1066E0002400188E42E6FFFF63120000F000000055
:1066F0000000000030000000EFC50800188E42E6E0
:10670000FFFF63120000F000000000000000E3FF44
:10671000FFFFF12B0000188E4BF1FFFF631200000A
:10672000F0000000000000009CFEFFFFA5232400F5
:10673000188E42E6FFFF10160000F0000000000077
:10674000000030000000EFC50800188E42E6FFFF91
:1067500010160000F000000000000000E3FFFFFF43
:10676000F12B0000188E4BF1FFFF11160000F00016
:106770000000000000009CFEFFFFA5232400188EEF
:10678000F7F4FFFF9DEDFFFF68010000000000002F
:1067900030000000BEA41E00188EF8F4FFFF9DED2F
:1067A000FFFFF000000000000000D0FFFFFFAE255B
:1067B0000000188EF8F4FFFF9DEDFFFFF0000000D1
:1067C00000000000E3FFFFFFF12B0000188EF8F43B
:1067D000FFFFA5F8FFFFF0000000000000009CFE96
:1067E000FFFFA5232400188EA5F8FFFF9DEDFFFFF6
:1067F000F00000000000000030000000EFC50800BD
:10680000188EA5F8FFFF9DEDFFFFF00000000000CF
:106810000000E3FFFFFFF12B0000188EA5F8FFFF3B
:10682000A5F8FFFFF0000000000000009CFEFFFF45
:10683000A5232400188E53FCFFFF9DEDFFFFF00001
:1068400000000000000030000000EFC50800188EB6
:1068500053FCFFFF9DEDFFFFF00000000000000073
:10686000E3FFFFFFF12B0000188E52FCFFFFA5F89D
:10687000FFFFF0000000000000009CFEFFFFA523CA
:106880002400188E000000009DEDFFFFF0000000C6
:106890000000000030000000EFC50800188E000066
:1068A00000009EEDFFFFF000000000000000E3FF8D
:1068B000FFFFF12B0000188E00000000A5F8FFFF7D
:1068C000F0000000000000009CFEFFFFA523240054
:1068D000188EAE0300009DEDFFFFF00000000000E9
:1068E000000030000000EFC50800188EAD03000066
:1068F0009DEDFFFFF000000000000000E3FFFFFF40
:10690000F12B0000188EAD030000A5F8FFFFF0008A
:106910000000000000009CFEFFFFA5232400188E4D
:106920005B0700009DEDFFFFF0000000000000008D
:1069300030000000EFC50800188E5B0700009DEDD9
:10694000FFFFF000000000000000E3FFFFFFF12B5D
:106950000000188E5B070000A5F8FFFFF0000000A4
:10696000000000009CFEFFFFA5232400188E080BEA
:1069700000009DEDFFFFF00000000000000030006F
:106980000000EFC50800188E080B00009DEDFFFF0A
:10699000F000000000000000E3FFFFFFF12B00000B
:1069A000188E080B0000A5F8FFFFF00000000000A3
:1069B00000009CFEFFFFA5232400188EB60E0000E9
:1069C0009DEDFFFFF000000000000000300000001F
:1069D000EFC50800188EB60E00009DEDFFFFF00019
:1069E000000000000000E3FFFFFFF12B0000188E05
:1069F000B50E0000A6F8FFFFF00000000000000048
:106A00009CFEFFFFA5232400188E631200009DED5D
:106A1000FFFFF00000000000000030000000EFC5A4
:106A20000800188E631200009DEDFFFFF0000000CB
:106A300000000000E3FFFFFFF12B0000188E63123F
:106A40000000A5F8FFFFF0000000000000009CFE21
:106A5000FFFFA5232400188E111600009DEDFFFFF7
:106A6000F00000000000000030000000EFC508004A
:106A7000188E101600009DEDFFFFF00000000000D2
:106A80000000E3FFFFFFF12B0000188E101600003E
:106A9000A5F8FFFFF0000000000000009CFEFFFFD3
:106AA000A5232400188EBE1900009DEDFFFFF00005
:106AB00000000000000030000000EFC50800188E44
:106AC000BE1900009DEDFFFFF00000000000000077
:106AD000E3FFFFFFF12B0000188EBE190000A5F8A0
:106AE000FFFFF0000000000000009CFEFFFFA52358
:106AF0002400188E6B1D00009DEDFFFFF0000000CC
:106B00000000000030000000EFC50800188E6B1D6B
:106B100000009DEDFFFFF000000000000000E3FF1B
:106B2000FFFFF12B0000188E6B1D0000A6F8FFFF81
:106B3000F0000000000000009CFEFFFFA5232400E1
:106B4000188E192100009DEDFFFFF00000000000ED
:106B5000000030000000EFC50800188E182100006A
:106B60009DEDFFFFF000000000000000E3FFFFFFCD
:106B7000F12B0000188E19210000A5F8FFFFF0008E
:106B80000000000000009CFEFFFFA52324001889E0
:106B9000108E18210000A5F8FFFF30F20000000061
:106BA0000000000000007CD178001888010A010272
:106BB00088010401FF891F86008800030200008607
:106BC00001880103020000860088001F020000887F
:106BD000011F020000891F5F0028060A1200002022
:106BE00020546865205265706C696361746F72200F
:106BF00020202000202020202D2D2D2D2D2D2D2D4D
:106C00002D2D20202020202000202020202020208A
:106C10002020202020202020202020202000466925
:106C2000726D776172652056657273696F6E20357B
:106C30002E2000436F6F6C210053746172742050DA
:106C40007265686561742100526967687420546FC9
:106C50006F6C004E4120004F4E20004F46460045CD
:106C600078747275646572004C65667420546F6F39
:106C70006C00506C6174666F726D0057656C636F69
:106C80006D65212020202020202020202020204948
:106C9000276D20746865205265706C696361746F3C
:106CA000722E20507265737320746865207265645B
:106CB000204D20746F202067657420737461727496
:106CC0006564212020202020202020004120626CAB
:106CD000696E6B696E6720274D27206D65616E7345
:106CE00049276D2077616974696E6720616E642041
:106CF00077696C6C636F6E74696E75652077686513
:106D00006E20796F7520202070726573732074680F
:106D10006520627574746F6E2E2E2E2000412073D4
:106D20006F6C696420274D27206D65616E7320208C
:106D30002049276D20776F726B696E6720616E64E2
:106D40002077696C6C757064617465206D7920734F
:106D50007461747573202020207768656E20492740
:106D60006D2066696E69736865642E2E2E004F75FE
:106D700072206E6578742073746570732077696C07
:106D80006C20676574206D652073657420757021B3
:106D900020202020202046697273742C20776527DC
:106DA0006C6C20726573746F72656D7920627569A1
:106DB0006C6420706C6174666F726D2E2E2E007381
:106DC0006F2069742773206E69636520616E64208B
:106DD0002020206C6576656C2E2049742773207006
:106DE000726F6261626C796120626974206F66669D
:106DF0002066726F6D2020202020207368697070DB
:106E0000696E672E2E2E202020202020202020009A
:106E1000416161682C2074686174206665656C73DB
:106E2000202020206D756368206265747465722E61
:106E300020202020202020204C6574277320676F9D
:106E4000206F6E20616E64206C6F6164736F6D657E
:106E500020706C6173746963212020202020202021
:106E6000005765276C6C2074727920616761696EC8
:106E70002120202020202020202020202020202011
:106E80002020202020202020202020202020202002
:106E900020202020202020202020202020202020F2
:106EA00020202020202020202020202020202020E2
:106EB00020005765276C6C206B65657020676F69D3
:106EC0006E6720202020616E64206C6F61642073E7
:106ED0006F6D6520202020202020706C6173746904
:106EE000632120466F722068656C7020676F746F35
:106EF000206D616B6572626F742E636F6D2F6865B4
:106F00006C70005765276C6C20676F20746F20745D
:106F10006865206D61696E6D656E752E204966200D
:106F2000796F75206E65656420202068656C70201F
:106F3000676F20746F3A2020202020202020206DB1
:106F4000616B6572626F742E636F6D2F68656C7014
:106F500020202000417765736F6D6521202020205F
:106F600020202020202020205765276C6C20676F70
:106F700020746F207468652053442020636172641C
:106F8000206D656E7520616E6420796F75202020FC
:106F900063616E2073656C6563742061206D6F643E
:106FA000656C21200049276D20676F696E6720742A
:106FB0006F206D616B6520202061207365726965AB
:106FC00073206F66206C696E657320736F77652020
:106FD00063616E2066696E64206D79202020202018
:106FE000206E6F7A7A6C6520616C69676E6D656E74
:106FF000742E202020004C6F6F6B20666F722074FF
:10700000686520626573742020206D617463686513
:1070100064206C696E6520696E20656163686178C3
:107020006973207365742E204C696E6573206172DC
:1070300065206E756D626572656420312D31332077
:10704000616E642E2E2E006C696E65206F6E652059
:1070500069732065787472612020206C6F6E672ED2
:1070600020546865205920617869732073657469BC
:1070700073206C656674206F6E2074686520706C78
:10708000617465616E64205820617869732069734A
:107090002072696768742E00477265617421202030
:1070A000492776652073617665642020746865736E
:1070B000652073657474696E677320616E64202047
:1070C00049276C6C20757365207468656D20746F3A
:1070D000202020206D616B65206E696365206D6FD7
:1070E00064656C73212020200053656C65637420F7
:1070F00062657374206C696E65732E005820417848
:107100006973204C696E65002D2D3E002020200003
:10711000592041786973204C696E6500446F6E6533
:1071200021004D792074656D7065726174757265AA
:107130002077617320206368616E676564206578DD
:107140007465726E616C6C792E20526573656C6526
:1071500063742066696C616D656E742020206D65B6
:107160006E7520746F2074727920616761696E2E6C
:10717000004D792065787472756465727320617250
:1071800065202020206E6F742068656174696E67C9
:107190002075702E2020202020436865636B206DB1
:1071A00079202020202020202020202020636F6EA6
:1071B0006E656374696F6E7321202020202020206B
:1071C0002000507265737320646F776E206F6E209D
:1071D000746865202020677265792072696E677314
:1071E00020617420746F70206F6674686520657804
:1071F0007472756465727320616E642020207075EE
:107200006C6C2074686520626C61636B2E2E2E207E
:10721000202000507265737320646F776E206F6E4C
:1072200020746865202020677265792072696E6716
:1072300020617420746F70206F662074686520650B
:107240007874727564657220616E642020202070ED
:10725000756C6C2074686520626C61636B2E2E2ED9
:107260002020200049276D2068656174696E6720C1
:107270007570206D79202020657874727564657250
:10728000212020202020202020202020506C6561FB
:10729000736520776169742E202020202020202013
:1072A00020202020202020202020202020202020DE
:1072B00020202020006775696465207475626573FD
:1072C000206F75742E204E6F776665656420666941
:1072D0006C616D656E742066726F6D2020746865D8
:1072E000206261636B207468726F756768207468D0
:1072F00065747562657320756E74696C2069742E8F
:107300002E2E2020200067756964652074756265E3
:10731000206F75742E20204E6F7766656564206639
:10732000696C616D656E742066726F6D2020746883
:1073300065206261636B207468726F756768207482
:1073400068657475626520756E74696C2069742E49
:107350002E2E2020202000706F7073206F757420F7
:10736000696E2066726F6E742E202049276D20682A
:10737000656174696E67207570206D7920202065C5
:107380007874727564657220736F2077652063610D
:107390006E20206C6F6164207468652066696C6182
:1073A0006D656E742E2E2E0054686973206D6967AA
:1073B00068742074616B65206120202066657720E9
:1073C0006D696E757465732E20202020202020208A
:1073D000416E64207761746368206F75742C20742B
:1073E000686520206E6F7A7A6C652077696C6C20F6
:1073F00067657420484F54210048656174696E6761
:107400002050726F67726573733A2020202020200D
:10741000202020202020202020202020202020206C
:10742000202020202020202020202020202020205C
:10743000202020202020202020202020202020204C
:10744000202020202020202020004F4B2049276D85
:107450002072656164792120202020202020466947
:10746000727374207765276C6C206C6F6164207474
:10747000686572696768742065787472756465728E
:107480002E2020202020507573682066696C616D65
:10749000656E7420696E2E2E2E2000477265617411
:1074A00021204E6F77207765276C6C202020206C80
:1074B0006F616420746865206C65667420202020EC
:1074C00020202065787472756465722E2050757363
:1074D0006820202020202066696C616D656E742014
:1074E0007468726F7567682E2E2E20004F4B2049EE
:1074F000276D2072656164792120202020202020C2
:1075000050757368207468652066696C616D656E7E
:1075100074202020646F776E207468726F756768BE
:107520002E2E2E2020202020202020202020202031
:10753000202020202020202020202020004F4B2011
:1075400049276D2072656164792120202020202048
:1075500020506F70207468652067756964652074B9
:1075600075626520206F666620616E642070757399
:1075700068207468652020202066696C616D656EE6
:1075800074207468726F7567682E2E2E20004F4B22
:107590002049276D207265616479212020202020F8
:1075A0002020506F702074686520677569646520BD
:1075B0007475626520206F666620616E6420707548
:1075C0006C6C202020202020202066696C616D6575
:1075D0006E742067656E746C792E2E2E20200074D8
:1075E000686520657874727564657220626C6F637B
:1075F0006B2020756E74696C20796F7520666565E7
:107600006C2074686520206D6F746F7220747567CC
:1076100067696E6720746865202020706C617374E0
:10762000696320696E2E2E2E20202020202020002D
:107630005768656E2066696C616D656E742069734C
:1076400020202020657874727564696E67206F75DC
:1076500074206F66207468656E6F7A7A6C652C2072
:10766000507265737320274D27202020746F20737C
:10767000746F7020657874727564696E672E20204F
:10768000005768656E2066696C616D656E7420696F
:107690007320202020657874727564696E67206F8E
:1076A0007574206F66207468656E6F7A7A6C652CCD
:1076B00020507265737320274D27202020746F207F
:1076C0006578697420202020202020202020202080
:1076D00020005768656E206D792066696C616D6564
:1076E0006E742069732072656C65617365642C200B
:1076F000202020202020202020205072657373201D
:10770000274D2720746F20657869742E2020202053
:107710002020202020202020202020202020202069
:10772000202000477265617421202049276C6C205D
:1077300073746F7020202072756E6E696E67206D95
:10774000792065787472756465722E5072657373F2
:10775000204D20746F20636F6E74696E75652E20E6
:107760002020202020202020202020202020202019
:10777000202020004F4B212049276C6C206B656531
:1077800070206D79202020206D6F746F72207275CB
:107790006E6E696E672E20596F7520206D6179209D
:1077A0006E65656420746F207075736820202020DA
:1077B0006861726465722E2E2E20202020202020E9
:1077C00020202020005765276C6C206B6565702099
:1077D000676F696E672E2020204C65747320747269
:1077E0007920746865206C65667420202065787443
:1077F00072756465722E20507573682020202020D9
:107800002066696C616D656E7420646F776E2E2ED4
:107810002E20202020005765276C6C206B6565703A
:1078200020676F696E672E202020496620796F756A
:1078300027726520686176696E6720202020747247
:107840006F75626C652C20636865636B206F75745F
:1078500020206D616B6572626F742E636F6D2F688F
:10786000656C70202020004D79206D6F746F722040
:1078700074696D6564206F7574202061667465722B
:107880002035206D696E757465732E202020205080
:1078900072657373204D20746F20657869742E2093
:1078A00020202020202020202020202020202020D8
:1078B0002020202020202000486F77276420697432
:1078C00020676F3F205265616479202000746F202B
:1078D0006D616B6520736F6D657468696E673F20BD
:1078E0002000596573202020004E6F2020202000AA
:1078F000446F6573206D79206E6F7A7A6C650068CD
:10790000656967687420636865636B206F75743F91
:10791000004D792068656967687420697320676F16
:107920006F6421004C65742773207472792061673D
:1079300061696E2E0044696420706C6173746963C0
:107940002065787472756465200066726F6D2074AE
:107950006865206E6F7A7A6C653F00556E6C6F615A
:107960006420726967687400556E6C6F6164004CC6
:107970006F6164206C65667400556E6C6F61642085
:107980006C656674004C6F6164207269676874008E
:107990004C6F61640020202020204A6F67206D6FAB
:1079A000646520202020202020002020202020206E
:1079B0002020582B202020202020202020200020A4
:1079C0002020202020284261636B29202020592D6F
:1079D0003E2020002020202020202020582D202064
:1079E00020202020202020200020202020202020B7
:1079F00020592B2020202020202020202000202063
:107A00003C2D5820284261636B2920205A2D3E20AE
:107A10002020002020202020202020592D20202040
:107A20002020202020202000202020202020202076
:107A30005A2D202020202020202020200020203C03
:107A40002D5920284261636B2920202020202020EE
:107A5000200020202020202020205A2B2020202001
:107A60002020202020200047414D45204F564552E0
:107A7000210048656174696E673A2020202020202B
:107A80002020202020200048656174696E673A003C
:107A9000202D2D25006572726F722100202020207C
:107AA00020202020202020202020202020202020D6
:107AB0000045787472756465723A2020202D2D2D52
:107AC0002F2D2D2D430052204578747275646572F8
:107AD0003A202D2D2D2F2D2D2D43004C204578742F
:107AE00072756465723A202D2D2D2F2D2D2D43009A
:107AF000506C6174666F726D3A2020202D2D2D2FF1
:107B00002D2D2D430020204E412020202000776184
:107B10006974696E6720002F2020204300432020D5
:107B2000202000205072656865617420536574746C
:107B3000696E677320202000526967687420546F53
:107B40006F6C20202020202020202020004C656603
:107B50007420546F6F6C20202020202020202020B3
:107B60002000506C6174666F726D202020202020F0
:107B70002020002052657365742053657474696E0B
:107B8000677320746F2020002044656661756C74F3
:107B90002076616C7565733F004275696C64205393
:107BA00074617469737469637320202000556E508A
:107BB0006175736520202020202020202020202097
:107BC0000050617573652020202020202020202077
:107BD000202020200043616E63656C204275696C33
:107BE0006420202020202020004368616E676520EB
:107BF00046696C616D656E742020202000536C65B1
:107C000065702028436F6C6420506175736529206E
:107C100000526573756D65204275696C6420202083
:107C200020202020004C454420436F6C6F722020A0
:107C30002020202020202020005245442020200009
:107C40004F52414E4745200050494E4B202000479F
:107C50005245454E2000424C55452020005055527B
:107C6000504C450057484954452000435553544F04
:107C70004D004F46462020200046696C616D656EC0
:107C8000742046616E2020202020202020004261A8
:107C9000636B20746F204D6F6E69746F72202020AB
:107CA00020004275696C642046696E69736865647A
:107CB00021202020202020202020202020202020C3
:107CC000202020202020202020204275696C642064
:107CD00054696D652020202020206820206D0042FE
:107CE00075696C642054696D653A202020202068F5
:107CF00020206D004C696E653A2020202020202035
:107D0000202020202020202000457374696D61749C
:107D10006564204275696C642054696D654C6966C0
:107D20006574696D6520546F74616C3A2020202061
:107D300068004C617374204275696C643A2020209D
:107D400020206820206D0043616E63656C2074689C
:107D50006973206275696C643F00517569742074A1
:107D60006869732070726F636573733F0042756951
:107D70006C642066726F6D205344202020202020E8
:107D8000005072656865617420202020202020202A
:107D900020202020005574696C6974696573202067
:107DA000202020202020202000496E666F20616E58
:107DB000642053657474696E67732020004D6F6E84
:107DC00069746F72204D6F64652020202020202070
:107DD000004368616E67652046696C616D656E740D
:107DE00020202020004C6576656C204275696C640B
:107DF00020506C6174652020004A6F67204D6F64CD
:107E000065202020202020202020202000486F6D89
:107E1000652041786573202020202020202020200C
:107E20000052756E205374617274757020536372C2
:107E30006970742000456E61626C652053746570D2
:107E400070657273202020200044697361626C6544
:107E50002053746570706572732020200053746F16
:107E60007020426C696E6B696E6721202020202093
:107E700000426C696E6B204C45447320202020200A
:107E8000202020200043616C696272617465204E7D
:107E90006F7A7A6C657320200065786974206D654F
:107EA0006E752020202020202020202000426F748A
:107EB00020537461746973746963732020202020D7
:107EC0000047656E6572616C2053657474696E67F6
:107ED00073202020005072656865617420536574BA
:107EE00074696E67732020200056657273696F6E27
:107EF000204E756D6265722020202020005265732F
:107F0000746F72652044656661756C7473202020FF
:107F100000536F756E642020202020202020202018
:107F2000202020200048656174656420506C6174D5
:107F30006500546F6F6C20436F756E742020202095
:107F400020202020200053494E474C4500445541F5
:107F50004C20200048656174204C4544732020204B
:107F6000202020202020200048656C702054657857
:107F700074202020202020202020200041636365E1
:107F80006C65726174652020202020202020200054
:107F90004E6F205344206361726420666F756E6477
:107FA00000534420636172642072656164206572CD
:107FB000726F7200492063616E277420726561647C
:107FC0002074686973202020534420636172642008
:107FD000666F726D617421202020202054727920F8
:107FE0007265666F726D617474696E6720202020FF
:107FF000746865206361726420746F204641543157
:10800000362E2000492063616E27742072656164FA
:108010002053442009202020636172647320776913
:1080200074682073746F7261676520206C61726779
:108030006572207468616E203247422E2020202015
:108040002020202020202020202020202020202030
:1080500020200020534420636172642072656164B3
:10806000206572726F72002049276D20616C726505
:10807000616479206275696C64696E67000100490A
:10808000033600FF006B00D100A000B800D500A6A9
:10809000000A0199003F018E0074018400A9017C4F
:1080A00000DE01740013026C00480265007D025D71
:1080B00000B2025600E7024E001C03460051033D89
:1080C0000086033200BB032200F0030300D0FEC091
:1080D000FF18FFD0FF63FFE0FFB1FFF0FF000000DB
:1080E0000051001000A4002000F8003000400140C2
:1080F00000A2015000F70160004B0270009F028057
:1081000000F20290004503A0009703B000E803C00E
:10811000003A04D0008C04E000DF04F000320500D7
:108120000186051001DB0520012F063001DA06501B
:10813000013007600186077001DC07800168089044
:10814000012039C9FFE03CE7FFF83F0000000000D4
:108150000008000000200319004006320060094BAF
:1081600000000A5000800C64000010800000665877
:108170009E58995B7664DB64186EAC6F317EF0823A
:108180006784F1926A948F959996D797249A88A6D6
:1081900069A74EABE5ABD7AC13AEAFB318B401B81B
:1081A000CABBC1DBA5DD27DF33E1EEE1CEE211245E
:1081B0001FBECFEFD1E2DEBFCDBF16E0A0E0B2E040
:1081C000EEEFFAEC01E00BBF02C007900D92A6356E
:1081D000B107D9F71AE1A6E5B6E001C01D92A834AF
:1081E000B107E1F711E8CEEAD1E800E006C0229736
:1081F0000109FE010BBF0E94B5E3CE36D10780E036
:108200000807A9F70E94C9640C947DE50C9400004E
:10821000CF92DF92EF92FF920F931F936B017C013D
:1082200020E030E040E05FE40E943B4587FD11C064
:10823000C701B60120E030E040E05FE40E94C142A7
:108240000E9445468B019C01005010402040304860
:1082500006C0C701B6010E9445468B019C01B801CA
:10826000C9011F910F91FF90EF90DF90CF9008957B
:10827000A0E0B0E0EEE3F1E40C9480E3EC014B010C
:10828000FA018881823008F442C1DB019C9192306E
:1082900008F43AC1843059F4943009F038C1998116
:1082A00011968C911197981709F02BC130C1943019
:1082B00009F42AC19230A9F4823009F028C1CE0114
:1082C00028E0DC010D90CD01DA010D92AD012150C5
:1082D000C1F7D40111968C911197998189238183DB
:1082E00015C1823009F410C1AA80BB80DB0112964F
:1082F0004D915C911397CC80DD80EE80FF801496C9
:108300000D911D912D913C911797C501841B950BE3
:10831000DC0197FF04C0AA27BB27A81BB90BA0321A
:10832000B1050CF06AC0181619068CF52801390140
:108330000A2E04C076946794579447940A94D2F70F
:1083400041E050E060E070E004C0440F551F661F3C
:10835000771FAA95D2F741505040604070404023AB
:1083600051236223732381E090E0A0E0B0E0411547
:1083700051056105710521F480E090E0A0E0B0E0D6
:108380008C019D01042915292629372942C000970F
:1083900009F43FC0AA0EBB1E260137010A2E04C0F5
:1083A00076946794579447940A94D2F741E050E04A
:1083B00060E070E004C0440F551F661F771FAA9548
:1083C000D2F741505040604070404C215D216E21F9
:1083D0007F2181E090E0A0E0B0E04115510561050A
:1083E000710521F480E090E0A0E0B0E06C017D0137
:1083F000C428D528E628F7280CC04A155B052CF4BC
:1084000000E010E020E030E004C05A01CC24DD247C
:1084100076018981D40111969C911197891709F4ED
:1084200045C0882329F00C191D092E093F0908C0F1
:10843000D701C601801B910BA20BB30B8C019D01D0
:1084400037FD04C01182B382A2820BC081E0818318
:10845000B382A28230952095109501951F4F2F4F22
:108460003F4F04831583268337830DC0880F991FE0
:10847000AA1FBB1F84839583A683B78382819381C0
:1084800001979383828384819581A681B781AC0112
:10849000BD0141505040604070404F3F2FEF5207A8
:1084A0002FEF62072FE3720708F30BC08183B382BB
:1084B000A2820C0D1D1D2E1D3F1D048315832683D6
:1084C000378383E08083448155816681778177FF9C
:1084D0001DC0DB01CA0181709070A070B0707695EC
:1084E000679557954795842B952BA62BB72B84839F
:1084F0009583A683B7838281938101969383828338
:1085000005C0CDE5D2E003C0E40101C0EF01CE011A
:10851000CDB7DEB7E0E10C949CE3A0E2B0E0E3E984
:10852000F2E40C948EE3DC01CB018D839E83AF8358
:10853000B88729833A834B835C83CE010596BE01BD
:10854000675E7F4F0E944348CE010196BE016F5E79
:108550007F4F0E944348CE014996BE016F5E7F4F18
:10856000AE01475F5F4F0E9438410E946947462F26
:10857000572F682F792FCB01BA01A096E2E00C9417
:10858000AAE3A0E2B0E0E7ECF2E40C948EE3DC01B5
:10859000CB018D839E83AF83B88729833A834B8336
:1085A0005C83CE010596BE01675E7F4F0E94434803
:1085B000CE010196BE016F5E7F4F0E9443488A89BB
:1085C00091E089278A8BCE014996BE016F5E7F4F6D
:1085D000AE01475F5F4F0E9438410E946947462FB6
:1085E000572F682F792FCB01BA01A096E2E00C94A7
:1085F000AAE3A0E2B0E0EFEFF2E40C9480E3DC0148
:10860000CB018D839E83AF83B88729833A834B83C5
:108610005C83CE010596BE01675E7F4F0E94434892
:10862000CE010196BE016F5E7F4F0E944348998D37
:10863000923078F089898230C0F0943019F4823019
:1086400041F4CCC0843019F4923079F4C7C0923030
:1086500051F481E02A8D9A89291709F480E08A8FE4
:10866000CE014996BDC0823051F481E02A8D9A89AD
:10867000291709F480E08A8BCE014196B1C04D8C58
:108680005E8C6F8C78A00D891E892F89388DE0E271
:10869000F0E040E050E060E070E08824992454016C
:1086A000CC24DD247601C201817090700097D9F04E
:1086B000C00ED11EE21EF31EDB01CA01880D991DFA
:1086C000AA1DBB1D41E050E060E070E0C016D1067D
:1086D000E206F30620F040E050E060E070E0480F72
:1086E000591F6A1F7B1F880C991CAA1CBB1C37FFD3
:1086F00008C081E090E0A0E0B0E0882A992AAA2A88
:10870000BB2A000F111F221F331F769467945794C2
:108710004794319741F68B8D9C8D2B893C89820F34
:10872000931F02969C878B8781E02A8D9A8929174F
:1087300009F480E08A872B853C8517C0CA018170C7
:108740009070009761F0F694E794D794C79480E016
:1087500090E0A0E0B0E8C82AD92AEA2AFB2A769558
:108760006795579547952F5F3F4F77FDE7CFC90135
:108770000BC0440F551F661F771FF7FC4160CC0CE0
:10878000DD1CEE1CFF1C01974030A0E05A07A0E062
:108790006A07A0E47A0768F38B879C87DB01CA012C
:1087A0008F779070A070B07080349105A105B105ED
:1087B00061F447FD0AC0C114D104E104F10429F0B9
:1087C000405C5F4F6F4F7F4F40784D875E876F876C
:1087D000788B83E08987CE01099602C08DE592E00F
:1087E0000E946947462F572F682F792FCB01BA0176
:1087F000A096E0E10C949CE3A8E1B0E0E2E0F4E4B0
:108800000C9488E3DC01CB018D839E83AF83B88712
:1088100029833A834B835C83CE010596BE016F5E4C
:108820007F4F0E944348CE010196BE01675F7F4F94
:108830000E9443489989923008F476C08985823035
:1088400008F475C02A893A8523272A8B943011F0C1
:10885000923021F4981709F067C06CC0843039F465
:108860001D8A1E8A1F8A188E1C8A1B8A5DC0823050
:1088700019F484E0898B58C02B893C898B859C85B1
:10888000281B390B3C8B2B8B8D899E89AF89B88D2A
:10889000CD84DE84EF84F8888C159D05AE05BF0578
:1088A00040F4880F991FAA1FBB1F215030403C8BFA
:1088B0002B8BEFE1F0E000E010E020E030E440E05E
:1088C00050E060E070E08C159D05AE05BF0540F0FE
:1088D000402B512B622B732B8C199D09AE09BF09BC
:1088E0003695279517950795880F991FAA1FBB1FC7
:1088F000319749F78A019B010F7710702070307013
:10890000003411052105310559F447FD09C00097D0
:10891000A105B10529F0405C5F4F6F4F7F4F407854
:108920004D8B5E8B6F8B788FCE01419605C0CE014B
:10893000099602C08DE592E00E946947462F572FA5
:10894000682F792FCB01BA016896E8E00C94A4E374
:10895000A8E1B0E0EEEAF4E40C948EE3DC01CB0194
:108960008D839E83AF83B88729833A834B835C834F
:10897000CE010596BE016F5E7F4F0E944348CE0137
:108980000196BE01675F7F4F0E944348898982300C
:1089900058F08985823040F0CE014196BE01675F74
:1089A0007F4F0E94AC4801C081E06896E2E00C94E1
:1089B000AAE3A8E1B0E0EFEDF4E40C948EE3DC016F
:1089C000CB018D839E83AF83B88729833A834B8302
:1089D0005C83CE010596BE016F5E7F4F0E944348C7
:1089E000CE010196BE01675F7F4F0E94434889898F
:1089F000823058F08985823040F0CE014196BE0128
:108A0000675F7F4F0E94AC4801C081E06896E2E05A
:108A10000C94AAE3A8E1B0E0E0E1F5E40C948EE365
:108A2000DC01CB018D839E83AF83B88729833A8392
:108A30004B835C83CE010596BE016F5E7F4F0E9423
:108A40004348CE010196BE01675F7F4F0E944348B5
:108A50008989823058F08985823040F0CE01419674
:108A6000BE01675F7F4F0E94AC4801C08FEF6896E0
:108A7000E2E00C94AAE3A8E1B0E0E1E4F5E40C94B0
:108A80008EE3DC01CB018D839E83AF83B88729837E
:108A90003A834B835C83CE010596BE016F5E7F4FA8
:108AA0000E944348CE010196BE01675F7F4F0E943E
:108AB00043488989823058F08985823040F0CE0160
:108AC0004196BE01675F7F4F0E94AC4801C08FEFA7
:108AD0006896E2E00C94AAE3A8E1B0E0E2E7F5E4EE
:108AE0000C948EE3DC01CB018D839E83AF83B8872A
:108AF00029833A834B835C83CE010596BE016F5E6A
:108B00007F4F0E944348CE010196BE01675F7F4FB1
:108B10000E9443488989823058F08985823040F02C
:108B2000CE014196BE01675F7F4F0E94AC4801C0F5
:108B300081E06896E2E00C94AAE3A8E1B0E0E3EA01
:108B4000F5E40C948EE3DC01CB018D839E83AF832F
:108B5000B88729833A834B835C83CE010596BE0197
:108B60006F5E7F4F0E944348CE010196BE01675F52
:108B70007F4F0E9443488989823058F0898582302E
:108B800040F0CE014196BE01675F7F4F0E94AC4826
:108B900001C081E06896E2E00C94AAE3CF92DF92F4
:108BA000EF92FF92CF93DF93CDB7DEB728970FB642
:108BB000F894DEBF0FBECDBF6B017C0183E08983DB
:108BC000D701C6018827B7FD83959927AA27BB2718
:108BD000282F8A83C114D104E104F10419F482E03E
:108BE000898335C08EE190E09C838B83222389F0BA
:108BF00080E0C81680E0D80680E0E80680E8F80645
:108C000059F1F094E094D094C094C11CD11CE11CA3
:108C1000F11CCD82DE82EF82F886C701B6010E9488
:108C2000154701971816190694F4082E04C0CC0CA9
:108C3000DD1CEE1CFF1C0A94D2F7CD82DE82EF828F
:108C4000F8862EE130E0281B390B3C832B83CE01C4
:108C500001960E94694704C060E070E080E09FECEC
:108C6000382F292F862F972FA32FB22FBC01CD018C
:108C700028960FB6F894DEBF0FBECDBFDF91CF911F
:108C8000FF90EF90DF90CF900895ACE0B0E0EBE480
:108C9000F6E40C948CE3DC01CB0189839A83AB83EB
:108CA000BC83CE010196BE016B5F7F4F0E9443489B
:108CB0008D81823069F1823058F1843039F02F8112
:108CC000388537FD25C02F31310544F08E8188234A
:108CD00021F100E010E020E030E823C08EE190E0D8
:108CE000821B930B09851A852B853C8504C036951C
:108CF0002795179507958A95D2F78E81882389F055
:108D000030952095109501951F4F2F4F3F4F09C06B
:108D100000E010E020E030E004C00FEF1FEF2FEF85
:108D20003FE7B801C9012C96E4E00C94A8E3A8E061
:108D3000B0E0EDE9F6E40C9488E36B017C011A8263
:108D4000611571058105910519F482E089835FC081
:108D500083E089830EE110E01C830B83CD82DE82E9
:108D6000EF82F886C701B6010E9415479C01215089
:108D7000304037FF39C0EE27FF27E21BF30B81E0BD
:108D800090E0A0E0B0E00E2E04C0880F991FAA1F4B
:108D9000BB1F0A94D2F70197A109B1098C219D212B
:108DA000AE21BF2141E050E060E070E00097A105F6
:108DB000B10521F440E050E060E070E004C0F694BA
:108DC000E794D794C794EA95D2F7C42AD52AE62A1D
:108DD000F72ACD82DE82EF82F8868EE190E0821B58
:108DE000930B9C838B8313C02115310581F0022ED8
:108DF00004C0CC0CDD1CEE1CFF1C0A94D2F7CD8203
:108E0000DE82EF82F886021B130B1C830B83CE01DC
:108E100001960E946947462F572F682F792FCB0163
:108E2000BA012896E8E00C94A4E3CF92DF92EF9287
:108E3000FF920F931F938B019C01003080E0180775
:108E400081E0280780E0380758F40F3F110521051D
:108E5000310509F090F480E090E0A0E0B0E016C0A9
:108E60000030E0E01E07E0E02E07E1E03E0750F4AE
:108E700080E190E0A0E0B0E009C088E090E0A0E0F0
:108E8000B0E004C088E190E0A0E0B0E040E250E053
:108E900060E070E0481B590B6A0B7B0B680179019D
:108EA00004C0F694E794D794C7948A95D2F7D70173
:108EB000C6018B599D4FFC018081481B51096109F6
:108EC0007109CA011F910F91FF90EF90DF90CF9031
:108ED0000895CF92DF92EF92FF920F931F93DC01E0
:108EE00014964D915D916D917C9117971196EC912F
:108EF00011978C91823020F460618FEF90E0A8C0D0
:108F0000843009F49FC0823009F496C041155105A0
:108F10006105710509F493C012968D919C91139788
:108F20002FEF823892070CF05BC022E83FEF281B3E
:108F3000390B2A3131056CF56A017B01022E04C020
:108F4000F694E794D794C7940A94D2F781E090E01E
:108F5000A0E0B0E004C0880F991FAA1FBB1F2A958C
:108F6000D2F70197A109B10984239523A623B7233A
:108F700041E050E060E070E00097A105B10521F408
:108F800040E050E060E070E04C295D296E297F29C7
:108F900004C040E050E060E070E0DB01CA018F7780
:108FA0009070A070B07080349105A105B10539F4BE
:108FB00047FF09C0405C5F4F6F4F7F4F04C0415C6B
:108FC0005F4F6F4F7F4F81E090E0403020E05207CD
:108FD00020E0620720E4720738F580E090E024C0CA
:108FE000803891057CF58A019B010F771070207005
:108FF0003070003411052105310539F447FF09C0EF
:10900000405C5F4F6F4F7F4F04C0415C5F4F6F4FBD
:109010007F4F77FD03C081589F4F06C076956795B7
:109020005795479580589F4F97E076956795579548
:1090300047959A95D1F70CC080E090E005C080E09C
:1090400090E006C08FEF90E040E050E060E070E01C
:10905000982F979599279795A62FAF77E795EE27A5
:10906000E79586953A2F392B282F2E2B842F952F75
:10907000A32FB22FBC01CD011F910F91FF90EF9054
:10908000DF90CF900895DC01FB014C9111965C912B
:10909000119712968C911297682F6F7770E0982F26
:1090A000991F9927991F13962C911397822F880F38
:1090B000892B90E0221F2227221F2183009739F558
:1090C000411551056105710511F482E029C082E85E
:1090D0009FEF9383828327E0440F551F661F771FFE
:1090E0002A95D1F783E0808309C0440F551F661F7E
:1090F000771F82819381019793838283403080E040
:10910000580780E0680780E4780778F320C08F3F35
:10911000910579F4411551056105710519F484E053
:109120008083089564FF03C081E0808310C01082B3
:109130000EC08F5790409383828383E0808387E0C3
:10914000440F551F661F771F8A95D1F770644483BB
:109150005583668377830895CF93FC01DB0190816B
:10916000923008F44CC08C91823008F448C094309E
:1091700069F42181843039F411968C91119790E033
:10918000821B910944C02223D1F13FC0843021F0D9
:10919000923041F48230B1F111968C91119788236D
:1091A000A1F12DC0C181823001F111968C911197EE
:1091B000C817D9F48281938112962D913C9113970F
:1091C0002817390794F082179307BCF04481558122
:1091D0006681778114968D919D910D90BC91A02D03
:1091E00084179507A607B70718F4CC2341F00DC0E4
:1091F000481759076A077B0728F4CC2331F081E030
:1092000090E005C080E090E002C08FEF9FEFCF912B
:109210000895F8942091E2063091E3068091E006EB
:109220009091E106821B930B789408958093D80661
:10923000089581E08093D60608958091D806089518
:109240008091D70608952091E2063091E30681E0EF
:109250002115310509F080E00895482F8091E2063C
:109260009091E3066091E0067091E10686179707FA
:10927000E8F42091E2063091E3068091E4069091B3
:10928000E506820F931F0E941AE3E091E606F09133
:10929000E706E80FF91F40838091E2069091E3060C
:1092A00001969093E3068093E206089581E0E0EE54
:1092B000F6E0808708951092E3061092E20610927D
:1092C000E5061092E4061092E8061092E906109264
:1092D000DA061092DB061092DC061092DD06109280
:1092E000D9061092D8061092D7061092D106109285
:1092F000D2061092D3061092D406109290061092C5
:10930000DE061092D0061092CF06089581E02091DB
:10931000CF063091D0062630310509F080E008955F
:109320006091DA067091DB068091DC069091DD0693
:1093300008951092DA061092DB061092DC06109265
:10934000DD0608954F925F926F927F928F929F9267
:10935000AF92BF92CF92DF92EF92FF920F931F9343
:10936000CF93DF93CDB7DEB7C656D0400FB6F89493
:10937000DEBF0FBECDBFCE01815B9F4F0E94227E1C
:10938000A4E7B6E0FE01E15BFF4F84E101900D929E
:109390008150E1F7CE010D9666E477E145E00E9449
:1093A000DEDE8F85882339F4ED85FE8590818989FD
:1093B000982381E009F480E08093730684E796E0C7
:1093C00060E070E00E94D77EFC0120813181428103
:1093D0005381A7962CAF3DAF4EAF5FAFA79784E701
:1093E00096E061E070E00E94D77EFC0140805180F1
:1093F0006280738084E796E062E070E00E94D77E2E
:10940000FC01C080D180E280F38084E796E063E0D5
:1094100070E00E94D77EFC0160817181828193811E
:109420000E94CE4527EE3CE840EC52E40E948D427B
:109430000E9445464B015C0184E796E064E070E0E1
:109440000E94D77E00D000D00DB71EB70F5F1F4F10
:10945000FC0160817181828193810E94CE4527EE5B
:109460003CE840EC52E40E948D420E944546DC01FB
:10947000CB01F80180839183A283B383CE01CB9685
:10948000A7964CAD5DAD6EAD7FADA7979301820100
:109490000E949B7E88E092E0A0E0B0E089879A87F6
:1094A000AB87BC870F900F900F900F90CE01CB969B
:1094B000BE01675F7F4F0E94D87989EF99E00E94D3
:1094C0009CB190938B0680938A0687EA9AE00E946B
:1094D0009CB190938D0680938C0685EB9CE00E9456
:1094E0009CB190938906809388068091D506882345
:1094F00091F089EF99E060E070E00E94CBB087EADC
:109500009AE060E070E00E94CBB085EB9CE060E008
:1095100070E00E94CBB0DE019796FE01FB9684E1DD
:1095200001900D928150E1F7CE01879662E070E0E4
:109530000E94D77E40E65AEE60E070E0FC01408376
:10954000518362837383DE015396FE01B79684E1F3
:1095500001900D928150E1F7CE01439660E070E0FA
:109560000E94D77E4EE557ED6FEF7FEFFC01408301
:10957000518362837383CE01439661E070E00E9461
:10958000D77E4AEC54EE6FEF7FEFFC0140835183AE
:10959000628373838CE890E0A0E0B0E08D839E83CB
:1095A000AF83B887CE018796BE016B5F7F4F0E9465
:1095B000D87982E890E0A0E0B0E089839A83AB8319
:1095C000BC83CE014396BE016F5F7F4F0E94D87966
:1095D00089EB99E060E00E94696CCA59DF4F0FB6D1
:1095E000F894DEBF0FBECDBFDF91CF911F910F91D9
:1095F000FF90EF90DF90CF90BF90AF909F908F90B3
:109600007F906F905F904F900895EF92FF920F932D
:109610001F93CF93DF93CDB7DEB76C970FB6F89457
:10962000DEBF0FBECDBFCE0109960E94227ECE01C5
:10963000099663E070E00E94D77E7C0104E716E0A3
:10964000C80163E070E00E94D77EFC0180819181B7
:10965000A281B381F70180839183A283B383CE017A
:10966000099664E070E00E94D77E7C01C80164E046
:1096700070E00E94D77EFC0180819181A281B3813C
:10968000F70180839183A283B383CE0109960E9460
:109690009A7DCE01099662E070E00E94D77E7C013F
:1096A000C80162E070E00E94D77EFC018081918158
:1096B000A281B381F70180839183A283B3838CE875
:1096C00090E0A0E0B0E08D839E83AF83B887CE01A9
:1096D0000996BE016B5F7F4F0E94D87982E890E0C7
:1096E000A0E0B0E089839A83AB83BC83C801BE014C
:1096F0006F5F7F4F0E94D87989EB99E06091730684
:109700000E94696C6C960FB6F894DEBF0FBECDBF99
:10971000DF91CF911F910F91FF90EF90089560918D
:109720008A0670918B0689EF99E00E94CBB0609118
:109730008C0670918D0687EA9AE00E94CBB060910A
:1097400088067091890685EB9CE00E94CBB085EB82
:109750009CE00E94B2B1882311F185EB9CE00E944D
:10976000CCB18823E1F489EF99E00E94CCB1882341
:1097700041F489EF99E061E00E94FEB181E08093BD
:10978000D90687EA9AE00E94CCB1882341F487EA9F
:109790009AE061E00E94FEB181E08093D9060895CD
:1097A000CF93DF93EB0170936A0360936903909109
:1097B000D706981709F44CC0882329F1209781F423
:1097C00081E08093D50689EA9BE06CE171E00E941C
:1097D0003BB581E090E090938F0680938E060FC09A
:1097E0006130710561F41092D50689EA9BE062E56B
:1097F00071E00E943BB5D0938F06C0938E0681E046
:109800008093D70625C080918E0690918F06813077
:10981000910529F410928F0610928E0617C082309F
:10982000910529F40E948F4B84E090E007C08330BB
:10983000910549F40E948F4B85E090E090938F064C
:1098400080938E0605C06230710511F41092D70620
:10985000DF91CF910895CF93DF93FC0182819381B3
:10986000009721F481E0818780E019C0848195818F
:1098700020813181B9010E941AE3C681D781C80FC6
:10988000D91F848195810196B9010E941AE39583BD
:109890008483828193810197938382838881DF917E
:1098A000CF910895EF92FF921F93CF93DF9300D053
:1098B000CDB7DEB780EEE82E86E0F82EC7010E9415
:1098C0002B4C682FC7016A830E942B4C782FC7014D
:1098D00079830E942B4C182FC7010E942B4C982F84
:1098E0006A817981812F0F900F90DF91CF911F9125
:1098F000FF90EF9008951F93CF93DF93C0EED6E0D3
:10990000CE010E942B4C182FCE010E942B4C982F79
:10991000812FDF91CF911F91089580EE96E00E94F4
:109920002B4C08953F924F925F926F927F928F924D
:109930009F92AF92BF92CF92DF92EF92FF920F93DE
:109940001F93CF93DF93CDB7DEB7CE56D0400FB67F
:10995000F894DEBF0FBECDBF8C018091DE06882358
:1099600009F0CEC10E948973882309F0C9C153C18F
:109970008091E2069091E3068931910508F4C0C117
:1099800089EB99E00E94F0680E948D4C81E090E0A4
:109990009093D0068093CF060E94524CAD966CAF48
:1099A0007DAF8EAF9FAFAD970E94524C8B019C0153
:1099B000AE962FAFAE97AF963FAFAF970E94524C87
:1099C0006B017C010E94524C4B015C010E94524C85
:1099D0002B013C010E94524CDC01CB0189839A830C
:1099E000AB83BC838091DA069091DB06A091DC0604
:1099F000B091DD060196A11DB11D8093DA0690930A
:109A0000DB06A093DC06B093DD06CE018B5A9F4F98
:109A10000E94227ECE018B5A9F4F62E070E00E942E
:109A2000D77EFC0180819181A601481B590BCA0198
:109A3000AE962FADAE97AF963FADAF9757FF03C031
:109A4000909581959F4FAA2797FDA095BA2F813AAF
:109A50005FE0950750E0A50750E0B50788F0AE96A7
:109A60002FAFAE97AF963FAFAF970E949573AE966C
:109A70002FADAE97AF963FADAF97882309F4D1C015
:109A800000D000D0EDB7FEB741825282638274826B
:109A9000CE018D96AD964CAD5DAD6EAD7FADAD9703
:109AA0000E949B7E0F900F900F900F90CE018D968D
:109AB000BE016F5F7F4F0E94D87922C18E3809F0B6
:109AC0001FC18091E2069091E3068A31910508F466
:109AD00017C189EB99E00E94F0680E948D4C81E0EB
:109AE00090E09093D0068093CF060E94524CAD96A2
:109AF0006CAF7DAF8EAF9FAFAD970E94524C8B0184
:109B00009C01AE962FAFAE97AF963FAFAF970E9436
:109B1000524C6B017C010E94524C4B015C010E9433
:109B2000524C2B013C010E94524CDC01CB01898339
:109B30009A83AB83BC830E948D4C382E8091DA06C9
:109B40009091DB06A091DC06B091DD060196A11D87
:109B5000B11D8093DA069093DB06A093DC06B093E8
:109B6000DD06CE018B5A9F4F0E94227ECE018B5A7A
:109B70009F4F62E070E00E94D77EFC01808191815E
:109B8000A601481B590BCA01AE962FADAE97AF96F2
:109B90003FADAF9757FF03C0909581959F4FAA2780
:109BA00097FDA095BA2F813A5FE0950750E0A50791
:109BB00050E0B50788F0AE962FAFAE97AF963FAFA7
:109BC000AF970E949573AE962FADAE97AF963FAD0F
:109BD000AF97882309F45CC000D000D0EDB7FEB782
:109BE0004182528263827482CE010596AD964CAD5D
:109BF0005DAD6EAD7FADAD970E949B7E0F900F90D7
:109C00000F900F90CE010596BE016F5F7F4F432DE1
:109C10000E945A7A75C0F80180818B3809F04ECFC6
:109C2000A7CE81E08093DE0600D000D0EDB7FEB76E
:109C30004182528263827482CE018F5B9F4FAD96C8
:109C40004CAD5DAD6EAD7FADAD970E949B7EAFE537
:109C5000B6E0FE01EF5BFF4F84E101900D92815071
:109C6000E1F710925706109258061092590610927A
:109C70005A061092560689819A81AB81BC818093E5
:109C80005B0690935C06A0935D06B0935E0634C0BD
:109C900081E08093DE0600D000D0EDB7FEB74182B0
:109CA000528263827482CE014996AD964CAD5DAD11
:109CB0006EAD7FADAD970E949B7EAFE5B6E0FE0135
:109CC000799684E101900D928150E1F789819A8122
:109CD000AB81BC818093570690935806A093590698
:109CE000B0935A063092560610925B0610925C06AC
:109CF00010925D0610925E060F900F900F900F90DD
:109D0000C259DF4F0FB6F894DEBF0FBECDBFDF9153
:109D1000CF911F910F91FF90EF90DF90CF90BF9068
:109D2000AF909F908F907F906F905F904F903F90FB
:109D300008951F93CF93DF930E948D4C182F0E949C
:109D40008D4CC82F0E948D4CCA3009F4D5C0CB3041
:109D5000B0F4C63009F4CDC0C73050F4C43009F4B3
:109D6000CBC0C53008F0C8C0C33009F0C8C01DC0A2
:109D7000C83009F4C1C0C93008F0BEC0BAC0CE3086
:109D800009F4BAC0CF3038F4CC3009F465C0CD3016
:109D900008F073C0B1C0C73109F457C0CF3109F41E
:109DA00077C0CF3009F0ABC0A7C0113019F4CEE8AE
:109DB000DAE002C0C0EED9E00E947B4CBC01CE01CB
:109DC00049960E94CBB085EB9CE00E94B2B18823FB
:109DD00009F49CC085EB9CE00E94CCB1882309F07B
:109DE00095C0113019F48EE89AE002C080EE99E037
:109DF00049960E94CCB1882309F088C081E0809305
:109E0000D906113019F48EE89AE002C080EE99E08C
:109E1000499661E004C08EE89AE0499660E00E94AD
:109E2000FEB189EB99E061E070E040E00E94AC6631
:109E3000113009F066C00E940E5A882309F461C0EF
:109E400089EB99E068E871E050C09091D80681E014
:109E500089270E94875E55C0113019F4CEE8DAE0F8
:109E600002C0C0EED9E00E948D4C682F70E0617096
:109E70007070CE010E94579744C00E948D4C682F8D
:109E800070E06170707089EB99E00E94696C39C074
:109E900089EB99E061E00E94646C0E947B4CBC01FC
:109EA00085EB9CE00E94CBB085EB9CE00E94CCB19E
:109EB000C1E0C827C093D90689EF99E06C2F0E94B2
:109EC000FEB187EA9AE06C2F0E94FEB189EB99E01F
:109ED00061E070E040E00E94AC660E94E05A882396
:109EE00081F489EB99E069ED71E040E00E948E69B0
:109EF00008C00E94524C05C00E948D4C02C080E0F8
:109F000001C081E0DF91CF911F910895113009F4D4
:109F100082CF80EE99E081CF4F925F926F927F92D5
:109F20008F929F92AF92BF92CF92DF92EF92FF9269
:109F30000F931F93CF93DF93CDB7DEB7C956D040B1
:109F40000FB6F894DEBF0FBECDBF0E946C81882390
:109F500009F5D5C02091E2063091E3068091E40630
:109F60009091E506820F931F0E941AE3E091E606A6
:109F7000F091E706E80FF91F40838091E206909187
:109F8000E30601969093E3068093E20604C00093F3
:109F9000E80601C001E08091E2069091E30620917D
:109FA000E0063091E1062817390711F40C94265881
:109FB0000E94D981882311F40C9426588091D106EF
:109FC0009091D206A091D306B091D4060196A11D1E
:109FD000B11D8093D1069093D206A093D306B0937F
:109FE000D4060E94DC81482F8091E2069091E3061E
:109FF0006091E0067091E1068617970708F4AACFF2
:10A00000C6CFC090D106D090D206E090D306F09093
:10A01000D4060E941D81DC01CB01C816D906EA06D0
:10A02000FB0610F00C942C5880919006882311F0B8
:10A030000C942C5889EA9BE00E9497B489EB99E034
:10A040006AE272E040E00E948E6981E080939006AF
:10A050000E94107C1092E3061092E2061092E50630
:10A060001092E4061092E8061092E90689EF99E052
:10A0700060E070E00E94CBB087EA9AE060E070E0B8
:10A080000E94CBB085EB9CE060E070E00E94CBB01A
:10A09000CE01805B9F4F0E94227ECE01805B9F4F4E
:10A0A00062E070E00E94D77E40E65AEE60E070E029
:10A0B000DC014D935D936D937C9313971092D806BA
:10A0C00086E990E0A0E0B0E08E839F83A887B987FF
:10A0D000CE01805B9F4FBE016A5F7F4F0E94D8799F
:10A0E0000CC08091E2069091E306009741F48091C4
:10A0F000CF069091D006009711F40E94EB810E9448
:10A10000B193882309F550C02091E2063091E3060F
:10A110008091E4069091E506820F931F0E941AE356
:10A12000E091E606F091E706E80FF91F4083809181
:10A13000E2069091E30601969093E3068093E2068F
:10A1400004C00093E80601C001E08091E20690910E
:10A15000E3062091E0063091E1062817390709F45B
:10A1600081C70E94BA93882309F47CC70E94C893D0
:10A17000482F8091E2069091E3066091E00670918D
:10A18000E1068617970708F4BFCFDBCF8091E20680
:10A190009091E306009741F48091CF069091D0060C
:10A1A000009711F40E9464948091D906882391F05D
:10A1B00085EB9CE00E9478B1882361F089EF99E0FB
:10A1C00060E00E94FEB187EA9AE060E00E94FEB182
:10A1D0001092D9068091D806882309F05FC7809134
:10A1E000D606882309F05AC78091CF069091D006F1
:10A1F0008330910581F40E94C484882341F081EB6F
:10A2000096E00E9465E1882331F00E94107C109254
:10A21000D0061092CF068091CF069091D006813063
:10A22000910509F09FC00E94C484882339F580916C
:10A23000DE068823F1F08091570690915806A09190
:10A240005906B0915A060097A105B10539F48FE57A
:10A2500096E06BE576E00E94D87908C08FE596E03D
:10A2600067E576E0409156060E945A7A1092DE0623
:10A2700079C01092D0061092CF0674C08091E20689
:10A280009091E306009709F46DC08091D70688236A
:10A2900009F068C089EB99E00E94F0688091E406BB
:10A2A0009091E5066091E0067091E1060E941AE344
:10A2B000E091E606F091E706E80FF91F80818983B7
:10A2C0008B3811F08E3829F4CE0101960E94924C01
:10A2D00049C0893801F58091E2069091E306823009
:10A2E000910508F43FC00E948D4C0E948D4C8091D6
:10A2F000DA069091DB06A091DC06B091DD060196AE
:10A30000A11DB11D8093DA069093DB06A093DC06B5
:10A31000B093DD0627C0863929F58091E206909139
:10A32000E30683309105F0F00E948D4C0E948D4C25
:10A33000082F0E948D4C4091DA065091DB06609107
:10A34000DC067091DD064F5F5F4F6F4F7F4F40938C
:10A35000DA065093DB066093DC067093DD06802FEF
:10A360000E94E4B38091CF069091D006823091058F
:10A3700051F480EC96E00E9465E1882321F0109270
:10A38000D0061092CF068091CF069091D0068430EF
:10A39000910509F04BC082EA96E00E9465E18823AE
:10A3A00041F089EB99E06BE772E040E00E948E6932
:10A3B00039C08091DF06813019F48EE89AE002C03E
:10A3C00080EE99E049960E9478B1882309F450C63E
:10A3D0008091DF06813019F48EE89AE002C080EEA9
:10A3E00099E081579F4FFC018081882309F040C686
:10A3F00087E00E94726F16C080EE99E049960E9435
:10A40000B2B1882399F48091DF06813019F48EE887
:10A410009AE002C080EE99E081579F4FDC018C9159
:10A42000882321F41092D0061092CF068091CF0697
:10A430009091D00685309105F1F482EA96E00E9471
:10A4400065E1882341F089EB99E060EB72E040E040
:10A450000E948E690CC085EB9CE00E94B2B18823FB
:10A4600031F085EB9CE00E9478B1882321F01092B6
:10A47000D0061092CF068091CF069091D0068630FC
:10A48000910561F583E996E00E9465E1882351F02A
:10A490008091910681FF1EC089EB99E060E00E94E7
:10A4A000A06C1CC089EA9BE00E94F9B78823B1F038
:10A4B0008091910682FF04C089EA9BE00E94C4B5A6
:10A4C00089EB99E060E070E040E050E00E9459695B
:10A4D0000E9488991092D0061092CF068091CF06E4
:10A4E0009091D006009709F094C58091D7068823F3
:10A4F00009F4AAC080918E0690918F068130910553
:10A50000C9F48091690390916A03009729F489EA5C
:10A510009BE065EE72E007C08130910531F489EA75
:10A520009BE063E373E00E943BB50E94A24982E096
:10A5300090E00DC08230910509F0A2C50E94C4844C
:10A54000882309F09DC50E94FDB383E090E09093BD
:10A550008F0680938E06A2C50E94C484882341F092
:10A5600080918E0690918F068530910509F091C5F6
:10A5700089EA9BE065E673E00E943BB51092DF0636
:10A5800085E090E09093D0068093CF0682EA96E033
:10A5900040E052ED69E47BE60E943FE186E090E016
:10A5A00090938F0680938E0689EB99E063E040E0FC
:10A5B00024E10E94D46672C51092DF0684E090E028
:10A5C0009093D0068093CF0682EA96E040E052ED69
:10A5D00069E47BE60E943FE187E090E0B8CF8730F6
:10A5E0009105A1F481E08093DF0684E090E09093F0
:10A5F000D0068093CF0682EA96E040E052ED69E40F
:10A600007BE60E943FE188E090E0A1CF8830910591
:10A6100049F489EB99E00E94EA660E94054B89E0C3
:10A6200090E095CF8930910509F038C50E94C48427
:10A63000882309F033C510928F0610928E060E946F
:10A64000FDB31092D7062AC58091E2069091E306E9
:10A65000009709F4DEC489EB99E00E94F0688091CC
:10A66000E4069091E5062091E0063091E106E09144
:10A67000E606F091E706B9010E941AE38E0F9F1FCC
:10A68000DC018C9189838B3811F08E3829F4CE014E
:10A6900001960E94924CBDC4863829F58091E2064D
:10A6A0009091E3068230910508F4B3C40E948D4C6A
:10A6B0000E948D4C8093DF064091DA065091DB06B4
:10A6C0006091DC067091DD064F5F5F4F6F4F7F4FEB
:10A6D0004093DA065093DB066093DC067093DD0648
:10A6E0000E94047C96C48938D9F58091E206909145
:10A6F000E3068230910508F48CC40E948D4C0E94C0
:10A700008D4C4091DA065091DB066091DC06709129
:10A71000DD064F5F5F4F6F4F7F4F4093DA065093D8
:10A72000DB066093DC067093DD06F82EFF1CFF2429
:10A73000FF1C00E010E0C82EDD24C601002E02C080
:10A74000959587950A94E2F780FF04C0802F6F2DBE
:10A750000E94568C0F5F1F4F0530110571F759C4C9
:10A760008C3809F054C08091E2069091E30685315F
:10A77000910508F44EC40E948D4C0E94524C6B010E
:10A780007C010E94524C2B013C010E94524C4B0117
:10A790005C010E94524CA8966CAF7DAF8EAF9FAF0C
:10A7A000A8970E94524CAB01BC018091DA069091AF
:10A7B000DB06A091DC06B091DD060196A11DB11D5E
:10A7C0008093DA069093DB06A093DC06B093DD0657
:10A7D00000D000D0EDB7FEB741835283638374830A
:10A7E000CE01CC96B701A6019301820175016401E7
:10A7F000A8968CAC9DACAEACBFACA8970E949B7EDB
:10A800000F900F900F900F90CE01CC9675C28538A7
:10A81000A1F58091E2069091E3068530910508F458
:10A82000F8C382E090E09093D0068093CF060E9418
:10A830008D4C0E94524CAB01BC018091DA06909184
:10A84000DB06A091DC06B091DD060196A11DB11DCD
:10A850008093DA069093DB06A093DC06B093DD06C6
:10A86000CB01BA0128EE33E040E050E00E94EFE275
:10A87000AB01BC0180EC96E090C1843909F049C07D
:10A880008091E2069091E3068530910508F4C1C3FA
:10A890000E948D4C0E948D4C809392060E947B4CAE
:10A8A0008C010E948D4C809391068091DA069091E4
:10A8B000DB06A091DC06B091DD060196A11DB11D5D
:10A8C0008093DA069093DB06A093DC06B093DD0656
:10A8D0000115110581F0B80180E090E020E432E438
:10A8E0004FE050E00E94EFE2AB01BC0183E996E04B
:10A8F0000E943FE1A1C0CE0149960E943BE1A3E93D
:10A90000B6E0FE0179968FE001900D928150E1F75B
:10A9100093C0853909F0A5C089EA9BE00E94BDB4C7
:10A920006C018091E2069091E3068630910508F46F
:10A9300070C30E948D4C0E948D4C082F0E948D4C3C
:10A94000882E0E948D4CE82E0E948D4CF82E40914E
:10A95000DA065091DB066091DC067091DD064F5FF0
:10A960005F4F6F4F7F4F4093DA065093DB06609343
:10A97000DC067093DD0610E000FD03C0C6010E94F6
:10A980001AD8D60112968C9212971396EC92C601A1
:10A9900060EE76E00E947BD701FF3BC3E091860C1E
:10A9A000FF27E7FDF095EE0FFF1FE858F34F80817A
:10A9B00091818C159D0531F089EA9BE0B6010E94DA
:10A9C000C8B403C0C6010E9469D804701070FF208B
:10A9D00039F00115110521F4C6016F2D0E9453D8DD
:10A9E0000115110509F415C3FF2089F06F2D70E0E2
:10A9F00080E090E020E432E44FE050E00E94EFE29B
:10AA0000AB01BC0183E996E00E943FE10DC0CE019D
:10AA10000A960E943BE1A3E9B6E0FE013A968FE078
:10AA200001900D928150E1F781E080939206809130
:10AA3000910684708093910689EB99E069E170E05A
:10AA40004FE050E00E94596989EA9BE060919206CC
:10AA50000E94F4B786E090E09093D0068093CF06F2
:10AA6000D8C2982F9358923008F047C08091E206E0
:10AA70009091E3068830910508F4CBC20E948D4C7A
:10AA80000E948D4C082F0E94524C6B017C010E9449
:10AA90007B4C4091DA065091DB066091DC067091A8
:10AAA000DD064F5F5F4F6F4F7F4F4093DA06509345
:10AAB000DB066093DC067093DD0623E030E0309324
:10AAC000D0062093CF06BC0180E090E020E432E481
:10AAD0004FE050E00E94EFE2AB01BC0181EB96E059
:10AAE0000E943FE181E09981943809F080E0602F75
:10AAF000A70196010E94388B8CC28738A9F48091F7
:10AB0000E2069091E3068630910508F482C284E063
:10AB100090E09093D0068093CF060E948D4C0E94C7
:10AB20008D4C8093DF0614C08D38D1F58091E206FC
:10AB30009091E3068630910508F46BC285E090E0C1
:10AB40009093D0068093CF060E948D4C0E948D4C2E
:10AB50000E947B4C0E947B4C4091DA065091DB06B0
:10AB60006091DC067091DD064F5F5F4F6F4F7F4F46
:10AB70004093DA065093DB066093DC067093DD06A3
:10AB8000BC0180E090E020E432E44FE050E00E941D
:10AB9000EFE2AB01BC0182EA96E00E943FE139C2DC
:10ABA0008F3809F055C08091E2069091E30682301B
:10ABB000910508F42EC20E948D4C0E948D4C40914C
:10ABC000DA065091DB066091DC067091DD064F5F7E
:10ABD0005F4F6F4F7F4F4093DA065093DB066093D1
:10ABE000DC067093DD06EEE0EE2EF12C00E010E0C6
:10ABF000C82EDD24C601002E02C0959587950A94C3
:10AC0000E2F780FF1BC0CE0188960E949686CE0197
:10AC10008896B8010E94CF7EFC0180819181A2813B
:10AC2000B3818A839B83AC83BD83F894CE01029663
:10AC3000B70144E050E00E942CE578940F5F1F4F6D
:10AC400084E090E0E80EF91E0530110599F6E1C1A7
:10AC5000803909F054C08091E2069091E306823079
:10AC6000910508F4D6C10E948D4C0E948D4C482E4F
:10AC70008091DA069091DB06A091DC06B091DD06AA
:10AC80000196A11DB11D8093DA069093DB06A09377
:10AC9000DC06B093DD0620E5C22ED12CCC0EDD1EE5
:10ACA000C6010E9496863EE0E32EF12C00E010E003
:10ACB00055248C2CCD2CC201002E02C09595879571
:10ACC0000A94E2F780FF0CC0F894882D9C2DB801FF
:10ACD0000E94D77EB70144E050E00E9416E57894C8
:10ACE0000F5F1F4FA4E0B0E0EA0EFB1E0530110518
:10ACF00011F7CE01805B9F4F0E949A7D8AC18139F6
:10AD000049F58091E2069091E3068330910508F4BD
:10AD100080C10E948D4C0E948D4C082F0E948D4C4A
:10AD2000982F4091DA065091DB066091DC06709115
:10AD3000DD064F5F5F4F6F4F7F4F4093DA065093B2
:10AD4000DB066093DC067093DD06802F692F0E947E
:10AD5000A68C5FC18239C9F58091E2069091E30625
:10AD60008630910508F455C10E948D4C0E948D4C8F
:10AD7000F82E0E948D4CAA968FAFAA970E948D4CF8
:10AD8000A9968FAFA9970E948D4C0E948D4C00917F
:10AD9000DA061091DB062091DC063091DD060F5FAC
:10ADA0001F4F2F4F3F4F0093DA061093DB0620937F
:10ADB000DC063093DD068F2DAA966FADAA97A99673
:10ADC0004FADA9970E94769924C1833951F580919E
:10ADD000E2069091E3068630910508F41AC10E94BC
:10ADE0008D4C0E947B4C8C010E947B4C6C010E941C
:10ADF0008D4C8091DA069091DB06A091DC06B09133
:10AE0000DD060196A11DB11D8093DA069093DB0645
:10AE1000A093DC06B093DD06C801B6010E940D6F59
:10AE2000F8C08838B1F58091E2069091E30684304D
:10AE3000910508F4EEC08091E4069091E50600913A
:10AE4000E2061091E3060396B9010E941AE38E0F01
:10AE50009F1FFC01808190E004960817190708F4F1
:10AE6000D8C00E948D4C8091DA069091DB06A091AB
:10AE7000DC06B091DD060196A11DB11D8093DA06B6
:10AE80009093DB06A093DC06B093DD060E94994EFA
:10AE9000C0C0863939F58091E2069091E30683308F
:10AEA000910508F4B6C00E948D4C0E948D4C082F6D
:10AEB0000E948D4C4091DA065091DB066091DC06D1
:10AEC0007091DD064F5F5F4F6F4F7F4F4093DA0603
:10AED0005093DB066093DC067093DD06802F0E94A2
:10AEE000E4B397C0873919F58091E2069091E306A3
:10AEF0008230910508F48DC00E948D4C0E948D4CCB
:10AF00004091DA065091DB066091DC067091DD0617
:10AF10004F5F5F4F6F4F7F4F4093DA065093DB06D2
:10AF20006093DC067093DD060E94726F72C08839F0
:10AF300039F58091E2069091E3068230910508F49C
:10AF400068C00E948D4C0E948D4C8091DA069091D1
:10AF5000DB06A091DC06B091DD060196A11DB11DB6
:10AF60008093DA069093DB06A093DC06B093DD06AF
:10AF70000E94635A89EB99E060E00E94A06C49C08E
:10AF8000893921F58091E2069091E306853091059B
:10AF900008F43FC00E948D4C0E94524C8091DA060A
:10AFA0009091DB06A091DC06B091DD060196A11D13
:10AFB000B11D8093DA069093DB06A093DC06B09374
:10AFC000DD0680EE96E00E94DC5E23C08A3909F53A
:10AFD0008091E2069091E30682309105D0F00E94C4
:10AFE0008D4C0E948D4C4091DA065091DB066091A9
:10AFF000DC067091DD064F5F5F4F6F4F7F4F4093D0
:10B00000DA065093DB066093DC067093DD060E943F
:10B01000F45F8091DA069091DB06A091DC06B09196
:10B02000DD068130FAEC9F07FAE9AF07FBE3BF07C3
:10B03000A8F181E09AECAAE9BBE38093DA06909349
:10B04000DB06A093DC06B093DD0628C00E94D98100
:10B05000882311F40C9401500E94D981882309F4AB
:10B0600040C84DC80E94BA93882309F48FC89CC871
:10B070008091DF06813009F0BFC98EE89AE0BEC931
:10B0800080918E0690918F068430910509F068CAF0
:10B0900063CA8630910509F0A2CA8ECAC759DF4F2C
:10B0A0000FB6F894DEBF0FBECDBFDF91CF911F91D9
:10B0B0000F91FF90EF90DF90CF90BF90AF909F9057
:10B0C0008F907F906F905F904F9008958AEE98E0F8
:10B0D00064E477E140E00E94DEDE80E092E090935D
:10B0E000E1068093E0061092E3061092E2061092C9
:10B0F000E5061092E4068AEE96E09093E7068093C8
:10B10000E6061092E8061092E90680EC96E00E94AE
:10B110003BE181EB96E00E943BE182EA96E00E94EF
:10B120003BE183E996E00E943BE184E796E00E94E0
:10B130009A7E8FE596E00E949A7E089586E199E0D6
:10B1400064E477E140E00E94DEDE80EF98E00E9458
:10B1500041DE0895CF93DF9300D0CDB7DEB7BC01B9
:10B1600081E0898382E38A83CE01019642E050E048
:10B170000E942CE50F900F90DF91CF910895CF930F
:10B18000DF93EC0140E050E060EE70E40E944EAFCF
:10B19000CE01029646E656E666EA7EE30E944EAF90
:10B1A000CE01049640E050E060E172E40E944EAFB0
:10B1B000DF91CF9108950F931F93CF93DF938B016E
:10B1C000EB016896009719F4CB0167E002C0CB0150
:10B1D00068E30E9436E5CE0162E30E9436E5C801CD
:10B1E0000A960E94BF58C80140960E94BF58C801E5
:10B1F0004A960E94AA58C801069664EF71E00E9420
:10B200004CE5C801029665E070E00E944CE5C8017B
:10B21000049664EF71E00E944CE5C80108966CE268
:10B2200071E00E944CE5DF91CF911F910F9108953D
:10B23000CF93DF93EC0140EA56E861E070E00E94B2
:10B2400044E5CE01049649E150E060E070E00E94E0
:10B2500044E5CE01089643EE5FE060E070E00E94B6
:10B2600044E5BE01605F7F4F8DE790E840E550E028
:10B270000E942CE5DF91CF9108950F931F93CF93F8
:10B28000DF9300D00F92CDB7DEB78C0160E00E9453
:10B2900036E5C801029661E00E9436E58FEF8983AA
:10B2A0001B821A82B8016C5F7F4FCE01019643E08A
:10B2B00050E00E942CE50F900F900F90DF91CF91FE
:10B2C0001F910F910895FF920F931F93CF93DF93D8
:10B2D00000D000D0CDB7DEB7F82E062F1FB7F894F8
:10B2E00080E491E068E04C830E9436E5F9820A83AD
:10B2F0004C814B83CE01019664E471E043E050E061
:10B300000E942CE51FBF0F900F900F900F90DF91C0
:10B31000CF911F910F91FF90089561E00E9436E553
:10B320000895CF93DF93EC0166EE70E00E944CE548
:10B33000CE01029666EE70E00E944CE5CE010496C6
:10B340006EE670E00E944CE5CE01069665E00E9434
:10B3500036E5DF91CF910895CF93CFB7F8948EE67D
:10B3600091E061E00E9436E580E791E060ED77E0F2
:10B370000E944CE582E791E06CED75E00E944CE59F
:10B3800084E791E06CED75E00E944CE586E791E082
:10B3900068EE73E00E944CE588E791E068EB7BE0A3
:10B3A0000E944CE58AE791E068EB7BE00E944CE567
:10B3B0008CE791E040E050E060EA71E40E944EAF1B
:10B3C0008EE791E040E050E060EA71E40E944EAF09
:10B3D00080E891E040E050E060E87FE30E944EAFFB
:10B3E00082E891E040E050E060E070E40E944EAFFF
:10B3F00084E891E040E050E060E070E40E944EAFED
:10B4000086E891E06FE070E00E944CE588E891E00A
:10B4100068E00E9436E5CFBFCF91089582E490E0C6
:10B4200061E00E941BAE91E0813009F090E0892F2D
:10B4300008951F93CF93DF93CDB7DEB764970FB610
:10B44000F894DEBF0FBECDBFDE011196E0E0F2E062
:10B4500084E101900D928150E1F70E940E5A8823F9
:10B4600081F085EE97E3A0E0B0E089839A83AB8317
:10B47000BC838AE79AE1A0E0B0E08D839E83AF832E
:10B48000B8871FB7F894CE0101966EE070E044E1F2
:10B4900050E00E942CE51FBF64960FB6F894DEBF03
:10B4A0000FBECDBFDF91CF911F910895CF93682F2D
:10B4B000CFB7F89482E490E00E9436E50E94195AD2
:10B4C000CFBFCF9108951F93CF93DF93CDB7DEB752
:10B4D00029970FB6F894DEBF0FBECDBFDE011596DB
:10B4E000E3E2F2E085E001900D928150E1F71FB7B1
:10B4F000F89484E192E062E270E044E150E00E945E
:10B500002CE581EC93E29A83898384E193ED9C831B
:10B510008B83CE01059666E070E045E050E00E9426
:10B520002CE584E090E06FE90E9436E58CE090E045
:10B530006BE10E9436E50E94195A80E793E06CE8BF
:10B5400071E044E150E00E942CE50E94AC5980E695
:10B5500091E061E00E9436E584E790E00E9418598E
:10B5600088E591E00E949159CE01019664E470E073
:10B5700044E050E00E942CE580E090E060E071E063
:10B580000E94DB5881E090E06CE171E00E94DB58A2
:10B5900080E491E00E943D598AE491E00E948D5937
:10B5A00086E591E060E00E9436E51FBF29960FB660
:10B5B000F894DEBF0FBECDBFDF91CF911F910895EC
:10B5C0008CE490E061E00E941BAE91E0813009F0D4
:10B5D00090E0892F0895CF93CFB7F89480E491E05D
:10B5E0000E943D598AE491E00E948D5988E591E0DE
:10B5F0000E94915980E691E061E00E9436E58EE676
:10B6000091E060E00E9436E581E00E94565A8CE4A9
:10B6100090E061E00E9436E5CFBFCF9108951F937F
:10B62000CF93DF93CDB7DEB72C970FB6F894DEBF7C
:10B630000FBECDBF1FB7F8948AE599E7A0E0B0E050
:10B6400089839A83AB83BC831D821E821F821886E6
:10B6500019861A861B861C86CE01019662E671E069
:10B660004CE050E00E942CE51FBF2C960FB6F894DA
:10B67000DEBF0FBECDBFDF91CF911F910895FF9226
:10B680000F931F93CF93DF93F82E162F80EA91E04C
:10B6900060E070E00E9439AEEC0182EA91E060E087
:10B6A0000E941BAE180F812F6CE30E940EE3092F3E
:10B6B0001D3308F021961FB7F894CF0DD11D80EAF5
:10B6C00091E0BE010E944CE582EA91E0602F0E9469
:10B6D00036E51FBFDF91CF911F910F91FF90089525
:10B6E000CF93CFB7F89482E090E067E10E9436E50F
:10B6F00082E490E061E00E9436E50E940F5B8CE4FA
:10B7000090E061E00E9436E580EA91E060E070E060
:10B710000E944CE582EA91E060E00E9436E584EA0E
:10B7200091E061E00E9436E5CFBF0E94635ACF915D
:10B7300008958CE199E064E477E140E00E94DEDE68
:10B740000895CF92DF92EF92FF920F931F93CF93C2
:10B75000DF93EC018B0188818823B1F16E01CE016A
:10B7600060E00E9429DE87FF2FC00E946F8188233E
:10B7700031F0CE010E947281C80161E80AC00E94C6
:10B780006C81882321F40E94B193882339F1C80188
:10B790006AE80E9489DE16C0C6016C2F0E9429DE6D
:10B7A0000E942D49219603C0C0E0D0E07901CE155A
:10B7B000DF0594F3C80161E802C0C80162E80E9495
:10B7C00089DE789481E001C080E0DF91CF911F9104
:10B7D0000F91FF90EF90DF90CF900895F894C8817B
:10B7E0000E9409492C2F30E082179307E8F6E5CF35
:10B7F00086E090E090933E0980933D0981E080933C
:10B80000220908950F931F93CF93DF93CDB7DEB72F
:10B8100064970FB6F894DEBF0FBECDBF8B01F894CE
:10B82000CE0101960E94227EC80161E80E9489DE55
:10B83000CE01019660E070E00E94CF7EFC01408165
:10B84000518162817381C8010E94A2DECE010196FE
:10B8500061E070E00E94CF7EFC01408151816281F5
:10B860007381C8010E94A2DECE01019662E070E001
:10B870000E94CF7EFC014081518162817381C801A9
:10B880000E94A2DE0E94C08C682FC8010E9489DE3F
:10B89000789464960FB6F894DEBF0FBECDBFDF91EB
:10B8A000CF911F910F9108950F931F93CF93DF9323
:10B8B000CDB7DEB764970FB6F894DEBF0FBECDBF2D
:10B8C0008B01F894CE0101960E94227EC80161E8A6
:10B8D0000E9489DECE01019660E070E00E94CF7E7A
:10B8E000FC014081518162817381C8010E94A2DE06
:10B8F000CE01019661E070E00E94CF7EFC014081A4
:10B90000518162817381C8010E94A2DECE0101963D
:10B9100062E070E00E94CF7EFC0140815181628133
:10B920007381C8010E94A2DECE01019663E070E03F
:10B930000E94CF7EFC014081518162817381C801E8
:10B940000E94A2DECE01019664E070E00E94CF7EEC
:10B95000FC014081518162817381C8010E94A2DE95
:10B960000E94C08C682FC80170E00E948CDE789421
:10B9700064960FB6F894DEBF0FBECDBFDF91CF91B6
:10B980001F910F9108958F929F92AF92BF92CF9285
:10B99000DF92EF92FF920F931F93CF93DF93CDB778
:10B9A000DEB78C017B018DB69EB6CEB6BDB6AEB607
:10B9B000CB0161E80E9489DEC80161E00E9429DEB6
:10B9C000882379F00E94DE82BC01009751F0C70104
:10B9D0000E9489DEC70160E00E9489DE8DBECEBE76
:10B9E00034C08DB79EB74F970FB6F8949EBF0FBE69
:10B9F0008DBFCDB6DEB60894C11CD11CC6016FE167
:10BA000040E050E00E947880BC01F60180818823EC
:10BA100029F06115710511F48E3281F3C7010E947E
:10BA200089DE10E0E12FF0E0C7011F3149F0EC0D95
:10BA3000FD1D6081662321F00E9489DE1F5FF2CF29
:10BA400060E00E9489DEBDBEAEBE0FB6F8949EBE19
:10BA50000FBE8DBEDF91CF911F910F91FF90EF90A0
:10BA6000DF90CF90BF90AF909F908F9008956F928E
:10BA70007F928F929F92AF92BF92CF92DF92EF927E
:10BA8000FF920F931F93CF93DF93CDB7DEB7A82E0E
:10BA9000E92E6B016DB67EB661E00E942EDE8C0150
:10BAA0008A2D9E2D63E00E9429DE482F882E99243E
:10BAB0008DB79EB7881999090FB6F8949EBF0FBE2F
:10BAC0008DBFADB6BEB60894A11CB11CEFB6F894FC
:10BAD000C501B80150E00E9416E5EFBEC60161E85D
:10BAE0000E9489DE750100E010E008C0F701619155
:10BAF0007F01C6010E9489DE0F5F1F4F08151905DF
:10BB0000ACF30FB6F8947EBE0FBE6DBEDF91CF9141
:10BB10001F910F91FF90EF90DF90CF90BF90AF906B
:10BB20009F908F907F906F9008952F923F925F9299
:10BB30006F927F928F929F92AF92BF92CF92DF923D
:10BB4000EF92FF920F931F93CF93DF9300D0CDB767
:10BB5000DEB7E82ED92E3B018DB79EB79A83898335
:10BB60008E2D9D2D61E00E942EDEC82EB92E8E2DC9
:10BB70009D2D63E00E9429DEF82E282E3324EDB798
:10BB8000FEB7E219F3090FB6F894FEBF0FBEEDBF82
:10BB90000DB71EB70F5F1F4F8FB6F894A02E512E12
:10BBA000C8016C2D7B2D4F2D50E00E9416E58FBEF5
:10BBB000480100E010E00BC0602F6C5F8E2D9D2DC2
:10BBC0000E9429DEF40181934F010F5F1F4F021580
:10BBD000130594F30FB7F8948A2D952D6C2D7B2DBA
:10BBE0004F2D50E00E942CE50FBFC30161E80E9479
:10BBF00089DEC3016F2D0E9489DE89819A810FB68B
:10BC0000F8949EBF0FBE8DBF0F900F90DF91CF9124
:10BC10001F910F91FF90EF90DF90CF90BF90AF906A
:10BC20009F908F907F906F905F903F902F9008959E
:10BC30000F931F93CF93DF9380915E09882379F44C
:10BC40000EE519E0C2E2D0E0CE0160E00E941BAE3A
:10BC5000F80181938F012196C233D105A9F7809114
:10BC60005E09882369F4AEE5B9E080E090E0FC016C
:10BC7000E658FC4FE491ED9301968E309105B9F7AB
:10BC80008EE599E0DF91CF911F910F9108958FE399
:10BC900099E0089580913D0990913E090895CF93D0
:10BCA000DF938FE399E00E946D82EC01009789F4A5
:10BCB0000E945B490E94E0850E94107C89EB99E01C
:10BCC00060E00E94A06C82E090E090933E09809337
:10BCD0003D09CE01DF91CF9108950E9403948823FE
:10BCE000A9F085E090E090933E0980933D0989EAB0
:10BCF0009BE00E94BFB489EB99E064E070E041E012
:10BD00000E94AC660E945B490E94107C0895CF930C
:10BD1000C82F0E941D49C817D1F08C2F0E941649C8
:10BD2000CC2351F083E090E090933C0980933B0951
:10BD300085E299E061E009C081E090E090933C09E0
:10BD400080933B0985E299E060E00E9495E1CF9104
:10BD500008951F93CF93DF93182FEB010E94204982
:10BD60001817D9F0812FBE010E94D04B112351F03A
:10BD700085E090E090933C0980933B0985E299E04F
:10BD800061E009C081E090E090933C0980933B0919
:10BD900085E299E060E00E9495E1DF91CF911F91EB
:10BDA000089585E299E040E054EA63E976ED0E9467
:10BDB0003FE1109234090895DF92EF92FF920F93C2
:10BDC0001F93CF93DF93CDB7DEB76F970FB6F8947D
:10BDD000DEBF0FBECDBFFC0180913D0990913E09B1
:10BDE0008130910509F44EC08230910524F400970A
:10BDF00009F442C076C08230910529F08530910562
:10BE000009F06FC03FC07E010894E11CF11C4FE1B6
:10BE1000DD24D39482819381009719F4D18680E048
:10BE20001AC08481958120813181B9010E941AE371
:10BE300006811781080F191F848195810196B90128
:10BE40000E941AE39583848382819381019793836F
:10BE50008283D8018C91D7018D937D01882309F4C9
:10BE600058C04150B9F655C08FE399E0BE016F5FED
:10BE70007F4F0E944BE435C081E090E090933E09F3
:10BE800080933D098FE3E82E89E0F82E4FE1DD2411
:10BE9000D39482819381009719F4D18680E01AC0EF
:10BEA0008481958120813181B9010E941AE3068144
:10BEB0001781080F191F848195810196B9010E948D
:10BEC0001AE395838483828193810197938382838C
:10BED000D8018C91D7018D937D01882311F04150B9
:10BEE000C1F60E94D15E0E94994981E090E0909352
:10BEF0003C0980933B096F960FB6F894DEBF0FBEE6
:10BF0000CDBFDF91CF911F910F91FF90EF90DF9008
:10BF10000895CE01019668E272E00E9442E4009723
:10BF200001F3A2CF85E299E00E9465E1882369F0E0
:10BF300085E299E040E054EA63E976ED0E943FE152
:10BF4000809134098F5F809334090895CF93DF93F4
:10BF5000FC01EB0180912509882339F480913A098D
:10BF600080838091390988830EC080913409808351
:10BF700085E299E00E94C4E120E037E843E953E01C
:10BF80000E9441E32883DF91CF910895CF93DF93FF
:10BF9000CDB7DEB72F970FB6F894DEBF0FBECDBF7B
:10BFA0008AE399E069E379E00E94A65F80913A090B
:10BFB000609139090E943F5BCE0101960E943BE1EE
:10BFC000A5E2B9E0FE0131968FE001900D9281501B
:10BFD000E1F7109234092F960FB6F894DEBF0FBE2A
:10BFE000CDBFDF91CF910895CF93DF9300D000D0E4
:10BFF00000D0CDB7DEB789EA9BE061E070E00E9437
:10C0000028B50E94C65F0E949049DC01CB01809355
:10C01000350990933609A0933709B093380982E027
:10C0200090E090933C0980933B0910923E09109256
:10C030003D09CE01019666E477E145E00E94DEDE2F
:10C04000E981FA8182819E818923828326960FB6B7
:10C05000F894DEBF0FBECDBFDF91CF9108951F933F
:10C06000CF93DF93CDB7DEB76A970FB6F894DEBFF4
:10C070000FBECDBF80913D0990913E09019782305E
:10C08000910508F067C00E94107C0E949049DC0175
:10C09000CB018093350990933609A0933709B0936B
:10C0A00038090E94C65F84E090E090933C09809339
:10C0B0003B0981E062E070E00E94D04BCE01029625
:10C0C000BE016F5F7F4F0E94A65F0E94EE92182F05
:10C0D000882309F43FC0CE0107960E94227ECE013C
:10C0E000079662E070E0113039F40E94D77E40E993
:10C0F00052EE60E070E006C00E94D77E40E65AEE45
:10C1000060E070E0FC01408351836283738380E0D0
:10C110000E94164986E990E0A0E0B0E08B839C8302
:10C12000AD83BE83CE010796BE016D5F7F4F0E9437
:10C13000D87989EA9BE069E873E00E943BB581E029
:10C140008093960C8EE699E040E45BE46CE470E04A
:10C150000E943FE180913D0990913E098130910517
:10C1600089F484E090E090933E0980933D0981E05A
:10C17000809322098DE799E040E452E46FE070E09B
:10C180000E943FE189EB99E064E070E040E00E94AA
:10C19000AC6681E08093240984E090E090933C09B0
:10C1A00080933B096A960FB6F894DEBF0FBECDBFF1
:10C1B000DF91CF911F9108950F931F93CF93DF933A
:10C1C00000D0CDB7DEB78C0161E80E9489DECE01D8
:10C1D0000296BE016F5F7F4F0E94A65FC80160910B
:10C1E0003B090E9489DEC8016A810E9489DEC8017C
:10C1F00069810E9489DE80913B0990913C098130E0
:10C20000910531F08330910519F08530910529F4BD
:10C210000E949049AB01BC0108C040913509509182
:10C2200036096091370970913809C8010E94A2DE71
:10C23000C80140E050E060E070E00E94A2DE0F9094
:10C240000F90DF91CF911F910F910895EF92FF9280
:10C250000F931F93CF93DF937C018B01FC018081AF
:10C26000882309F4F7C0C70161E00E9429DEC82FC6
:10C27000C70162E00E9429DE803209F44AC081329F
:10C2800068F4823019F1833018F48823B9F0E2C0E1
:10C29000863149F18E3109F0DDC032C0833209F4B4
:10C2A0004EC0843220F4813209F0D4C03FC08432C1
:10C2B00009F44FC0853209F0CDC084C0C80161E8DF
:10C2C0000E9489DEC8016AE572E0C0C0C80161E869
:10C2D0000E9489DEC13019F48EE89AE002C080EE37
:10C2E00099E0499613C0C80161E80E9489DEC13017
:10C2F00019F48EE89AE002C080EE99E0499625C0D4
:10C30000C80161E80E9489DE85EB9CE00E94A2B131
:10C310009BC0C80161E80E9489DEC13019F48EE833
:10C320009AE002C080EE99E0499606C0C80161E833
:10C330000E9489DE85EB9CE00E949CB185C0C8010B
:10C3400061E80E9489DE85EB9CE00E9478B1682F4D
:10C3500035C0C80161E80E9489DEC13019F48EE859
:10C360009AE002C080EE99E049960E94A5B3882326
:10C3700011F0D0E801C0D0E085EB9CE00E94A5B3AD
:10C38000882311F080E401C080E0D82BC13019F47B
:10C390008EE89AE002C080EE99E049960E94AAB326
:10C3A000D82BC13019F42EE83AE002C020EE39E073
:10C3B000C90149960E9478B16D2F682BC8010E946F
:10C3C00089DE46C0C80161E80E9489DEC13019F4E7
:10C3D0008EE89AE002C080EE99E049960E94A6B1EC
:10C3E000BC01C8010E948CDEC13019F48EE89AE0CD
:10C3F00002C080EE99E049960E94AAB1BC01C80132
:10C400000E948CDEC13019F48EE89AE002C080EE02
:10C4100099E049960E94AEB1BC01C8010E948CDE31
:10C4200085EB9CE00E94A6B1BC01C8010E948CDE95
:10C4300085EB9CE00E94AAB1BC01C8010E948CDE81
:10C4400085EB9CE00E94AEB1BC01C8010E948CDE6D
:10C4500081E001C080E0DF91CF911F910F91FF90AB
:10C46000EF900895AF92BF92CF92DF92EF92FF923A
:10C470000F931F93CF93DF93EC018B018881882367
:10C4800009F422C1FC2EED2ECE0160E00E9429DECF
:10C4900087FD1AC1E82FF0E0EC31F10508F014C176
:10C4A000EE58FF4FEE0FFF1F0590F491E02D099419
:10C4B0008C2F9D2F61E00E942EDE8A31910528F499
:10C4C000C80161E80E9489DEF9C0C80161E80E94E4
:10C4D00089DEC8016AE572E0F4C0C80161E80E9423
:10C4E00089DE4FE3E42E49E0F42ECC24E701C801B5
:10C4F000F70161917F010E9489DE8881882309F418
:10C50000E5C0C394FFE1CF1689F7E0C080913D09F3
:10C5100090913E099C01215030402230310518F0A5
:10C520008530910549F40E942F6089EB99E064E021
:10C5300070E00E94226960C081E0809324095CC0A1
:10C54000C80161E80E9489DE0E940949AC0160E0EF
:10C5500070E0C8010E94A2DEB9C0CE01B8010E94FD
:10C56000025CB4C0CE01B8010E94545CAFC0C801E7
:10C5700061E80E9489DECE0103960E949F822EC050
:10C58000C80161E80E9489DE0E949A81AB01BC016A
:10C59000C8010E94A2DE0E94FC8198C0C80161E827
:10C5A0000E9489DE2FE3A22E29E0B22E31E0C32EB5
:10C5B000D12C0BC08F2D9E2D6C2D0E9429DEF501F4
:10C5C00081935F010894C11CD11C888190E0C8163A
:10C5D000D90684F310925D090E944F5E682FC8014E
:10C5E0004EC0CE01B8010E94C35C70C00E941D49BC
:10C5F00091E089270E94875EC80161E840C0CE01B2
:10C60000B8010E94266163C0C80161E80E9489DE0A
:10C61000F8940E94C484882321F40E94234988232B
:10C6200011F460E001C061E0C8010E9489DE7894E5
:10C630004DC0CE01B8010E94375D48C0CE01B8019F
:10C640000E94955D43C08C2F9D2F61E00E9429DEE2
:10C65000C82F80FF02C00E94107CC1FF02C00E9450
:10C660005B49C80161E80E9489DEC80160E007C03B
:10C67000C80161E80E9489DEC8016091330D0E9403
:10C6800089DE24C0C8010E94DC6020C08C2F9D2F51
:10C6900061E00E942EDEC80161E80E9489DEC801C7
:10C6A0006AE572E00E948CDEC80160E070E00E94E2
:10C6B0008CDEC80160E070E00E948CDEC80160E0A2
:10C6C00070E00E948CDE02C080E001C081E0DF915A
:10C6D000CF911F910F91FF90EF90DF90CF90BF907F
:10C6E000AF9008958091321A9091331A009709F40F
:10C6F000EFC08091321A9091331A8430910509F07D
:10C70000F4C0E6C080912209882339F08DE799E0D2
:10C710000E9465E1882309F4E0C080916E098823B6
:10C7200059F08EE699E00E9465E1882329F40E9481
:10C73000C484882309F0D1C080913B0990913C09C1
:10C740008130910531F08330910519F085309105E4
:10C7500011F40E942F6080E062E070E00E94D04BF4
:10C7600010922409809123090E948E64109223095B
:10C770008CE899E00E948FE110925E0910923F09C7
:10C7800010923E0910923D09089580910C1A9091E3
:10C790000D1A84309105D1F080918C09882349F4D9
:10C7A0008CE899E040E45DE063E070E00E943FE1E6
:10C7B0000DC08CE899E00E9465E1882339F089EE8C
:10C7C00099E10E94C6DD84E080930B1A80910B1AD8
:10C7D000882321F089EE99E10E94D4DD80910C1A22
:10C7E00090910D1A8430910509F04AC08CE899E0C7
:10C7F0000E948FE18FE09AE10E9449DE80913D091D
:10C8000090913E09209122098630910561F48FE0D4
:10C810009AE1222331F069E80E9489DE1092220910
:10C8200027C06BE823C0222371F08FE09AE169E80A
:10C830000E9489DE1092220989EB99E066E070E09F
:10C840000E94226915C089EE99E16FE07AE10E94A9
:10C85000A15B882369F489EE99E16FE07AE10E9497
:10C860003262882329F48FE09AE165E80E9489DE2C
:10C8700089EE99E10E94D4DD85EE99E10E941DE2E6
:10C8800080913D0990913E098230910541F40E94CA
:10C890006C81882321F410923E0910923D09809109
:10C8A0003D0990913E098530910579F40E94B1933C
:10C8B000882321F410923E0910923D0989EB99E0FA
:10C8C00064E070E040E00E94AC660E94925F0895D0
:10C8D00080912409882309F015CF80910C1A90913A
:10C8E0000D1A009709F051CF71CF08958BE999E0A7
:10C8F00064E477E140E00E94DEDE8CE899E00E948B
:10C900003BE18DE799E00E943BE18EE699E00E94D1
:10C910003BE185E299E00E943BE10895CF93DF93EC
:10C920000F92CDB7DEB7682FF89484B76623A1F0D5
:10C9300088E10FB6F89480936000109260000FBEFB
:10C9400014BE89E228E130E00FB6F894A895209350
:10C9500060000FBE8093600069830E94FC810E948A
:10C96000246E0E94B4930E94847C0E94107C0E94DA
:10C970005B490E948DAE0E94E0850E940AE089EB2F
:10C9800099E069810E94A06C78940F90DF91CF911B
:10C99000089581E00E948E640E94E58578940E944B
:10C9A00072630E948C4F89EB99E00E94AC690E94EF
:10C9B000616FA895F4CF81EA99E064E477E140E003
:10C9C0000E94DEDE0895FC01A081B18112968C9157
:10C9D0001297662319F09481892B02C095818923CF
:10C9E00012968C93129708950F931F93CF93DF9312
:10C9F00000D000D000D0CDB7DEB7062F1FB7F89417
:10CA0000CE01019666E477E144E00E94DEDE61E05B
:10CA1000002309F460E0CE0101960E94E3641FBF89
:10CA200026960FB6F894DEBF0FBECDBFDF91CF9133
:10CA30001F910F910895AF92BF92CF92EF92FF9204
:10CA40000F931F93CF93DF93CDB7DEB7C254D0407F
:10CA50000FB6F894DEBF0FBECDBF5C0104960E94F6
:10CA60003BE1C50143960E943BE1CE01CD966CE4CB
:10CA700077E143E00E94DEDECE01C7966CE477E109
:10CA800044E00E94DEDECE01C19662E577E143E03C
:10CA90000E94DEDEC501879660E0AE01435C5F4F19
:10CAA0009E01295C3F4F8E010F5C1F4FE12CE1E09E
:10CAB000FE2E0E94A196CE018B9668E577E145E0B7
:10CAC0000E94DEDECE01859668E577E146E00E94B1
:10CAD000DEDECE014F9662E577E144E00E94DEDEC5
:10CAE000C5018B529F4F61E0AE01455D5F4F9E01D6
:10CAF0002B5D3F4F8E01015E1F4FFCE1EF2EF1E0F9
:10CB0000FF2E0E94A196C5018D579E4F0E943BE1CA
:10CB1000C5018E569E4F0E943BE185010F551E4F69
:10CB2000C80102960E943BE1C80141960E943BE188
:10CB3000C80180960E943BE1A4EDEA2EA1E0FA2E06
:10CB4000EA0CFB1CCE01499666E577E144E00E94C1
:10CB5000DEDECE01439666E577E143E00E94DEDE4D
:10CB6000CE010D9666E577E142E00E94DEDEC70168
:10CB7000BE01675E7F4FAE014D5E5F4F9E01235F3A
:10CB80003F4F0E9437B8CE01079666E577E145E052
:10CB90000E94DEDECE01019666E577E146E00E9466
:10CBA000DEDEC50180519E4FB801A7019E01295FBD
:10CBB0003F4F8E010F5F1F4F0E9420B4C50181526D
:10CBC0009D4F0E9434D1F501EE51FD4F8EED93E063
:10CBD00091838083850108511D4FC8016FE040E0BB
:10CBE0000E9465E0A50146505D4F88E893E0FA0198
:10CBF00091838083C50184509D4FB80100E513ECFB
:10CC000020E030E0B0E1EB2EB1E0FB2ECC240E941E
:10CC10007FB08CE490E061E00E941BAEF501EC581F
:10CC2000FC4F91E0882309F490E09083CE5BDF4FC6
:10CC30000FB6F894DEBF0FBECDBFDF91CF911F912D
:10CC40000F91FF90EF90CF90BF90AF9008950E940A
:10CC50005D6E1092200189E08093210110922201E3
:10CC600080E090E1909329018093280182E08093F5
:10CC700073001092B0009AE09093B1001092B3004C
:10CC80001092B4008093700091E0909380008BE04C
:10CC900080938100109289001092880010928B007E
:10CCA00010928A0010926F009093A0008093A100D0
:10CCB0001092A9001092A8001092AB001092AA0046
:10CCC0001092720008950F931F934FB7F894FC01D0
:10CCD00000811181228133814FBFB801C9011F91A9
:10CCE0000F9108950E941D49882311F40E94E18C40
:10CCF0000895CF93DF93EC01FC01E858FC4F71835A
:10CD0000608362307105E1F484509D4F0E94A5B3A9
:10CD10008823D9F40E940E5A8823B9F0CE01805C92
:10CD20009F4F0E94A5B38823A1F0CE0182519F4F4F
:10CD30000E94A5B3882369F008C081E08093B809F8
:10CD4000CB58DC4F81E0888304C08091B8098823E8
:10CD5000A1F3DF91CF910895FC01E658FC4F4423E5
:10CD600021F08081862B80830895609580816823DF
:10CD700060830895CF93DF93EC01805C9F4F0E9406
:10CD8000B2B1882369F4CE0182519F4F0E94B2B1A3
:10CD9000882331F4CE0184509D4F0E94B2B101C06E
:10CDA00081E0DF91CF910895FC01EF57FC4F31E016
:10CDB0003083FC01EE57FC4F6083FC01ED57FC4FC4
:10CDC0004083FC01EC57FC4F20838B579C4FFC01A8
:10CDD00010820895DF92EF92FF920F931F93CF93EB
:10CDE000DF938C01FC01EF57FC4F1082C4EDEC2E59
:10CDF000C1E0FC2EE80EF91EEC01CD57DC4FFC0122
:10CE0000EE57FC4FC701688140810E94BBBAD880B1
:10CE1000E801CC57DC4F06C0C70163E372E00E9413
:10CE2000ACB9D3948881D816B8F3DF91CF911F9114
:10CE30000F91FF90EF90DF9008958F929F92AF92A5
:10CE4000BF92CF92DF92FF920F931F93CF93DF9306
:10CE50004C01A62E142FC22E241708F476C0422FA0
:10CE600050E0411B5109802F90E0481759070CF4FE
:10CE70006CC0F401E258FC4F6081718116161706F0
:10CE8000D4F4F401E458FC4F808191819B01281B6C
:10CE9000390BC90137FF03C0909581959F4F849F3F
:10CEA0009001859F300D949F300D1124C9010E947F
:10CEB0002EE3F62E01C0FF24F01698F4E401CC52C4
:10CEC000DE4FCE01612F4A2D0E94BBBA012F06C052
:10CED000CE0163E372E00E94ACB90F5F0C15C1F79D
:10CEE00000E0D4EDCD2ED1E0DD2EC80CD91C602F92
:10CEF000610FC6014A2D0E94BBBAAA24BB24C02FD1
:10CF0000D0E00F2D10E007C0C6016FEF0E94FCBA01
:10CF10000894A11CB11CC5018C0F9D1F801791079F
:10CF20009CF3F401E058FC4F808191E089278083D5
:10CF3000882331F0C6016AEA73E00E94C3B906C0D3
:10CF4000C6016FEF0E94FCBA01C0FF248F2DDF9154
:10CF5000CF911F910F91FF90DF90CF90BF90AF9036
:10CF60009F908F9008958F929F92AF92BF92CF9291
:10CF7000DF92EF92FF920F931F93CF93DF937C0189
:10CF80005EE7A52E53E0B52EA80EB91EF50111825D
:10CF90001082EC01C458DC4F198218820E94BA66D4
:10CFA000882309F4ECC04CEFC42E42E0D42ECE0C02
:10CFB000DF1CC6010E94B2B18823C9F00881198123
:10CFC000C6010E94E8B1880F991F800F911F9983B5
:10CFD0008883F501C081D181C6010E949CB1880F70
:10CFE000991F8C0F9D1FF5019183808318C0F70155
:10CFF000EA54FF4F8081882331F0C701805C9F4F46
:10D0000060E00E94FEB1F701EC59FE4F8081882359
:10D0100031F0C70182519F4F60E00E94FEB100E4F1
:10D02000C02ED12CCE0CDF1CC6010E94B2B18823C9
:10D0300011F1F701EA54FF4F80818823E1F4870161
:10D0400004581C4FF801C081D181C6010E94E8B18B
:10D05000C80FD91FF801D183C083870102581C4F24
:10D06000F801C081D181C6010E949CB1C80FD91FAF
:10D07000F801D183C0831EEEC12ED12CCE0CDF1C53
:10D08000C6010E94B2B1882311F1F701EC59FE4F9D
:10D0900080818823E1F4870104581C4FF801C08186
:10D0A000D181C6010E94E8B1C80FD91FF801D18310
:10D0B000C083870102581C4FF801C081D181C6018D
:10D0C0000E949CB1C80FD91FF801D183C083F7011A
:10D0D000E258FC4F80819181009709F459C082E4A5
:10D0E00091E061E00E941BAE882309F451C080E406
:10D0F00091E067E00E941BAE873009F449C0E70168
:10D10000C558DC4F8881882321F40E94889881E0EB
:10D110008883F701E258FC4F60817181F701E45880
:10D12000FC4F008111814B01AA2497FCA094BA2CDA
:10D13000601B710B882777FD8095982F2FEF30E0CB
:10D1400040E050E00E94EFE2A50194010E9463E3F9
:10D15000C22FB801882777FD8095982F2FEF30E0F8
:10D1600040E050E00E94EFE2A50194010E9463E3D9
:10D170008C2F60E0422F20E00E949B9809C0E701BD
:10D18000C558DC4F8881882319F00E94889918823D
:10D19000F701EF57FC4F80818823A9F0F701EE5784
:10D1A000FC4FD701AD57BC4F97012C573C4FE701BF
:10D1B000CB57DC4FC70160814C91F9012081088178
:10D1C0000E941D678883DF91CF911F910F91FF907F
:10D1D000EF90DF90CF90BF90AF909F908F90089589
:10D1E000439640E052ED69E47BE60E943FE10895FA
:10D1F0001F920F920FB60F920BB60F9211242F931E
:10D200003F934F935F936F937F938F939F93AF93CE
:10D21000BF93EF93FF9389EB99E00E947266FF91B1
:10D22000EF91BF91AF919F918F917F916F915F919E
:10D230004F913F912F910F900BBE0F900FBE0F900B
:10D240001F9018950F931F93CF93DF9300D000D0BA
:10D2500000D0CDB7DEB78B016115710589F410924E
:10D26000B2091092B109CE01019668E577E147E075
:10D270000E94DEDECE01019660E00E94E3640CC0F5
:10D280008091B50990E08617970731F082E090E031
:10D290009093B2098093B1090093B50926960FB611
:10D2A000F894DEBF0FBECDBFDF91CF911F910F91DC
:10D2B00008954115510531F41092B0091092AF094B
:10D2C00081E008C06115710541F41092B009109217
:10D2D000AF0980E00E9404B408956093B4094093BC
:10D2E000B30981E090E09093B0098093AF0908956D
:10D2F000CF93DF93EC0169E170E04FE050E00E94D2
:10D300005969CE0180519E4F6FEF0E94F4B7CA5801
:10D31000DC4F81E08883DF91CF9108950F931F93B5
:10D32000CF93DF930F92CDB7DEB78C0180519E4F24
:10D3300049830E943BB5C8010E94786980E00E9441
:10D34000726FF801E958FC4F498140830F90DF91DB
:10D35000CF911F910F910895DF92EF92FF920F935B
:10D360001F93CF93DF938C01FC0186A18823F1F0FA
:10D37000E801C051DE4FCE010E94A0B474E0E72E58
:10D38000F12CE00EF11EC7010E9465E1882371F0C7
:10D39000CE010E945DB6CE010E94A6B4AB01BC01D5
:10D3A000C7010E943FE1DD24D39401C0DD24F801D0
:10D3B000EC58FC4F80818823A1F0E801CE56DE4F67
:10D3C000CE010E9465E1882361F0C80184509D4F21
:10D3D0000E9488B2CE0140E553EC60E070E00E940C
:10D3E0003FE166E7E62E63E0F62EE00EF11EF70160
:10D3F0008081882301F1E801C051DE4FCE010E94F7
:10D40000F9B78823C1F0C80160E070E040E050E067
:10D410000E9459690E948899F7011082CE010E94EA
:10D4200009B6F801E958FC4F8081882311F00E9469
:10D430002F601092B609E8016396CE010E9465E163
:10D44000882309F459C0F801EB58FC4F80818823E8
:10D4500009F052C00E944A5E8230910509F44CC026
:10D460000E944A5E8130910509F446C0CE010E94B7
:10D4700092E1F801E658FC4F808180648E7F8083C2
:10D48000E801C05CDF4FCE010E949CB1181619065E
:10D4900084F0C80182519F4F0E949CB11816190652
:10D4A00044F0C80184509D4F0E949CB11816190683
:10D4B00084F4C80180519E4F6CEA73E00E943BB532
:10D4C000C8010E94786980E060E04FEF21E00E948F
:10D4D0009B98CE0160E070E00E94CBB0C801825101
:10D4E0009F4F60E070E00E94CBB0C80184509D4F18
:10D4F00060E070E00E94CBB0E801CB58DC4F88813F
:10D50000882309F4A5C08091B609882309F0A0C03A
:10D510000E945E6F882309F09BC081E08093B6096A
:10D52000C8016AE070E04AE050E00E945969F801E1
:10D53000E858FC4F8081918188309105C9F089308D
:10D54000910544F48230910549F18430910509F048
:10D5500057C008C08031910599F08032910509F0DB
:10D560004FC014C0C80180519E4F65ED73E005C0E7
:10D57000C80180519E4F65E274E00E943BB540C0F7
:10D58000C80180519E4F66E774E0F7CFC80167EC91
:10D5900074E040E00E948E69188282C0C80168E190
:10D5A00075E040E00E948E69E801C05CDF4FCE016B
:10D5B0000E94A5B3882329F0CE0160E070E00E94AC
:10D5C000CBB0E801C251DF4FCE010E94A5B3882342
:10D5D00029F0CE0160E070E00E94CBB0E801C450B9
:10D5E000DD4FCE010E94A5B3882329F0CE0160E073
:10D5F00070E00E94CBB0F801EB58FC4F108250C095
:10D60000C801805C9F4F60E070E00E94CBB0C80111
:10D6100082519F4F60E070E00E94CBB0C8018450FF
:10D620009D4F60E070E00E94CBB080E00E94726F7E
:10D630000E948E980E94F85B0E9419490E94107CFB
:10D64000C0E08C2F60E00E94568CCF5FC530C9F7D8
:10D65000E801CD57DE4FCE010E9465E18823E1F05D
:10D66000DD20D1F4C80187960E944997C8010E9425
:10D67000B367CE0140E251EA67E070E00E943FE10B
:10D6800081E08093B7090CC0C8018B529F4F0E9464
:10D6900049971092B70904C08091B7098823A1F770
:10D6A000DF91CF911F910F91FF90EF90DF90089540
:10D6B0001F920F920FB60F920BB60F9211242F9359
:10D6C0003F934F935F936F937F938F939F93AF930A
:10D6D000BF93EF93FF93CF93DF93CDB7DEB76297FE
:10D6E000DEBFCDBF8091B9099091BA09A091BB0965
:10D6F000B091BC0980589F4FAF4FBF4F8093B9097D
:10D700009093BA09A093BB09B093BC098091A70973
:10D710009091A8099C012F5F3F4F3093A809209357
:10D72000A7098138910508F4B7C01092A809109292
:10D73000A7098091AD099091AE091816190614F445
:10D7400001973CC08091B1099091B2098130910557
:10D7500001F58091AB099091AC0901969093AC09C9
:10D760008093AB0982E090E09093B2098093B10975
:10D7700082E190E09093AE098093AD09CE010D96C1
:10D7800068E577E147E00E94DEDECE010D9660E0BD
:10D790004DC08230910569F58091B50990E02091E6
:10D7A000AB093091AC09281739076CF083E090E0A1
:10D7B0009093B2098093B10980E590E09093AE090F
:10D7C0008093AD0935C081E090E09093B2098093D9
:10D7D000B10982E190E09093AE098093AD09CE014A
:10D7E000079668E577E147E00E94DEDECE01079606
:10D7F0001CC083309105E1F41092AC091092AB0982
:10D8000081E090E09093B2098093B10982E190E0C9
:10D810009093AE098093AD09CE01019668E577E15A
:10D8200047E00E94DEDECE01019661E00E94E364E3
:10D830008091A9099091AA091816190634F4019744
:10D840009093AA098093A90927C08091AF0990916C
:10D85000B0098130910571F482E090E09093B009B5
:10D860008093AF098091B4098093A9091092AA0905
:10D8700081E010C08230910579F481E090E09093CE
:10D88000B0098093AF098091B3098093A9091092E0
:10D89000AA0980E00E9404B46296DEBFCDBFDF918A
:10D8A000CF91FF91EF91BF91AF919F918F917F9118
:10D8B0006F915F914F913F912F910F900BBE0F9001
:10D8C0000FBE0F901F901895FC01EC58FC4F608321
:10D8D0000895EF92FF920F931F93CF93DF93CDB7ED
:10D8E000DEB72C970FB6F894DEBF0FBECDBFE62E85
:10D8F000FFB6F89406E417E1CE010796B80145E0BB
:10D900000E94DEDECE01079661E00E9413DFCE01A9
:10D910000196B80145E00E94DEDECE0101966E2D33
:10D920000E94E364FFBE2C960FB6F894DEBF0FBED4
:10D93000CDBFDF91CF911F910F91FF90EF90089590
:10D94000AF92BF92CF92DF92EF92FF920F931F930D
:10D95000CF93DF93CDB7DEB7E0970FB6F894DEBF75
:10D960000FBECDBF7C01C62E60E070E00E94226930
:10D9700082E090E060E00E941BAE082F8CE291E113
:10D980000E947F83802F8095881F8827881F0E9490
:10D99000E88685EE99E161E00E943FE289EE99E137
:10D9A0000E94D4DDF7011082118212821382C70116
:10D9B0000E9427660E94B7B3F70186A3882389F1E6
:10D9C000870100511E4FC8010E947BB586E591E09A
:10D9D00060E00E941BAEB701882319F46E517D4FA1
:10D9E00002C061527D4FC8010E94C8B4CC2051F0E2
:10D9F00020E335E740E951E0CA010197F1F72150F2
:10DA00003040D1F7B7016C527E4FC8010E94ECB391
:10DA1000C8010E94A6B4AB01BC01C70104960E94D4
:10DA20003FE1C70160E070E040E050E00E945969CA
:10DA3000CC2009F466C0CE018B9668E577E147E01B
:10DA40000E94DEDECE018B9661E00E9413DFCE01E4
:10DA5000859666E577E141E00E94DEDECE0185969F
:10DA600061E00E9413DFCE014F9666E577E140E06A
:10DA70000E94DEDECE014F9661E00E9413DFCE01F0
:10DA800049966EE477E141E00E94DEDECE014996E0
:10DA900061E00E9413DFCE01439668E577E147E03D
:10DAA0000E94DEDECE01439661E00E9413DFCE01CC
:10DAB0000D966EE477E140E00E94DEDECE010D9629
:10DAC00061E00E9413DFCE01079668E477E146E04B
:10DAD0000E94DEDECE01079661E00E9413DF0E9405
:10DAE0001F9A83E00E94726FF701EB58FC4F10827F
:10DAF000F701E858FC4F11821082C70182960E94FC
:10DB00004296F701E658FC4F1082C7018D579E4F91
:10DB100040E251EA67E070E00E943FE1C70160E047
:10DB20000E94696C8701095D1F4FC8010E942897F8
:10DB3000A5EDAA2EB12CAE0CBF1CC5010E942897E2
:10DB4000CE01019666E477E144E00E94DEDECE017C
:10DB5000019661E00E9413DFC70188519D4F0E942A
:10DB60005EE0BCEFCB2EB2E0DB2ECE0CDF1CC6019C
:10DB70000E948AAFC801499660E070E00E94CBB075
:10DB80008501075E1F4FC80160E070E00E94CBB0C6
:10DB9000C60160E070E00E94CBB0C7018E569E4F78
:10DBA00040E553EC60E070E00E943FE10E940E5AB5
:10DBB000682FC8010E94BFB00E94E05A61E0682748
:10DBC000C6010E94BFB00E948899F701EA58FC4F35
:10DBD0001082F701E458FC4F11821082F701E258DD
:10DBE000FC4F11821082F701E558FC4F1082F701BB
:10DBF000EF57FC4F1082F701EE57FC4F1082F701F0
:10DC0000ED57FC4F1082F701EC57FC4F1082E09665
:10DC10000FB6F894DEBF0FBECDBFDF91CF911F913D
:10DC20000F91FF90EF90DF90CF90BF90AF9008954D
:10DC30008FE39DE064E477E140E00E94DEDE89EB63
:10DC400099E00E941B650895CF93DF9300D000D028
:10DC500000D0CDB7DEB78AE491E061E00E941BAE50
:10DC600091E0882309F490E09093EF0D1092480D15
:10DC70001092470D10924A0D1092490D10924D0DC1
:10DC800010924E0D80EF9DE00E9492E11092FF0DE8
:10DC9000CE0101966EE477E145E00E94DEDECE0122
:10DCA000019661E00E9413DF26960FB6F894DEBF5E
:10DCB0000FBECDBFDF91CF91089514BC15BC17BC2A
:10DCC00018BC16BC10926E000895CF92DF92EF92AE
:10DCD000FF92CF938091470D9091480D009739F4B2
:10DCE00080EF9DE00E9492E11092FF0D4FC021E075
:10DCF0002093FF0D8091470D9091480D009731F4CE
:10DD000020934E0DCC24DD2476012EC08091490D48
:10DD100090914A0D2091450D3091460DB9010E9418
:10DD20001AE3880F991F880F991FE0914B0DF0910E
:10DD30004C0DE80FF91F8091490D90914A0D019605
:10DD4000B9010E941AE390934A0D8093490D809186
:10DD5000470D9091480D01979093480D8093470D82
:10DD6000C080D180E280F380B70180E090E028EEAF
:10DD700033E040E050E00E94EFE2AB01BC0180EFF5
:10DD80009DE00E943FE1C601009719F40E945D6E7C
:10DD90003EC0A0E0B0E082342FE0920720E0A2076E
:10DDA00020E0B20780F4883E21E0920720E0A2073D
:10DDB00020E0B20758F48A379105A105B10548F073
:10DDC000C4E068E008C0C2E063E005C0C3E066E00C
:10DDD00002C0C5E06AE09C01AD01220F331F441F61
:10DDE000551F04C0220F331F441F551F6A95D2F7D9
:10DDF00060E074E284EF90E00E9441E3215082E110
:10DE000084BDC5BD27BD18BC16BC10926E00CF9155
:10DE1000FF90EF90DF90CF900895CF93482FE92F98
:10DE2000F62FC72F8091EF0D882309F445C060912C
:10DE3000450D7091460D8091470D9091480D6817E2
:10DE40007907A1F18091470D9091480D86179707AA
:10DE500050F52091470D3091480D8091490D9091DA
:10DE60004A0D820F931F0E941AE3880F991F880F93
:10DE7000991FA0914B0DB0914C0DA80FB91F4C9359
:10DE80001196EC9311971296FC9312971396CC93DC
:10DE900013978091470D9091480D01969093480DEE
:10DEA0008093470D03C081E080934D0D8091FF0D5D
:10DEB000882311F40E94656ECF9108958091FF0D23
:10DEC00008958091EF0D882361F08091FF0D8823E4
:10DED00041F080EF9DE00E9465E1882311F00E94EF
:10DEE000656E0895EF92FF921F93CF93DF93883072
:10DEF00038F5E82FF0E0EE0FFF1FE657FC4FE0800B
:10DF0000F180E114F104E1F010E0812F90E0880F3E
:10DF1000991F880F991FF701E80FF91F2591349178
:10DF200002968E0D9F1DFC01C591D491209721F082
:10DF3000C901BE010E940D6F1F5F209731F706C017
:10DF40008BE790E064EF71E00E940D6FDF91CF915D
:10DF50001F91FF90EF90089580E09EE064E477E1E8
:10DF600040E00E94DEDE88E290E09093460D8093D0
:10DF7000450D1092480D1092470D10924A0D1092C7
:10DF8000490D8FE49DE090934C0D80934B0D1092C2
:10DF90004D0D10924E0D80EF9DE00E943BE10895E3
:10DFA00080936B030895CF92DF92EF92FF926B0103
:10DFB0007C014530B8F450E084E190E0489FF001E6
:10DFC000499FF00D589FF00D1124E955FF4E222373
:10DFD00029F0C482D582E682F78204C0C086D18649
:10DFE000E286F386FF90EF90DF90CF9008950F9335
:10DFF0001F93CF93DF938B019C014530F0F450E0E9
:10E0000084E190E0489FE001499FD00D589FD00DDA
:10E010001124C955DF4EC901B8010E94CE4528819F
:10E0200039814A815B810E94F9420E940841DC01EA
:10E03000CB018C879D87AE87BF87DF91CF911F91E2
:10E040000F9108952F923F924F925F926F927F921D
:10E050008F929F92AF92BF92CF92DF92EF92FF92F8
:10E060000F931F93CF93DF93CDB7DEB760970FB6B3
:10E07000F894DEBF0FBECDBF1C018B01DC015E96A4
:10E080008D909D90AD90BC909197D696CD90DD905F
:10E09000ED90FC90D997C701B6010E9497462B01DD
:10E0A0003C01F10162A173A184A195A1A501940194
:10E0B0000E94FC439B01AC01C301B2010E94F942E2
:10E0C0000E947AE40E94084169837A838B839C834F
:10E0D000D8016D917D918D919C91A50194010E9433
:10E0E000FC439B01AC01C301B2010E94F9420E94B2
:10E0F0007AE40E9408416D837E838F83988729810B
:10E100003A814B815C81283731054105510540F446
:10E1100088E790E0A0E0B0E089839A83AB83BC837A
:10E120002D813E814F8158852837310541055105A4
:10E1300040F488E790E0A0E0B0E08D839E83AF8359
:10E14000B88769817A818B819C819B01AC010E9497
:10E15000EFE269877A878B879C876D817E818F81CB
:10E1600098859B01AC010E94EFE26D877E878F87C7
:10E17000988BC701B601A70196010E94EFE22B011F
:10E180003C01F101EE5BFF4FC080D180E280F38063
:10E19000CC0CDD1CEE1CFF1CC114D104E104F10405
:10E1A00079F029853A854B855C85621B730B840B5E
:10E1B000950BA70196010E9463E349015A0103C030
:10E1C00088249924540122273327A9012C193D09B9
:10E1D0004E095F0969F06D857E858F859889641980
:10E1E0007509860997090E9463E389019A0104C0B1
:10E1F00000E010E020E030E0D10154968D919C9138
:10E2000055972C0166247724D301C20188199909F6
:10E21000AA09BB09801B910BA20BB30BB7FF3FC030
:10E2200046015701880C991CAA1CBB1C811491043F
:10E23000A104B10409F1C701B601A30192010E9432
:10E24000EFE2DC01CB0129853A854B855C85821B99
:10E25000930BA40BB50B2D853E854F855889820FF6
:10E26000931FA41FB51FBC01CD01A50194010E94FD
:10E2700063E349015A0103C0882499245401B7FE7D
:10E2800003C0882499245401481459046A047B0467
:10E2900014F45301420180E090E0A0E0B0E04FB7F9
:10E2A000F8949401F101978A868A280F391F318FDB
:10E2B000208F89819A81AB81BC8182AF93AFA4AF5B
:10E2C000B5AF9101225C3F4F8D819E81AF81B885B2
:10E2D000F90180839183A283B3834FBF81E060966D
:10E2E0000FB6F894DEBF0FBECDBFDF91CF911F9167
:10E2F0000F91FF90EF90DF90CF90BF90AF909F90E5
:10E300008F907F906F905F904F903F902F900895E7
:10E310003F924F925F926F927F928F929F92AF92B5
:10E32000BF92CF92DF92EF92FF920F931F93CF9302
:10E33000DF9300D000D0CDB7DEB78091350E90913D
:10E34000360E5090370E6090380E850D891B862151
:10E35000823008F4A3C0B090350E2091390E309170
:10E360003A0E3A83298307E4B09E80011124020FFC
:10E37000131F5A94B7E44B2E82E0382E02C00B8153
:10E380001C81B50CB620B49CC0011124E981FA812E
:10E390008E0F9F1F9C838B83009709F47AC0FC012A
:10E3A000A6A097A080A471A462A173A184A195A145
:10E3B0009401CA2CD32EE22EF72CA70196010E94BD
:10E3C000D944882309F465C0EB81FC81EA5BFF4FE7
:10E3D0008081882309F05DC0F801C2A0D3A0E4A029
:10E3E000F5A08A2D992DA82DB72DBC01CD01A7012F
:10E3F00096010E943B4587FD3DC0C701B601A701BC
:10E4000096010E94F9426B017C01EB81FC8186A59B
:10E4100097A5A0A9B1A99C01AD015058CA01B901A5
:10E420000E948D42EB81FC8122A533A544A555A510
:10E430000E94F9429B01AC01C701B6010E94C14292
:10E440000E94D8E4C62EF72EE82ED92E8A2D992DBB
:10E45000A82DB72DBC01CD01A7010C2D152F242F00
:10E460003D2DA90198010E946C4587FD03C0AC2C8D
:10E4700047017D2C8A2D992DA82DB72DEB81FC818C
:10E4800082A393A3A4A3B5A3EB81FC81EA5BFF4F16
:10E4900030828091360EB81609F071CF0F900F9030
:10E4A0000F900F90DF91CF911F910F91FF90EF9000
:10E4B000DF90CF90BF90AF909F908F907F906F90A4
:10E4C0005F904F903F9008956F927F928F929F92AE
:10E4D000AF92BF92CF92DF92EF92FF920F931F9372
:10E4E000CF93DF93EC013B01009709F479C0FC0165
:10E4F000EA5BFF4F808182FD73C0CAA0DBA0ECA065
:10E50000FDA0FB01B2A0A3A094A085A0C701B60105
:10E51000F501A4010F2F1E2F252F342FA9019801DB
:10E520000E949D4518160CF45BC0C701B601A701F7
:10E5300096010E94F9426B017C018EA59FA5A8A9B6
:10E54000B9A99C01AD015058CA01B9010E948D4280
:10E550002AA53BA54CA55DA50E94F9429B01AC01F3
:10E56000C701B6010E94C1420E94D8E4C62EC72F3F
:10E57000D82FF92EA5019401852F942FA32FB22F08
:10E58000BC01CD010C2D1C2F2D2F3F2DA901980171
:10E590000E946C4587FF04C0CB2CCA2DD92DF82CC6
:10E5A000A5019401852F9A2DA32FB82DBC01CD0173
:10E5B0000C2D1C2F2D2F3F2DA90198010E94D9440D
:10E5C000882371F0802F9C2FAD2FBF2DF30182A3E4
:10E5D00093A3A4A3B5A3EA5BFF4F808182608083ED
:10E5E000DF91CF911F910F91FF90EF90DF90CF902F
:10E5F000BF90AF909F908F907F906F900895EF9213
:10E60000FF920F931F93CF93DF93C091360EEE24AA
:10E61000FF2480E090E0D7E413C0CD9F9001112447
:10E620000091390E10913A0E020F131FB701A80185
:10E630000E946472CF5F8091380EC823C7017801B1
:10E640002091350EC21749F7B70140E050E00E9413
:10E650006472DF91CF911F910F91FF90EF90089519
:10E66000EF92FF920F931F93CF93DF931091360E8B
:10E67000C0E0D0E007E429C0109FC0011124E09061
:10E68000390EF0903A0EE80EF91E2097C9F0FE01FF
:10E69000EA5BFF4F808181FD08C0F701EA5BFF4F15
:10E6A000908191FF0DC080FD0BC0B7016E5D7F4F63
:10E6B000CE010E942270CA5BDF4F88818D7F8883E4
:10E6C0001F5F8091380E1823E7018091350E212FAE
:10E6D000332727FD309590E02817390769F6BE01EA
:10E6E0006E5C7F4FCE010E942270CA5BDF4F888133
:10E6F0008D7F888381E0DF91CF911F910F91FF90F3
:10E70000EF9008950E9488710E94FF720E943073FA
:10E7100008959091350E2091360E9F5F8091380EAE
:10E72000982381E0921380E008952091350E909116
:10E73000360E81E0291380E008958091060E88232B
:10E7400049F42091350E9091360E81E0291719F485
:10E7500080E0089580E008952091360E87E4289F98
:10E76000900111248091390E90913A0E820F931FDF
:10E7700008958091360E8F5F9091380E8923809393
:10E78000360E08952F923F924F925F926F927F9232
:10E790008F929F92AF92BF92CF92DF92EF92FF92B1
:10E7A0000F931F93CF93DF93CDB7DEB7CA54D040FA
:10E7B0000FB6F894DEBF0FBECDBF89AB9AAB4BABA3
:10E7C0005CAB6DAB7EAB3CA72BA79091350E87E47D
:10E7D000989FC00111242091390E30913A0E280FD4
:10E7E000391F3AA729A7F901EA5BFF4F1082D90127
:10E7F000E9A9FAA984E101900D928150E1F78BA576
:10E800009CA560E070E00E94CF7EDC01CD90DD90A1
:10E81000ED90FC901397F7FE08C0F094E094D0942C
:10E82000C094C11CD11CE11CF11C8BA59CA560E00F
:10E8300070E00E94CF7EFC016081718182819381B2
:10E840000E94CE452091A7103091A8104091A910A8
:10E850005091AA100E94FC43162F072F382E292E04
:10E86000A8019101852F942FA32FB22F8D8B9E8B02
:10E87000AF8BB88F8BA59CA561E070E00E94CF7E26
:10E88000DC018D909D90AD90BC901397B7FE08C0B1
:10E89000B094A09490948094811C911CA11CB11CF4
:10E8A0008C149D04AE04BF0414F4460157018BA5DB
:10E8B0009CA561E070E00E94CF7EFC0160817181C7
:10E8C000828193810E94CE452091BB103091BC1073
:10E8D0004091BD105091BE100E94FC43762E472EF1
:10E8E000682E592E862F942DA62DB52D898F9A8F9F
:10E8F000AB8FBC8F8BA59CA562E070E00E94CF7EA1
:10E90000FC0180819181A281B381B7FF07C0B095DE
:10E91000A095909581959F4FAF4FBF4F75016401B2
:10E9200088169906AA06BB0614F46C017D018BA516
:10E930009CA562E070E00E94CF7EDC016D917D912C
:10E940008D919C910E94CE452091CF103091D01096
:10E950004091D1105091D2100E94FC43B62EA72EA8
:10E96000982E892EA5019401852F942FA32FB22FC5
:10E970008D8F9E8FAF8FB8A3C114D104E104F10431
:10E9800009F44EC0A8019101852F902FA32FB22D1D
:10E99000BC01CD01F801A1010F2F1E2F252F3B2F08
:10E9A000A90198010E94F9426DA77EA78FA798AB95
:10E9B000362D872D942DA62DB52DBC01CD01072D0B
:10E9C000142D232F3B2FA90198010E94F9429B018E
:10E9D000AC016DA57EA58FA598A90E948D422B0143
:10E9E0003C01A5019401852F942FA32FB22FBC01C8
:10E9F000CD01F501A4010F2F1E2F252F342FA901C2
:10EA000098010E94F9429B01AC01C301B2010E942E
:10EA10008D420E94D8E4962E872E482E792E04C06F
:10EA200099248824442477248BA59CA563E070E076
:10EA30000E94CF7EFC0180819181A281B381B7FFCA
:10EA400007C0B095A095909581959F4FAF4FBF4F50
:10EA50008DA79EA7AFA7B8AB8C159D05AE05BF05CA
:10EA600024F4CDA6DEA6EFA6F8AA8BA59CA563E0AC
:10EA700070E00E94CF7EDC016D917D918D919C9123
:10EA80000E94CE452091E3103091E4104091E510B2
:10EA90005091E6100E94FC43162F072FB82EA92E86
:10EAA000C62ED72EE82EF92E862F902FAB2DBA2DFD
:10EAB00089A39AA3ABA3BCA3A401852F982DA42D51
:10EAC000B72DBC01CD0120E030E040E050E00E94D5
:10EAD000A844882399F4812F902FAB2DBA2DBC0127
:10EAE000CD0120E030E040E050E00E940A451816D9
:10EAF00054F0F7FAF094F7F8F09405C09401C32E9F
:10EB0000D82CE42CF72C8BA59CA564E070E00E9427
:10EB1000CF7EFC0180819181A281B381B7FF07C0C4
:10EB2000B095A095909581959F4FAF4FBF4F2DA564
:10EB30003EA54FA558A9281739074A075B0724F4B3
:10EB40008DA79EA7AFA7B8AB8BA59CA564E070E08E
:10EB50000E94CF7EDC016D917D918D919C910E94F0
:10EB6000CE452091F7103091F8104091F910509156
:10EB7000FA100E94FC43162F072FB82EA92E862FBD
:10EB8000902FAB2DBA2D21968CAF9DAFAEAFBFAFFE
:10EB900021978DA39EA3AFA3B8A7C701B60120E01C
:10EBA00030E040E050E00E94A8448823E1F4812F47
:10EBB000902FAB2DBA2DBC01CD0120E030E040E01C
:10EBC00050E00E940A451816A4F021962CAD3DADE8
:10EBD0004EAD5FAD2197505821962CAF3DAF4EAF53
:10EBE0005FAF219706C02196CCAEDDAEEEAEFFAE94
:10EBF00021978DA59EA5AFA5B8A90097A105B10540
:10EC000009F4BBC30BA91CA9FDA8EEA880916B0356
:10EC10008823B9F5E9A5FAA5A9A9BAA984E10D90B7
:10EC200001928150E1F760E472E48FE090E0980196
:10EC30004F2D5E2D0E9441E3A9A5BAA5D6962D932E
:10EC40003D934D935C93D99757961C921E9256977D
:10EC5000EDA5FEA55596FC93EE9354975996FC931B
:10EC6000EE9358975A961D921D921D921C925D9795
:10EC70008091350E8F5F9091380E89238093350EE9
:10EC800078C30E946C81882301F56DA57EA58FA5B0
:10EC900098A998014F2D5E2D0E94EFE2DC01CB0177
:10ECA0008031E7E29E07E0E0AE07E0E0BE0768F4EF
:10ECB00060E177E280E090E02DA53EA54FA558A940
:10ECC0000E9441E38901F42EE52EB8018F2D9E2D7F
:10ECD0002DA53EA54FA558A90E94EFE20E94974698
:10ECE0009B01AC0160E074E284E799E40E94FC437C
:10ECF000C62E772E682E592E6DA57EA58FA598A9B4
:10ED00000E9497466FAB78AF89AF9AAF60E070E032
:10ED100080E89FE321962CAD3DAD4EAD5FAD2197D0
:10ED20000E94FC439B01AC016FA978AD89AD9AADFF
:10ED30000E94F942362E272E8BAF9CAF21966CADE8
:10ED40007DAD8EAD9FAD21978C2C972CA62CB52C2C
:10ED5000A50194010E94F94269AB7AAB8BAB9CABE5
:10ED600060E472E48FE090E098014F2D5E2D0E94E8
:10ED700041E3A9A5BAA5D6962D933D934D935C93F7
:10ED8000D99775E1E72EF12CEC0EFD1E5E0108947B
:10ED9000A11CB11CE9E28E2E912C8C0E9D1EF70158
:10EDA00061917191819191917F014C2D572DE62DAB
:10EDB000F52D8A019F01A90198010E94F942DC0109
:10EDC000CB01F50181939193A193B1935F01E81475
:10EDD000F90429F7A1013BAD2CAD852F922DA32F6E
:10EDE000B22FBC01CD012091A3103091A41040910D
:10EDF000A5105091A6100E94F9420E947AE40E9448
:10EE000008416DAB7EAB22968FAF229723969FAFC2
:10EE1000239763EBC62E60E1D62EEE24FF248BA54C
:10EE20009CA5B7010E94CF7E8C01D6018D909D904C
:10EE3000AD90BC906DA97EA922968FAD22972396A6
:10EE40009FAD23970E9497462B013C01F8018081DA
:10EE50009181A281B381B7FF07C0B095A09590952D
:10EE600081959F4FAF4FBF4FBC01CD010E94CE4552
:10EE70002FA938AD49AD5AAD0E94FC439B01AC01AE
:10EE8000C301B2010E94F9420E940841DC01CB019A
:10EE900088169906AA06BB0640F48DAA9EAA229659
:10EEA000AFAE22972396BFAE23970894E11CF11CC6
:10EEB00024E130E0C20ED31E35E0E316F10409F080
:10EEC000AECF6DA97EA922968FAD229723969FADD6
:10EED00023970E949746F1015BAD4CAD0F2F122D89
:10EEE000252F342FA90198010E94FC43462F572F4C
:10EEF000682F792F2B964CAF5DAF6EAF7FAF2B97FE
:10EF0000A9A5BAA59E964D935D936D937C93D197D9
:10EF10006DA97EA922968FAD229723969FAD239748
:10EF200022E43FE040E050E00E9441E3E9A5FAA579
:10EF3000228F338F448F558FF0919F10FBA7209124
:10EF4000A0102FAB3091A1103BAF4091A2104CAF5D
:10EF5000422F2CAD8F2F942FA32FB22FBC01CD01A8
:10EF6000F9A9EAA95BA94CA90F2F1E2F252F342F31
:10EF7000A90198010E946C4587FF05C0BBA4AFA8FA
:10EF80009BAC8CAC04C0B9A8AAA89BA88CA89091F3
:10EF9000350E8091360E981709F40AC160917310EE
:10EFA00070917410809175109091761020E030E08F
:10EFB00040E050E00E940A4518160CF0F9C080911C
:10EFC000771090917810A0917910B0917A102796CF
:10EFD0008CAF9DAFAEAFBFAF279769817A818B8130
:10EFE0009C8127962CAD3DAD4EAD5FAD27970E941D
:10EFF000C1429B01AC010E94F942162F072F782EC7
:10F00000692EC0907B10D0907C10E0907D10F09025
:10F010007E106D817E818F819885A70196010E9467
:10F02000C1429B01AC010E94F942B62FA72F382F95
:10F03000292FF801C3014F2F5E2F692F782FCB01A5
:10F04000BA01FD01A9010F2F1E2F252F342FA90171
:10F0500098010E948D420E94D8E42B013C01279622
:10F060006CAD7DAD8EAD9FAD279720E030E040E0E8
:10F0700050E00E94D944882351F4C701B60120E032
:10F0800030E040E050E00E94D944882321F0B9A844
:10F09000AAA89BA88CA8C0900B11D0900C11E0904E
:10F0A0000D11F0900E11C301B201A70196010E944B
:10F0B0000A451816B4F4C701B601A30192010E94D3
:10F0C000FC439B01AC01F501B4018F2F9A2DA72FB2
:10F0D000B82DBC01CD010E94F942B62EA72E982E64
:10F0E000892E0FE710E1DE0119962596BFAFAEAF6E
:10F0F00025979FED292E90E1392EC10118018C0131
:10F10000F10161917191819191911F012596AEADAF
:10F11000BFAD25972D913D914D915D912596BFAF46
:10F12000AEAF25970E94C142472F382F292FC62EF8
:10F13000D72EE82EF92E862F942FA32FB22FBC01A5
:10F14000CD0120E030E040E050E00E940A45181672
:10F1500024F0F7FAF094F7F8F094F8014080518029
:10F1600062807380C701B601A30192010E940A4523
:10F170001816B4F4C301B201A70196010E94FC4322
:10F180009B01AC01F501B4018F2F9A2DA72FB82D4B
:10F19000BC01CD010E94F942B62EA72E982E892ED1
:10F1A0000C5E1F4FFBE82F16F0E13F0609F0A8CFD9
:10F1B000A5019401852F9A2DA32FB82DE9A5FAA5B5
:10F1C00086A397A3A0A7B1A75BA54FA93BAD2CAD84
:10F1D000852F942FA32FB22FBC01CD01FA010F2F41
:10F1E0001E2F232F3B2FA90198010E94F9426B018A
:10F1F0007C012B962CAD3DAD4EAD5FAD2B9750589D
:10F20000CA01B9010E948D4221962CAD3DAD4EAD93
:10F210005FAD21970E94F9429B01AC01C701B60185
:10F220000E94C1420E94D8E4F62EE72EC82E492E35
:10F23000A5019401852F9A2DA32FB82DBC01CD01D6
:10F24000F7010F2F1E2F2C2D342DA90198010E949C
:10F250006C4587FD03C057019C2C842CA5019401AB
:10F26000852F9A2DA32FB82DE9A5FAA582A393A3E4
:10F27000A4A3B5A359A94AA93BA92CA9852F942FCA
:10F28000A32FB22FBC01CD01F7010F2F1E2D2C2D66
:10F29000342DA90198010E949D45E9A5FAA5EA5BD4
:10F2A000FF4F18161CF08081846002C080818B7F24
:10F2B0008083808182608083A7E7B0E1FE01319680
:10F2C00084E101900D928150E1F759A94AA93BA927
:10F2D0002CA9852F942FA32FB22F80937310909376
:10F2E0007410A0937510B093761021962CAD3DAD9F
:10F2F0004EAD5FAD2197A9A5BAA59A962D933D93E2
:10F300004D935C939D97EDA5FEA55596FC93EE93CA
:10F3100054973BA92CA9A32FB22FE9A5FAA5868F54
:10F32000978FA0A3B1A3EE5BFF4F2DA920833EA929
:10F33000318322964FAD2297428323965FAD239768
:10F3400053835BA54FA93BAD2CAD852F942FA32FE5
:10F35000B22FE9A5FAA582AB93ABA4ABB5AB809174
:10F36000350E8F5F9091380E89238093350E0E9461
:10F3700082730E94B88C81E001C080E0C65BDF4FE1
:10F380000FB6F894DEBF0FBECDBFDF91CF911F91B6
:10F390000F91FF90EF90DF90CF90BF90AF909F9034
:10F3A0008F907F906F905F904F903F902F90089537
:10F3B000CF92DF92EF92FF920F931F93CF93DF9341
:10F3C000CDB7DEB7EC970FB6F894DEBF0FBECDBF5A
:10F3D0006C018B01CE0145960E949A7E40910B0EE6
:10F3E00050910C0ECE018996B6010E946B7FDE0112
:10F3F0005596FE01B99684E101900D928150E1F796
:10F40000CE01459662E070E00E94D77EFC0140810B
:10F410005181628173818091D3109091D410A09119
:10F42000D510B091D61084179507A607B7079CF49E
:10F43000CE01459662E070E00E94D77E4091D310E5
:10F440005091D4106091D5107091D610FC0140837A
:10F45000518362837383F801C080D180E280F3809E
:10F46000CE010196BE016B5E7F4F4BE850E10E94DA
:10F47000DF7ECE014596B701A6019E012F5F3F4F6B
:10F480000E94C273ABE8B0E1FE01759684E1019081
:10F490000D928150E1F7EC960FB6F894DEBF0FBEE7
:10F4A000CDBFDF91CF911F910F91FF90EF90DF9033
:10F4B000CF9008952F923F924F925F926F927F92DA
:10F4C0008F929F92AF92BF92CF92DF92EF92FF9274
:10F4D0000F931F93CF93DF93CDB7DEB7C054D040C7
:10F4E0000FB6F894DEBF0FBECDBF2C017EAF6DAF5F
:10F4F000C42ECE0145960E949A7E40910B0E5091EB
:10F500000C0ECE018996B2010E946B7FDE015596EA
:10F51000FE01B99684E101900D928150E1F700E07F
:10F5200010E08824992454012C2C332427FC309497
:10F53000C101002E02C0959587950A94E2F780FFDD
:10F540002CC0CE014596B8010E94D77E3C018BE8C5
:10F5500090E1B8010E94D77EFC01C080D180E2809A
:10F56000F380C201B8010E94CF7EFC0180819181AD
:10F57000A281B3818C0D9D1DAE1DBF1DF301808343
:10F580009183A283B383C201B8010E94CF7EFC01A4
:10F5900080819181A281B38140C0CE014596B8019E
:10F5A0000E94D77E3C01C201B8010E94CF7EFC01BF
:10F5B000C080D180E280F38080910B0E90910C0E80
:10F5C000B8010E94D77EFC0180819181A281B38124
:10F5D0008C0D9D1DAE1DBF1DF30180839183A28301
:10F5E000B383CE014596B8010E94D77EFC01C0804E
:10F5F000D180E280F3808BE890E1B8010E94D77E51
:10F60000FC0180819181A281B381A7019601281B11
:10F61000390B4A0B5B0BDA01C901B7FF07C0B09584
:10F62000A095909581959F4FAF4FBF4F8816990633
:10F63000AA06BB0614F44C015D010F5F1F4F053095
:10F64000110509F075CFCE01459662E070E00E9489
:10F65000D77EFC0140815181628173818091D310FA
:10F660009091D410A091D510B091D6108417950721
:10F67000A607B7079CF4CE01459662E070E00E94B1
:10F68000D77E4091D3105091D4106091D5107091D5
:10F69000D610FC014083518362837383EDADFEADD0
:10F6A0006081718182819381A50194010E9463E34D
:10F6B000C42E052FCE010196BE016B5E7F4F4BE835
:10F6C00050E12FAF21963FAF21970E94DF7ECE0100
:10F6D00045962FAD422F21963FAD2197532F6C2D8C
:10F6E000702F9E012F5F3F4F0E94C273ABE8B0E1C5
:10F6F000FE01759684E101900D928150E1F7C05CA6
:10F70000DF4F0FB6F894DEBF0FBECDBFDF91CF91B4
:10F710001F910F91FF90EF90DF90CF90BF90AF902F
:10F720009F908F907F906F905F904F903F902F9021
:10F7300008954F925F927F928F929F92AF92BF9265
:10F74000CF92DF92EF92FF920F931F93CF93DF93AD
:10F750007FB6F89402E611E0C0E0D0E0FAE08F2E28
:10F76000912CA12CB12CC80140E050E060E070E089
:10F770000E945FAE6B017C018DE09EE0BE010E94A5
:10F78000D77E2C01C701B601A50194010E9463E355
:10F79000F201208331834283538321960C5F1F4FF4
:10F7A000C330D10501F7C2E0D0E08DE09EE0BE019C
:10F7B0000E94D77EFC011082118212821382219650
:10F7C000C530D10591F7C0E0D0E081E29EE0BE01F6
:10F7D0000E94D77EFC011082118212821382219630
:10F7E000C530D10591F77FBEDF91CF911F910F9169
:10F7F000FF90EF90DF90CF90BF90AF909F908F9051
:10F800007F905F904F900895813019F48DE09EE0D5
:10F8100002C081E29EE090930C0E80930B0E08953F
:10F82000CF93DF93CDB7DEB764970FB6F894DEBF02
:10F830000FBECDBF0E943686CE0101960E949686ED
:10F84000ABE8B0E1FE01319684E101900D92815068
:10F85000E1F70E94997B80E00E94047C80E090E0C8
:10F86000A0E0B0E08093771090937810A093791087
:10F87000B0937A1080937B1090937C10A0937D10AE
:10F88000B0937E1080937F1090938010A09381108E
:10F89000B09382108093831090938410A09385106E
:10F8A000B09386108093871090938810A09389104E
:10F8B000B0938A108093731090937410A093751076
:10F8C000B09376101092350E1092360E8EE691E0BF
:10F8D00061E00E941BAE91E0882309F490E09093D0
:10F8E0006B031092070E1092080E1092090E1092E0
:10F8F0000A0E1092060E64960FB6F894DEBF0FBE85
:10F90000CDBFDF91CF91089582E691E04FEF5FEF99
:10F910006FEF7FEF0E945FAEDC01CB018F3F2FEFD7
:10F9200092072FEFA2072FEFB20711F40E940F5B8F
:10F9300087E897E4ACEBB2E48093A7109093A8100B
:10F94000A093A910B093AA108093BB109093BC1001
:10F95000A093BD10B093BE1080E090E0A8ECB3E49B
:10F960008093CF109093D010A093D110B093D21069
:10F9700087EE9CE8A0ECB2E48093E3109093E4104F
:10F98000A093E510B093E6108093F7109093F810D1
:10F99000A093F910B093FA1088E891E06FEF0E94FD
:10F9A0001BAE883011F00E94AC5980E791E060ED09
:10F9B00077E00E9439AEBC0180E090E00E94CE4525
:10F9C000DC01CB018093A3109093A410A093A51009
:10F9D000B093A61082E791E06CED75E00E9439AE1D
:10F9E000BC0180E090E040E00E94F76F84E791E086
:10F9F0006CED75E00E9439AEBC0180E090E041E022
:10FA00000E94F76F86E791E068EE73E00E9439AEDE
:10FA1000BC0180E090E042E00E94F76F88E791E04F
:10FA200068EB7BE00E9439AEBC0180E090E043E0EF
:10FA30000E94F76F8AE791E068EB7BE00E9439AEA5
:10FA4000BC0180E090E044E00E94F76F8CE791E019
:10FA500040E050E060EA71E40E94FFAEDC01CB01BF
:10FA600080930B1190930C11A0930D11B0930E1174
:10FA700080E891E040E050E060E87FE30E94FFAE64
:10FA8000DC01CB018093DF109093E010A093E11094
:10FA9000B093E21082E891E040E050E060E070E472
:10FAA0000E94FFAEDC01CB018093F3109093F41021
:10FAB000A093F510B093F61084E891E040E050E098
:10FAC00060E070E40E94FFAEDC01CB01809307117F
:10FAD00090930811A0930911B0930A1186E891E060
:10FAE0006FE070E00E9439AEBC0180E090E00E94BF
:10FAF0009746DC01CB0180939F109093A010A093B8
:10FB0000A110B093A21084E991E040E65AEE60E0C3
:10FB100070E00E945FAE42E021E00E94D36F60E09F
:10FB200070E080E090E042E020E00E94D36F0E940D
:10FB3000107C0895CF93DF93CDB7DEB764970FB6EF
:10FB4000F894DEBF0FBECDBFBC0140910B0E5091AB
:10FB50000C0ECE0101960E946B7FABE8B0E1FE0176
:10FB6000319684E101900D928150E1F78BE890E1AC
:10FB700062E070E00E94D77EFC0140815181628189
:10FB800073818091D3109091D410A091D510B09131
:10FB9000D61084179507A607B7079CF48BE890E169
:10FBA00062E070E00E94D77E4091D3105091D41053
:10FBB0006091D5107091D610FC014083518362830F
:10FBC00073838BE890E10E94728680E090E0A0E071
:10FBD000B0E08093771090937810A0937910B09351
:10FBE0007A1080937B1090937C10A0937D10B0933B
:10FBF0007E1080937F1090938010A0938110B0931B
:10FC000082108093831090938410A0938510B093FA
:10FC100086108093871090938810A0938910B093DA
:10FC20008A108093731090937410A0937510B09302
:10FC3000761064960FB6F894DEBF0FBECDBFDF918D
:10FC4000CF910895CF93DF93EC0140910B0E50912B
:10FC50000C0E6BE870E10E94DF7ECE01DF91CF9148
:10FC60000895EF92FF920F931F93CF93DF93CDB739
:10FC7000DEB7C754D0400FB6F894DEBF0FBECDBF7D
:10FC80008FE091E164E477E140E00E94DEDE8BE802
:10FC900090E10E949A7E0BE31EE0C8010E949A7ECA
:10FCA000095B1F4F80E103371807B9F71092350E33
:10FCB0001092360E88E08093370E87E08093380EDE
:10FCC0008BE39EE090933A0E8093390EFF24A7E4D5
:10FCD000EA2E16C0FE9CC00111240091390E10912D
:10FCE0003A0E080F191FCE0101960E949A7ED80184
:10FCF000FE01319687E401900D928150E1F7F39473
:10FD00008091370EF81630F381E29EE00E949A7ED1
:10FD10008DE09EE00E949A7EC95BDF4F0FB6F8949B
:10FD2000DEBF0FBECDBFDF91CF911F910F91FF902E
:10FD3000EF90089508958F929F92AF92BF92CF92C5
:10FD4000DF92EF92FF920F931F93CF93DF93CDB784
:10FD5000DEB7FC0140835183628373830483158380
:10FD600026833783C086D186E286F386848695868D
:10FD7000A686B7868F859889A989BA89808B918B49
:10FD8000A28BB38BDF91CF911F910F91FF90EF90DA
:10FD9000DF90CF90BF90AF909F908F900895660FA7
:10FDA000771F660F771F680F791FCB010895660FC5
:10FDB000771F660F771F680F791FCB0108952F9269
:10FDC0003F924F925F926F927F928F929F92AF92EB
:10FDD000BF92CF92DF92EF92FF920F931F93CF9338
:10FDE000DF9300D000D0CDB7DEB71C01DB01149645
:10FDF0004D905D906D907C901797FA01048115816C
:10FE000026813781401A510A620A730A18968D902A
:10FE10009D90AD90BC901B97008511852285338500
:10FE2000801A910AA20AB30A1C96CD90DD90ED903B
:10FE3000FC901F970485158526853785C01AD10A41
:10FE4000E20AF30A50960D911D912D913C91539722
:10FE500080899189A289B389081B190B2A0B3B0B56
:10FE6000FB0180819181A281B381FA01408151819E
:10FE700062817381841B950BA60BB70BF101808304
:10FE80009183A283B383448255826682778280867F
:10FE90009186A286B386C486D586E686F786008BD1
:10FEA000118B228B338BC1010F900F900F900F900D
:10FEB000DF91CF911F910F91FF90EF90DF90CF9046
:10FEC000BF90AF909F908F907F906F905F904F907A
:10FED0003F902F9008952F923F924F925F926F9292
:10FEE0007F928F929F92AF92BF92CF92DF92EF92CA
:10FEF000FF920F931F93CF93DF9300D000D0CDB725
:10FF0000DEB71C01DB0114964D905D906D907C90E6
:10FF10001797FA010481158126813781400E511E01
:10FF2000621E731E18968D909D90AD90BC901B978D
:10FF30000085118522853385800E911EA21EB31E79
:10FF40001C96CD90DD90ED90FC901F970485158553
:10FF500026853785C00ED11EE21EF31E50960D91E8
:10FF60001D912D913C91539780899189A289B389E4
:10FF7000080F191F2A1F3B1FFB0180819181A2815D
:10FF8000B381FA014081518162817381840F951F91
:10FF9000A61FB71FF10180839183A283B38344829C
:10FFA00055826682778280869186A286B386C486D1
:10FFB000D586E686F786008B118B228B338BC101A9
:10FFC0000F900F900F900F90DF91CF911F910F9195
:10FFD000FF90EF90DF90CF90BF90AF909F908F9069
:10FFE0007F906F905F904F903F902F9008950F9368
:10FFF00080E798EA6DE279EA49E35AEA24EF3AEABF
:020000021000EC
:1000000000E00E9490A69093251180932411009700
:1000100079F480E798EA6DE279EA49E35AEA24EF55
:100020003AEA0FEF0E9490A6909325118093241135
:1000300081E020912411309125112115310509F419
:1000400080E00F91089580912411909125110E94D4
:10005000929F9C01909323118093221181E021159E
:10006000310509F480E00895CF93DF93CDB7DEB773
:10007000AB970FB6F894DEBF0FBECDBF80912211B3
:100080009091231165E372E0AE014F5F5F4F0E94D4
:10009000ECA48091221190912311BE016F5F7F4FDC
:1000A0000E94DAA39C01909321118093201181E09A
:1000B0002115310509F480E0AB960FB6F894DEBF48
:1000C0000FBECDBFDF91CF91089580912211909105
:1000D00023110E9465A6DC01CB0180959095A09527
:1000E000B0958827B7FD83959927AA27BB27089540
:1000F000AF92BF92CF92DF92EF92FF921F93CF9376
:10010000DF93CDB7DEB7AB970FB6F894DEBF0FBE67
:10011000CDBF7C015A0115E0C62EDD240894C1082C
:10012000D1088091201190912111BE016F5F7F4F06
:100130000E941DA4F7018823E1F0DE01119680E002
:1001400090E08C159D0534F42D91222319F0219314
:100150000196F7CFF701E80FF91F1082009731F0F1
:10016000A114B10439F0F501808304C01150C9F61F
:1001700001C0108280E090E0AB960FB6F894DEBF2D
:100180000FBECDBFDF91CF911F91FF90EF90DF9019
:10019000CF90BF90AF9008950F931F93CF93DF93AD
:1001A0008C01EB010EC0CE01B8010E9442E4009721
:1001B00041F480912011909121110E9477A581E056
:1001C00009C08091201190912111BE010E941DA4AF
:1001D000882349F7DF91CF911F910F9108950F93D5
:1001E0001F93CF93DF93CDB7DEB7AB970FB6F894DD
:1001F000DEBF0FBECDBF8B01BE016F5F7F4F0E9480
:10020000CC80882371F08091221190912311BE013E
:100210006F5F7F4F0E943DA1F8019183808381E051
:1002200001C080E0AB960FB6F894DEBF0FBECDBF25
:10023000DF91CF911F910F91089580911E119091A0
:100240001F110E945FA60895CF93DF93CDB7DEB74D
:10025000AB970FB6F894DEBF0FBECDBFBE016F5F88
:100260007F4F0E94CC80882359F080912211909179
:100270002311BE016F5F7F4F0E94E1A581E001C0A5
:1002800080E0AB960FB6F894DEBF0FBECDBFDF9116
:10029000CF910895CF93DF93CDB7DEB7AB970FB66D
:1002A000F894DEBF0FBECDBFBC01809120119091AC
:1002B0002111AE014F5F5F4F0E9484A591E088231A
:1002C00009F490E0892FAB960FB6F894DEBF0FBE0D
:1002D000CDBFDF91CF91089580911C110895809139
:1002E0001D110895CF93DF93EC0180911E11909121
:1002F0001F110097E1F0BE016E5F7F4F488150E013
:100300000E9499A228818091181190911911A091B1
:100310001A11B0911B11820F911DA11DB11D809367
:10032000181190931911A0931A11B0931B11DF911A
:10033000CF91089580911D11882381F080911E1125
:1003400090911F11009721F00E9474A10E9417A89C
:1003500010921F1110921E1110921D116091181110
:100360007091191180911A1190911B1108950E949A
:10037000D1A7882391F080911E1190911F1167E100
:1003800071E141E050E00E9487A121E018161906B2
:100390000CF020E020931611089589EB99E06DE0B0
:1003A00077E041E00E948E691092161110921511AB
:1003B0000895809116110895CF93DF930F92CDB7D2
:1003C000DEB78091171189830E94B78189810F90D0
:1003D000DF91CF91089510921C1180911E11909180
:1003E0001F11009721F00E9474A10E9417A810927B
:1003F0001F1110921E11089580911C11882311F075
:100400000E94EB8180911D11882311F00E949A8136
:100410008091201190912111009731F00E9417A432
:10042000109221111092201180912211909123118C
:10043000009731F00E9437A11092231110922211DF
:100440008091241190912511009731F00E9461A7AD
:10045000109225111092241108950E9481A98823D9
:1004600071F40E94D1A7882329F40E94FC8181E0C5
:1004700090E008950E94FC8182E090E008950E943F
:10048000F77F882329F40E94FC8183E090E008959F
:100490000E942380882329F40E94FC8184E090E05C
:1004A00008950E943480882329F40E94FC8185E00D
:1004B00090E008950E946580882329F40E94FC81C1
:1004C0008AE090E008950E94F5A7882319F086E05D
:1004D00090E0089580E090E00895CF93DF93EC01E1
:1004E0000E94FC810E942D82009719F086309105B0
:1004F000D9F4109218111092191110921A11109229
:100500001B1110921F1110921E11CE016EE171E1AC
:100510000E94EF80882331F080911E1190911F116D
:10052000009729F487E090E0DF91CF91089581E072
:1005300080931C110E94B78180E090E0F5CF0F936B
:100540001F93CF93DF938C010E94FC810E942D8228
:10055000EC01009769F51092181110921911109280
:100560001A1110921B1110921F1110921E11C80126
:100570000E942481C8010E944A81882389F0C80111
:100580006EE171E10E94EF80882369F080911E1175
:1005900090911F11009751F081E080931D1108C0C8
:1005A000C7E0D0E005C0C3E0D0E002C0C8E0D0E0C2
:1005B000CE01DF91CF911F910F9108950E94FC8190
:1005C0000E942D82009719F08630910541F48091A8
:1005D0002011909121110E9477A580E090E008956C
:1005E00086E291E164E477E140E00E94DEDE089576
:1005F000CF92DF92EF92FF920F931F93CF93DF93EF
:10060000CDB7DEB76E970FB6F894DEBF0FBECDBF85
:100610006C017C018C01025E1F4FC7010E94D0DE7D
:1006200086E090E0E80EF91EE016F106B1F7C6018B
:100630004E966AE477E145E00E94DEDE85E0F60151
:1006400084A3CE01499660E577E143E00E94DEDEB7
:10065000D601FE01799686E001900D928150E1F776
:10066000CE01439660E577E147E00E94DEDED601E9
:100670001696FE01739686E001900D928150E1F787
:10068000CE010D9668E477E143E00E94DEDED601FC
:100690001C96FE013D9686E001900D928150E1F797
:1006A000CE0107966AE577E145E00E94DEDED601DD
:1006B0005296FE01379686E001900D928150E1F747
:1006C000CE0101966AE477E146E00E94DEDED601C3
:1006D0005896FE01319686E001900D928150E1F727
:1006E0006E960FB6F894DEBF0FBECDBFDF91CF91EF
:1006F0001F910F91FF90EF90DF90CF900895FF92A0
:100700000F931F93CF93DF938C01FF2414C08F2D81
:1007100090E0EC01CC0FDD1FC80FD91FCC0FDD1FFF
:10072000C00FD11FCE0161E00E9413DFCE0161E056
:100730000E94E364F394F80184A1F81640F3025E8A
:100740001F4FC80161E00E9413DFC80161E00E94F1
:10075000E364DF91CF911F910F91FF9008951F9354
:10076000CF93DF93EC0115E1812F8A95F1F7CE014C
:100770004E9661E00E94E3641A95F1F710E00FC015
:10078000212F30E0C901880F991F820F931F880F16
:10079000991F8C0F9D1F61E00E94E3641F5F8CA175
:1007A000181770F385E18A95F1F7DF91CF911F91CA
:1007B0000895BF92CF92DF92EF92FF920F931F9313
:1007C000CF93DF93D62EEA01A8E0EA2EF12CB0E811
:1007D000CB2E8C01025E1F4F25E1B22E8C2D8D2178
:1007E00061E009F460E0CE010E94E364C80161E0C9
:1007F0000E94E3648B2D8A95F1F7C80160E00E94A6
:10080000E364C6940894E108F108E114F10431F7B7
:10081000CE0161E00E94E364CE0160E00E9413DF3C
:10082000C80161E00E94E3648A81882349F4E88179
:10083000F98180819C818923EE24E394882309F443
:10084000EE24C80160E00E94E364CE0161E00E94F2
:1008500013DF81E0E11080E0DF91CF911F910F91D4
:10086000FF90EF90DF90CF90BF900895EF92FF92AE
:100870000F931F93CF93DF93EC01162F7A0100E0C3
:100880000FC0202F30E0C901880F991F820F931FDE
:10089000880F991F8C0F9D1F60E00E94E3640F5F1B
:1008A0008CA1081770F385E18A95F1F7CE014E9679
:1008B00060E00E94E364CE01612FA7010E94D9830A
:1008C000DF91CF911F910F91FF90EF90089581E5F7
:1008D00091E164E477E140E00E94DEDE8CE291E1A8
:1008E0000E94F88208952091601130E08AE791E13A
:1008F000F901EE0FFF1FE20FF31FEE0FFF1FEE0FC8
:10090000FF1FE80FF91F448155816681778140936D
:10091000761150937711609378117093791120912B
:10092000601130E0F901EE0FFF1FE20FF31FEE0F31
:10093000FF1FEE0FFF1FE80FF91F408151816281F9
:1009400073814093651150936611609367117093A2
:1009500068112091601130E0F901EE0FFF1FE20FE6
:10096000F31FEE0FFF1FEE0FFF1FE80FF91F80852B
:100970009185A285B38580936E1190936F11A0939A
:100980007011B093711108958091F711882349F483
:1009900080915A11882329F40E94957391E0982739
:1009A00001C091E0892F0895DF92EF92FF920F939B
:1009B0001F93CF93DF93809A819A8A9A829A849A1E
:1009C000859A8E9A869A80910701816080930701AB
:1009D0008091070182608093070180910801846003
:1009E00080930801809107018460809307010A9A2F
:1009F0000B9A149A0C9A0E9A0F9AA29A9A9A09EE46
:100A000011E184EEE82E81E1F82EC0E0D0E082E032
:100A100090E060E00E941BAED82E84E090E060E0A1
:100A20000E941BAE2C2F87FF09C090E00C2E02C045
:100A3000959587950A94E2F7817001C081E0F801ED
:100A400081938F018D2D90E002C0959587952A9511
:100A5000E2F781709070F70181937F012196C53094
:100A6000D105A9F680910A018D7F80930A018091BA
:100A7000E911882321F080910B01826003C08091ED
:100A80000B018D7F80930B0180910A018E7F8093F3
:100A90000A018091E911882321F080910B01816086
:100AA00003C080910B018E7F80930B0180910A011E
:100AB000877F80930A018091EA11882321F0809139
:100AC0000B01886003C080910B01877F80930B012D
:100AD00080910A018B7F80930A018091EA1188231B
:100AE00021F080910B01846003C080910B018B7F0A
:100AF00080930B0180910A018F7780930A01809186
:100B0000EB11882321F080910B01806803C0809154
:100B10000B018F7780930B0180910A018F7B80936B
:100B20000A018091EB11882321F080910B018064F0
:100B300003C080910B018F7B80930B01C0E0D0E05C
:100B4000CE01880F991F8C0F9D1F880F991F880F4A
:100B5000991F88509E4E6C2F0E9406AE2196C5307C
:100B6000D10571F7DF91CF911F910F91FF90EF9019
:100B7000DF90089580E090E041E09C01220F331F58
:100B8000220F331FF901E053FE4E108211821282B0
:100B90001382F901E454FE4E1082118212821382F4
:100BA00028553E4EF9011082118212821382FC01F7
:100BB000E256FE4E4083019685309105F1F6089588
:100BC0000E94D4841092EE1108951092F7111092A1
:100BD0005A110E94D4840E94BA8510925C1110921E
:100BE0005D1110925E1110925F11109258111092C7
:100BF0005711EAE7F1E11082118212821382108606
:100C000011861286138614821582168217823C96EC
:100C100081E1EE39F80779F7109276111092771189
:100C20001092781110927911109272111092731122
:100C300010927411109275111092691110926A112C
:100C400010926B1110926C1181E080936D111092D3
:100C5000611110926211109263111092641110923E
:100C6000601180935B111092EE1108951092F711AC
:100C700010925A1110925C1110925D1110925E1137
:100C800010925F1110925811109257111092761114
:100C900010927711109278111092791110927211AE
:100CA00010927311109274111092751110926911B3
:100CB00010926A1110926B1110926C1181E0809366
:100CC0006D111092611110926211109263111092C5
:100CD00064111092601180E090E19093290180935B
:100CE000280108950F931F93CF93DF938C01C0E0E9
:100CF000D0E0C801BE010E94CF7EFC0180819181BD
:100D0000A281B381FE01EE0FFF1FEE0FFF1FE05324
:100D1000FE4E80839183A283B3832196C530D10593
:100D200041F7DF91CF911F910F9108958F929F927C
:100D3000AF92BF92CF92DF92EF92FF920F931F93E9
:100D4000CF93DF93EC014091D0115091D11160917C
:100D5000D2117091D3110091D4111091D51120911D
:100D6000D6113091D711C090D811D090D911E09000
:100D7000DA11F090DB118090DC119090DD11A090E1
:100D8000DE11B090DF118091E0119091E111A091FE
:100D9000E211B091E31100D000D0EDB7FEB781832E
:100DA0009283A383B483CE010E949B7E0F900F9009
:100DB0000F900F90CE01DF91CF911F910F91FF9077
:100DC000EF90DF90CF90BF90AF909F908F9008955D
:100DD0008093591108958091721190917311A0918F
:100DE0007411B0917511813020E8920720E0A207BC
:100DF00020E0B2072CF08EE190E0A0E0B0E054C01B
:100E00008091721190917311A0917411B09175112C
:100E10008030E0E29E07E0E0AE07E0E0BE07CCF005
:100E20008091721190917311A0917411B09175110C
:100E300080509042A040B04044E0B595A79597956A
:100E400087954A95D1F7835E984FFC01849190E095
:100E500029C08091721190917311A0917411B09179
:100E6000751180329105A105B10564F480E290E02E
:100E7000A0E0B0E08093721190937311A09374116D
:100E8000B09375118091721190917311A0917411AA
:100E9000B0917511FC01EE0FFF1FE25EF24F25913C
:100EA0003491C901A0E0B0E08093691190936A1178
:100EB000A0936B11B0936C1110926D110895CF93A4
:100EC000DF93CDB7DEB7CE01059660E070E00E94FB
:100ED000D77E4091D0115091D1116091D211709173
:100EE000D311FC0180819181A281B381841B950B78
:100EF000A60BB70B8093A8119093A911A093AA11E8
:100F0000B093AB11CE01059661E070E00E94D77EF0
:100F10004091D4115091D5116091D6117091D71193
:100F2000FC0180819181A281B381841B950BA60B6A
:100F3000B70B8093AC119093AD11A093AE11B09309
:100F4000AF11CE01059662E070E00E94D77E40911D
:100F5000D8115091D9116091DA117091DB11FC0117
:100F600080819181A281B381841B950BA60BB70B65
:100F70008093B0119093B111A093B211B093B311BB
:100F8000CE01059663E070E00E94D77E4091DC11AF
:100F90005091DD116091DE117091DF11FC018081B3
:100FA0009181A281B381841B950BA60BB70B809313
:100FB000B4119093B511A093B611B093B711CE01AF
:100FC000059664E070E00E94D77E4091E011509158
:100FD000E1116091E2117091E311FC018081918136
:100FE000A281B381841B950BA60BB70B8093B8111C
:100FF0009093B911A093BA11B093BB118091A8112D
:101000009091A911A091AA11B091AB110097A105DF
:10101000B105D9F18A988091A8119091A911A09158
:10102000AA11B091AB11B7FF1BC08091A81190918C
:10103000A911A091AA11B091AB11B095A09590956E
:1010400081959F4FAF4FBF4F8093A8119093A911E7
:10105000A093AA11B093AB111092A3118FEF03C00C
:1010600081E08093A31180939E118091E4118823E5
:1010700029F08091A31191E0892702C08091A311EA
:10108000882311F0889A01C088988091AC119091C2
:10109000AD11A091AE11B091AF110097A105B105AE
:1010A000D9F18E988091AC119091AD11A091AE11B3
:1010B000B091AF11B7FF1BC08091AC119091AD11F1
:1010C000A091AE11B091AF11B095A095909581957A
:1010D0009F4FAF4FBF4F8093AC119093AD11A09332
:1010E000AE11B093AF111092A4118FEF03C081E045
:1010F0008093A41180939F118091E511882329F09A
:101100008091A41191E0892702C08091A4118823C5
:1011100011F08C9A01C08C988091B0119091B1110E
:10112000A091B211B091B3110097A105B10509F4D6
:1011300045C0809108018B7F809308018091B01198
:101140009091B111A091B211B091B311B7FF1BC032
:101150008091B0119091B111A091B211B091B311E1
:10116000B095A095909581959F4FAF4FBF4F8093BD
:10117000B0119093B111A093B211B093B31110922A
:10118000A5118FEF03C081E08093A5118093A0117A
:101190008091E611882329F08091A51191E089279B
:1011A00002C08091A511882321F0809108018160FF
:1011B00003C0809108018E7F809308018091B41153
:1011C0009091B511A091B611B091B7110097A105FA
:1011D000B105D9F114988091B4119091B511A091F5
:1011E000B611B091B711B7FF1BC08091B4119091A7
:1011F000B511A091B611B091B711B095A095909589
:1012000081959F4FAF4FBF4F8093B4119093B5110D
:10121000A093B611B093B7111092A6118FEF03C02F
:1012200081E08093A6118093A1118091E71188231A
:1012300029F08091A61191E0892702C08091A61122
:10124000882311F0129A01C012988091B8119091E0
:10125000B911A091BA11B091BB110097A105B105C8
:10126000D9F1A2988091B8119091B911A091BA11B9
:10127000B091BB11B7FF1BC08091B8119091B9110B
:10128000A091BA11B091BB11B095A09590958195A0
:101290009F4FAF4FBF4F8093B8119093B911A09358
:1012A000BA11B093BB111092A7118FEF03C081E068
:1012B0008093A7118093A2118091E811882329F0CF
:1012C0008091A71191E0892702C08091A7118823FE
:1012D00011F0169A01C01698DF91CF910895EF9200
:1012E000FF920F931F93CF93DF931092F711E0912A
:1012F0005711F0915811309759F0EA5BFF4F8081F8
:101300008E7F80830E94B9731092581110925711EA
:101310000E949D73882339F40E94957391E0982769
:101320009093F7110DC10E94AC7390935811809364
:101330005711FC01EA5BFF4F208121622083DC0111
:101340005496ED90FC905597EDB7FEB774970FB695
:10135000F894FEBF0FBEEDBF319684E10D9001926F
:101360008150E1F70E945F87109260111092721114
:10137000109273111092741110927511C09157113F
:10138000D09158118E899F892DB73EB72C5E3F4F63
:101390000FB6F8943EBF0FBE2DBF009791F14AAD36
:1013A0005BAD6CAD7DAD4093721150937311609342
:1013B000741170937511AC0160E070E040937E1180
:1013C00050937F1160938011709381114A8D5B8DD2
:1013D0006C8D7D8D40937A1150937B1160937C11BD
:1013E00070937D114EA95FA968AD79AD40938211CC
:1013F00050938311609384117093851121E030E044
:1014000002C020E030E0088D198D8017910770F53B
:101410004EA95FA968AD79AD2115310541F440931E
:101420007211509373116093741170937511F901D7
:10143000EE0FFF1FE20FF31FEE0FFF1FEE0FFF1F58
:10144000E658FE4ED801A81BB90BCD01A0E0B0E0D4
:1014500084839583A683B7831082118212821382BC
:1014600040875187628773872F5F3F4F8C899D89A3
:1014700008171907E8F52115310561F48AAD9BAD10
:10148000ACADBDAD8093721190937311A0937411A4
:10149000B0937511F901EE0FFF1FE20FF31FEE0F6E
:1014A000FF1FEE0FFF1FE658FE4E8FEF9FE7A0E0F5
:1014B000B0E084839583A683B7838A8D9B8DAC8DA2
:1014C000BD8DB095A095909581959F4FAF4FBF4F23
:1014D00080839183A283B383DE01DE968D919D91FB
:1014E0000D90BC91A02D80879187A287B38715C0EE
:1014F00021503040F901EE0FFF1FE20FF31FEE0FF6
:10150000FF1FEE0FFF1FE658FE4E8FEF9FE7A0E094
:10151000B0E084839583A683B783CA5BDF4F88815D
:101520008F7D88838091721190917311A0917411B5
:10153000B09175110097A105B10521F41092F71132
:1015400080E08FC080916011833010F40E9473841A
:101550000E94EB8681E090E0A0E0B0E08093611112
:1015600090936211A0936311B093641110925C1177
:1015700010925D1110925E1110925F11C701A0E0F0
:10158000B0E08093F3119093F411A093F511B09310
:10159000F6118091F3119091F411A091F511B09191
:1015A000F6118093EF119093F011A093F111B09385
:1015B000F2118091F3119091F411A091F511B09175
:1015C000F611B595A79597958795B095A0959095A7
:1015D00081959F4FAF4FBF4F8093BC119093BD112A
:1015E000A093BE11B093BF118093C0119093C1110D
:1015F000A093C211B093C3118093C4119093C511ED
:10160000A093C611B093C7118093C8119093C911CC
:10161000A093CA11B093CB118093CC119093CD11AC
:10162000A093CE11B093CF1181E08093F7118091F8
:10163000B0119091B111A091B211B091B311813A52
:10164000EFE09E07E0E0AE07E0E0BE071CF080E0C0
:1016500098E002C080E090E19093290180932801F6
:1016600081E0DF91CF911F910F91FF90EF9008954E
:101670000F931F93962FB9010FEF1FEF2FEF3FE747
:101680000093EF111093F0112093F1113093F211A8
:1016900001E010E020E030E00093F3111093F4112A
:1016A0002093F5113093F6118B019A010093691183
:1016B00010936A1120936B1130936C1120E038E085
:1016C00030932901209328014FEF5FEF6FEF7FEFF9
:1016D0004093BC115093BD116093BE117093BF1124
:1016E0001092A8111092A9111092AA111092AB1188
:1016F0004093C0115093C1116093C2117093C311F4
:101700001092AC111092AD111092AE111092AF1157
:101710004093C4115093C5116093C6117093C711C3
:101720001092B0111092B1111092B2111092B31127
:101730004093C8115093C9116093CA117093CB1193
:101740001092B4111092B5111092B6111092B711F7
:101750004093CC115093CD116093CE117093CF1163
:101760001092B8111092B9111092BA111092BB11C7
:1017700090FF28C08093A3112091E411222329F027
:101780002091A31131E0232702C02091A31122232D
:1017900011F0889A01C088988A9841E050E060E092
:1017A00070E04093A8115093A9116093AA1170930F
:1017B000AB112091A311222311F021E001C02FEFE2
:1017C00020939E1191FF28C08093A4112091E511D0
:1017D000222329F02091A41131E0232702C0209177
:1017E000A411222311F08C9A01C08C988E9841E0AC
:1017F00050E060E070E04093AC115093AD11609305
:10180000AE117093AF112091A411222311F021E0A9
:1018100001C02FEF20939F1192FF32C08093A5113A
:101820008091E611882329F08091A51191E0892704
:1018300002C08091A511882321F080910801816068
:1018400003C0809108018E7F809308018091080178
:101850008B7F8093080181E090E0A0E0B0E080936E
:10186000B0119093B111A093B211B093B3118091C4
:10187000A511882311F081E001C08FEF8093A011A2
:101880008091691190916A11A0916B11B0916C11C6
:1018900080935C1190935D11A0935E11B0935F11E2
:1018A00081E080935A111F910F9108958230C1F009
:1018B000833028F4882341F0813039F50BC0833020
:1018C000C9F0843011F51CC0662311F48A9A08957A
:1018D0008A980895662311F48E9A08958E98089533
:1018E00080910801662311F4846001C08B7F80938E
:1018F00008010895662311F4149A08951498089520
:10190000662311F4A29A0895A2980895823081F076
:10191000833028F4882361F08130B9F405C0833026
:1019200059F0843091F40CC081E07E9B0EC00BC056
:1019300081E07A9B0AC007C081E0049B06C003C017
:1019400081E0929B02C080E008950895853078F48C
:10195000282F30E0C901880F991F820F931F880F2D
:10196000991F880F991F88509E4E0E945EAD089562
:101970008091F711882319F481E08093F71108957D
:1019800020910901221F2227221F2295220F207E4B
:101990008091090186FF02C050E101C050E04091F2
:1019A0000901909109013091090180910901947018
:1019B0004870942B3270932B8170892B822B852B4E
:1019C00008958F929F92AF92BF92CF92DF92EF9243
:1019D000FF920F931F93CF938091F711882309F4FF
:1019E000C7C38091571190915811009729F40E9414
:1019F0006F89882309F4B9C380915C1190915D11BE
:101A0000A0915E11B0915F1180509140A040B04014
:101A100080935C1190935D11A0935E11B0935F1160
:101A200080915C1190915D11A0915E11B0915F1158
:101A3000B7FF16C380915C1190915D11A0915E116A
:101A4000B0915F114091691150916A1160916B11D1
:101A500070916C11840F951FA61FB71F80935C11A6
:101A600090935D11A0935E11B0935F1181E090E0BF
:101A7000A0E0B0E0C82F40915C1150915D116091E1
:101A80005E1170915F1177FF2FC08C019D01409115
:101A9000EF115091F0116091F1117091F2110196D6
:101AA000A11DB11D0417150726073707ECF4409157
:101AB0005C1150915D1160915E1170915F11009108
:101AC000691110916A1120916B1130916C11400FC6
:101AD000511F621F731F40935C1150935D116093FF
:101AE0005E1170935F11C6CF8091A8119091A911DA
:101AF000A091AA11B091AB110097A105B10571F0A9
:101B00008091A311882331F080910901E1E081FDEA
:101B100006C004C080910901E1E080FFE0E080910F
:101B2000AC119091AD11A091AE11B091AF11009791
:101B3000A105B10571F08091A411882331F0809145
:101B4000090131E083FD06C004C08091090131E044
:101B500082FF30E08091B0119091B111A091B2114B
:101B6000B091B3110097A105B10571F08091A51155
:101B7000882331F020910901221F2227221F05C04E
:101B80008091090121E086FF20E0C090B411D0903F
:101B9000B511E090B611F090B7118090B811909007
:101BA000B911A090BA11B090BB11F0E00C2F112721
:101BB00007FD1095F9C1EE2309F45FC08091BC11B7
:101BC0009091BD11A091BE11B091BF114091A8118B
:101BD0005091A9116091AA117091AB11840F951FBA
:101BE000A61FB71F8093BC119093BD11A093BE1187
:101BF000B093BF118091BC119091BD11A091BE1105
:101C0000B091BF11B7FD39C0899A8091BC119091F4
